:10000000E47F001079050000830500001DBF020099
:1000100087050000890500008B05000068A5FCEF3E
:100020000000000000000000000000008D0500003E
:100030008F050000000000009105000093050000FE
:100040009505000097050000990500009B0500003C
:100050009D0500009F050000A1050000A30500000C
:10006000A5050000A7050000A9050000AB050000DC
:10007000AD05000000000000AF050000B105000064
:10008000B3050000B5050000B7050000B905000084
:10009000BB050000BD050000BF0500004989020046
:1000A000C3050000C5050000C7050000C905000024
:1000B000CB050000CD050000CF050000D1050000F4
:1000C000D3050000D5050000D7050000D9050000C4
:1000D000DB050000DD050000DF050000E105000094
:0400E000E305000034
:10010000DECEA5ED02003078343038380000000033
:10011000000000000000484D49343330000000006A
:1001200000000000000053696D706C65484D490087
:1001300000000000000000000000000000000000BF
:100140000000000000000507FE00DAF7DECEA5ED96
:100150000200307834303838000000000000000021
:10016000000053504C6174436F6E74726F6C6C6519
:1001700072004170706C69636174696F6E00000099
:10018000000000000000000000000000000000006F
:0801900000000000FE00DAF798
:0802FC002143658700000000AA
:1003040081000200140000006125020014000000B6
:10031400513E020014000000294002000F000000BA
:10032400B940020018000000054302001300000059
:10033400D564020013000000AD6A0200130000003F
:10034400897102001700000091760200FA00000093
:10035400A97902000A0000007D8902000100000062
:10036400958A02000D0000003D8D02000C00000083
:10037400E590020000000000419602000900000020
:100384008D96020005000000119802000400000090
:10039400F99A02000400000049A3020002000000D0
:1003A40001A502001E00000041AE02001000000082
:1003B400A1B902000E0000007DBD02000300000090
:1003C400BDC302000600000021C7020014000000A3
:1003D40039E203001200000025EE03000A000000C9
:1003E40079F203000A00000085FA030014000000FB
:1003F4004500040008000000F90A0400170000008A
:100404000D46040007000000B54C04001000000075
:10041400A15104001300000035650400130000001E
:10042400199904001600000065F904001700000083
:100434001533050016000000E53305001700000021
:080444006D45050015000000E4
:10044C002F49072291438D462E492F480A1A06D070
:10045C000722914381F30988022282F314882B48E6
:10046C002B492C4A00F039F82B482C492C4A00F027
:10047C0034F82C482C492D4A00F02FF82C482D49E3
:10048C002D4A00F02AF82D482D492E4A00F025F867
:10049C002D482E492E4A00F020F82E482E490022D5
:1004AC0000F026F82D482E49091A082903DB0022F2
:1004BC000260043001601F481F49884205D0026861
:1004CC00043003B4904703BCF7E700208646EC46A3
:1004DC0000200021234A9047FEE7884207D0521A99
:1004EC0005D0037801300B700131013AF9D1704716
:1004FC00884202D002700130FAE770471A48704700
:10050C00E47F0010E48F0010E47F001020DA060076
:10051C00E8000010080200100000020000000200B9
:10052C00C816060020DA0600E8000010E8000010EB
:10053C00EC050000EC050000EC050000EC050000EB
:10054C00EC050000EC050000181806001818060051
:10055C0020DA060008020010907B0010DC7B0010F3
:10056C00E47B0010F19C0200FFFFFFFF1A481B49BF
:10057C000160FFF765BFFEE7FEE7FEE7FEE7FEE77B
:10058C00FEE7FEE7FEE7FEE7FEE7FEE7FEE7FEE737
:10059C00FEE7FEE7FEE7FEE7FEE7FEE7FEE7FEE727
:1005AC00FEE7FEE7FEE7FEE7FEE7FEE7FEE7FEE717
:1005BC00FEE7FEE7FEE7FEE7FEE7FEE7FEE7FEE707
:1005CC00FEE7FEE7FEE7FEE7FEE7FEE7FEE7FEE7F7
:1005DC00FEE7FEE7FEE7FEE708ED00E000000000A6
:020000021000EC
:1000000000000000000000000000000000000000F0
:1000100000000000000000000000000000000000E0
:1000200000000000000000000000000000003F4B46
:10003000F4033DFD00000083199F833BC50F01863B
:1000400000004A8601004A6800202906AA005729B4
:100050000755005780006BF40300DB000000F60238
:10006000FC022DF602FD023D800077831A7A831B85
:1000700038831C40831CF6F430F10500F0030000C7
:100080000B09F00000000B09F00700000BF106005F
:100090009900000000F61F3C93980000007E09962E
:1000A0001CF610FB020164F609FB0402F610FB07C4
:1000B0000202300230020309F00001000C09F007CF
:1000C00000000CF106000999A3D70A7890F1050009
:1000D000F00300000CF00000000C0983192EF6104C
:1000E000FB1801405C43484D49343330204661637E
:1000F000746F7279205465737403F610FB0D0165FB
:100100000227464630303030303003F00600C085DC
:10011000F10101F10100F610FB0D01405C6E466932
:10012000726D776172653AEF4445EF4545F60AFB1B
:10013000F610FB012EEF4446EF454601F60AFBF6AA
:1001400010FB0103EF4545F40EF406F402600320B2
:100150000159F4070000C8014B83192EF610FB105B
:1001600001405C43546F75636873637265656E0329
:10017000F610FB0D01650227464630303030303036
:100180000383199FF10A0001F00100000AF610FB39
:100190003C01405C6E546F75636820746865207420
:1001A0006F75636873637265656E2E2020446F659A
:1001B000732069745C6E7265717569726520726511
:1001C00063616C6962726174696E673F03F610FB6C
:1001D0002B0150310234023002332E3802392E38CE
:1001E00002526563616C0202020202020227464665
:1001F0003130313031300202020E0203F610FB07BB
:1002000001463130023003F610FB2201404F7220CC
:100210006A756D7020737472616967687420746F99
:1002200020746865205254432063616C03F610FB10
:100230002C0150023132023002332E3802392E386E
:1002400002446F2052544302020202020202274675
:10025000463130313031300202020F0203F40260C5
:10026000022002816004200281600320028180025A
:100270005DF610FB0401530203F00000000A800148
:1002800059F10A0000F00100000A600220027160CA
:100290000420150B83192EF610FB1401405C433328
:1002A00056332063616C6962726174696F6E03F624
:1002B00010FB0D01650227464630303030303003E8
:1002C000830088F610FB1401405C6E4578697374F6
:1002D000696E672043616C203D2003F610FB11011D
:1002E000666E6F726D616C626F6C642E666F6E030A
:1002F000F62DF610FB020140EF4445EF4545810322
:1003000009F609FB0503800312F610FB05556E6321
:10031000616CF610FB0103EF454582032298000053
:10032000007E961CF610FB11016673797364656696
:1003300061756C742E666F6E03F610FB0E01405CE7
:100340006E4E65772043616C203D03F610FB2A0159
:10035000500233023002332E3802392E38025570E3
:100360000272323002020202020227464631303166
:10037000303130020202100203F610FB2C01500251
:1003800037023002332E3802392E3802446F776E2E
:100390000272323002020202020227464631303136
:1003A000303130020202110203F610FB2B01500221
:1003B0003302313002372E380231312E3802536188
:1003C00076650202020202020227464630304646A5
:1003D0003030020202120203830423F4026003207D
:1003E000043D8003DBF610FB1101666E6F726D61D8
:1003F0006C626F6C642E666F6E03F610FB0701462D
:100400003202313003F610FB020140EF9647941C94
:10041000F609FB0503F610FB0103EF944709990366
:10042000126F75941C90961C8300798003E5998364
:10043000126F758004238300826803200983192EBC
:10044000F610FB23016330250230250233332E33AF
:100450002502323025020301650227464630383036
:1004600030303003015203F610FB1A0163023230C0
:100470002502020203016502274646313030303042
:100480003003015203F610FB1A01630234302502D7
:100490000202030165022746463230303030300315
:1004A000015203F610FB1A016302363025020202E4
:1004B00003016502274646343030303030030152A4
:1004C00003F610FB1A016302383025020202030111
:1004D000650227464638303030303003015203F68B
:1004E00010FB24016333332E332502302502023101
:1004F000362E363725020301650227464630303056
:1005000034303003015203F610FB1D016302313613
:100510002E36372502020203016502274646303097
:100520003038303003015203F610FB1D01630233F3
:10053000332E33342502020203016502274646307A
:10054000303130303003015203F610FB1A016302E0
:10055000353025020202030165022746463030325B
:1005600030303003015203F610FB1D0163023636B2
:100570002E36382502020203016502274646303036
:100580003430303003015203F610FB1D0163023892
:10059000332E333525020202030165022746463019
:1005A000303830303003015203F610FB210163363E
:1005B000362E36250230250202323025020301652F
:1005C0000227464630303030303803015203F610EF
:1005D000FB1A016302323025020202030165022781
:1005E000464630303030313003015203F610FB1AEA
:1005F00001630234302502020203016502274646E8
:1006000030303030323003015203F610FB1A0163F0
:1006100002363025020202030165022746463030C9
:100620003030343003015203F610FB1A01630238F4
:100630003025020202030165022746463030303081
:10064000383003015203F610FB0E01633002300212
:100650003102313030250203F610FB0D016502270F
:10066000464630303030433003F610FB030152036E
:10067000F610FB03016303F610FB0F01405C434CD3
:1006800043442052474235363503F610FB140150DF
:10069000300202020202020202020202020202020C
:1006A0000203F40261032006A283192EF610FB1A3E
:1006B00001405C434C434420436F6C6F75722026AD
:1006C00020436F6E747261737403F610FB0D016545
:1006D0000227464630303030303003F610FB13012D
:1006E000633525023025023430250231322E35257E
:1006F0000203F610FB0D016502274646303030300C
:10070000303003F610FB03015203F610FB160163B1
:1007100035250231322E3525023430250231322E74
:1007200035250203F610FB0D0165022746463234DB
:100730003234323403F610FB03015203F610FB147B
:100740000163352502323525023430250231322E3F
:1007500035250203F610FB0D0165022746463438A5
:100760003438343803F610FB03015203F610FB163D
:10077000016335250233372E352502343025023109
:10078000322E35250203F610FB0D01650227464681
:1007900036433643364303F610FB03015203F6108B
:1007A000FB14016335250235302502343025023132
:1007B000322E35250203F610FB0D01650227464651
:1007C00039303930393003F610FB03015203F6108B
:1007D000FB16016335250236322E352502343025CD
:1007E0000231322E35250203F610FB0D016502277A
:1007F000464642344234423403F610FB03015203AE
:10080000F610FB14016335250237352502343025F7
:100810000231322E35250203F610FB0D0165022749
:10082000464644394439443903F610FB0301520368
:10083000F610FB16016335250238372E35250234B4
:1008400030250231322E35250203F610FB0D0165ED
:100850000227464646464646464603F610FB030137
:100860005203F610FB14016334352502302502349F
:1008700030250231322E35250203F610FB0D0165BD
:100880000227464646464646464603F610FB030107
:100890005203F610FB1701633435250231322E3531
:1008A00025023430250231322E35250203F610FBA5
:1008B0000D01650227464643303030303003F610D4
:1008C000FB03015203F610FB150163343525023298
:1008D0003525023430250231322E35250203F6103B
:1008E000FB0D01650227464643304330303003F6A6
:1008F00010FB03015203F610FB1701633435250288
:1009000033372E3525023430250231322E3525027B
:1009100003F610FB0D0165022746463030433030A8
:100920003003F610FB03015203F610FB150163348C
:10093000352502353025023430250231322E352559
:100940000203F610FB0D01650227464630304330A6
:10095000433003F610FB03015203F610FB1701634B
:100960003435250236322E35250234302502313217
:100970002E35250203F610FB0D0165022746463091
:10098000303030433003F610FB03015203F610FB06
:1009900015016334352502373525023430250231FF
:1009A000322E35250203F610FB0D0165022746465F
:1009B00043303030433003F610FB03015203F6108E
:1009C000FB1701633435250238372E3525023430C4
:1009D000250231322E35250203F610FB0D0165028A
:1009E00027464630303030303003F610FB030152DA
:1009F00003F40261032009F183192EF610FB200194
:100A00005030023002300231303025023130302592
:100A1000020268310202020202020202020203F62C
:100A200010FB0D01650227464646464646464603EC
:100A3000F610FB03015203F4026103200A37831905
:100A40002EF610FB200150300230023002313030DF
:100A50002502313030250202683102020202020210
:100A60000202020203F610FB0D016502274646460C
:100A7000463030303003F610FB03015203F40261BC
:100A800003200A7D83192EF610FB2001503002301E
:100A90000230023130302502313030250202683117
:100AA0000202020202020202020203F610FB0D0120
:100AB000650227464630304646303003F610FB03C9
:100AC000015203F4026103200AC383192EF610FBBE
:100AD00020015030023002300231303025023130F6
:100AE0003025020268310202020202020202020200
:100AF00003F610FB0D0165022746463030303043C7
:100B00003003F610FB03015203F4026103200B09CA
:100B100083192EF610FB1001405C43446967697429
:100B2000616C20492F4F03F610FB0D01650227462B
:100B30004630303030303003F610FB1801503002B0
:100B4000020202020268316431020202020202025F
:100B500002020203F610FB0E01633102300233027F
:100B6000313030250203F610FB03015203F610FB6F
:100B700003016303F610FB050146310203F610FB87
:100B80001C014054657374696E672C20706C65613C
:100B9000736520776169742E2E2E5C6E03B900B7E1
:100BA000001E000014B200820BD0BAF610FB060142
:100BB0004042697420EF4445EF4545F60AFBF610C4
:100BC000FB08206661696C656403EF4545800C2174
:100BD0004F00500054810C97F610FB1D0140556EDC
:100BE00065787065637465642061637469766520F7
:100BF000696E7075743A5C6E03F610FB0701404F26
:100C0000503D25034F004A08831A00F610FB0801E7
:100C1000402049503D250350004A08831A00800CAB
:100C200021F610FB18015030020202020202683065
:100C300064300202020202020202020203F610FB08
:100C40002B0150310234023002332E3802392E3853
:100C500002526574727902020202020202274646BB
:100C60003130313031300202020E0203F4026003EF
:100C7000200CB06102200C6C690220F610FB1501FB
:100C80005031020202023002020202020202020299
:100C900002020203800B38B800BCBA87080B9FF62B
:100CA00010FB0D0140492F4F20616C6C206F6B03CE
:100CB0004A004AFF51001E00006483192EF610FB03
:100CC0000B01405C4342656570657203F610FB0DD5
:100CD00001650227464630303030303003F610FBD5
:100CE0002801405C6E5072657373204E65787420E5
:100CF0006966207468652062656570657220697335
:100D00002062656570696E67035808F4026103200C
:100D10000D0B430883192EF610FB1A01405C434269
:100D200061636B6C696768742063616C696272618E
:100D300074696F6E03F610FB0D016502274646309D
:100D40003030303030038300BE961CF610FB1401A7
:100D5000405C6E4578697374696E672043616C20EE
:100D60003D2003F610FB1101666E6F726D616C62BF
:100D70006F6C642E666F6E03AA0D8EF610FB020177
:100D800040F609FB0402F610FB0103800D99F610F2
:100D9000FB0701404E6F6E65038300B898000000AA
:100DA0007F83009FF610FB1101667379736465669B
:100DB00061756C742E666F6E03F610FB0E01405C5D
:100DC0006E4E65772043616C203D03F610FB3001C9
:100DD000500233023002332E3802392E380242726A
:100DE000696768746572027232300202020202029E
:100DF000274646313031303130020202130203F609
:100E000010FB2E01500237023002332E3802392EE9
:100E1000380244696D6D657202723230020202025C
:100E200002022746463130313031300202021402CC
:100E300003F610FB2B0150023302313002372E38FB
:100E40000231312E3802536176650202020202023B
:100E50000227464630304646303002020215020371
:100E6000830E6DF4026003200EE2800E63F610FB29
:100E70001101666E6F726D616C626F6C642E666FCD
:100E80006E03F610FB0701463202313003F610FB09
:100E9000020140EF9647941CF609FB0402F610FB92
:100EA0000103EF944709941C9923D70A789099007D
:100EB00000007FF61D0EBC980000007F83009F801D
:100EC0000E6D941C99A3D70A78909900000000F643
:100ED0001F0EBC9800000000800EBC8300C7680392
:100EE000200983199F83192EF610FB0F01405C43E4
:100EF000416E616C6F677565205403F610FB0D0140
:100F0000650227464630303030303003983851EC97
:100F10007BAF00F610FB0D016527464639303930AE
:100F200039300203F610FB7201405C6E506C656153
:100F3000736520696E736572742054206C696E6BE2
:100F40007320616E645C6E696E7374616C6C207486
:100F50006865207465737420706C75672E5C6E28EC
:100F6000416E4F757420746F20416E496E3120615F
:100F70006E64207669612034375220746F20416E90
:100F8000496E302E295C6E4E657874207768656EE8
:100F90002072656164792E2E2E03F40C0320690300
:100FA000208311C6F610FB0A0140302E3330325C2C
:100FB0006E03F610FB080140302E323937038F44A0
:100FC000001E00000A6003200FFCF610FB0A0163FC
:100FD0003702313702020203B900981AFBA07D8361
:100FE000122CB9019818129D7D83122CF610FB0368
:100FF0000163032944030FC11E00006483192EF608
:1010000010FB0F01405C43416E616C6F677565209A
:101010004903F610FB0D016502274646303030309B
:10102000303003984569757CAF00F610FB0D016503
:101030002746463930393039300203F610FB3D017E
:10104000405C6E506C65617365206D6F7665206CD9
:10105000696E6B7320746F20746865204920706F0F
:10106000736974696F6E2E5C6E4E65787420776854
:10107000656E2072656164792E2E2E03F40C0320B8
:101080006903208311C6F610FB0A0140302E32316D
:10109000395C6E03F610FB080140302E3238310304
:1010A0008F44001E00000A60032010DEF610FB0AC9
:1010B00001633702313702020203B90098600D1B49
:1010C0007C83122CB901980FDF3B7D83122CF61024
:1010D000FB0301630329440310A31E00006483196A
:1010E0002EF610FB0F01405C43416E616C6F67751B
:1010F00065205603F610FB0D016502274646303089
:101100003030303003980000007EAF00F610FB0D49
:1011100001652746463930393039300203F610FB75
:101120003D01405C6E506C65617365206D6F766546
:10113000206C696E6B7320746F2074686520562074
:10114000706F736974696F6E2E5C6E4E6578742073
:101150007768656E2072656164792E2E2E03F40C1B
:1011600003206903208311C6F610FB080140302ECE
:10117000355C6E03F610FB060140302E35038F44BC
:10118000001E00000A60032011BCF610FB0A016378
:101190003702313702020203B900980000007E8353
:1011A000122CB901980000007E83122CF610FB036C
:1011B00001630329440311811E00006498000000AC
:1011C00000AF00801265F610FB06014636023003C0
:1011D000F610FB1D014020202020202020457870A3
:1011E0006563743A202020536565696E673A5C6ECA
:1011F00003F610FB0B0140416E496E303A5C6E0302
:10120000F610FB090140416E496E313A03F610FBBE
:101210000D01652746464646464646460203F610F9
:10122000FB0901633702370202020309EE60004442
:101230003C939923D70A788319B701EE660044825C
:101240001255F610FB020140F609FB0503F610FBF0
:10125000035C6E0309F610FB0B014050617373656C
:10126000645C6E030983192EF610FB0F01405C438A
:1012700054544C2053657269616C03F610FB0D01E8
:10128000650227464630303030303003F610FB3BE5
:1012900001405C6E436F6E6E656374206120274E63
:1012A000554C4C204D4F44454D27206361626C6581
:1012B0005C6E6265747765656E20746865203220A7
:1012C00054544C20706F7274732E03F610FB1D0182
:1012D000405C6E434F4D30202D3E20434F4D313A00
:1012E0002054657374696E672E2E2E03F40260031A
:1012F0002013AB4AFFF637FDF610FC0731323334CA
:101300002E350D1E0000054A0DF636FD86FF12EC47
:10131000F63BFDFF991A500089F6258112ECF61074
:10132000FB06014602313403F610FB0D014050610B
:10133000737320202020202003F610FB1D01405C49
:101340006E434F4D31202D3E20434F4D303A2054B7
:10135000657374696E672E2E2E03F40260032013EA
:10136000AB4AFFF637FCF610FD073637382E32351C
:101370000D1E0000054A0DF636FC86FF135AF63B9B
:10138000FCFF9929900088F62581135AF610FB0678
:10139000014602313403F610FB0D014050617373B6
:1013A000202020202020031E00006483192EF61028
:1013B000FB1401405C4354544C20587769726520FB
:1013C000262034383503F610FB0D0165022746460A
:1013D00030303030303003F610FB4401405C6E4357
:1013E0006F6E6E656374206120484D493433302040
:1013F00077697468207468652058776972652F343E
:1014000038352074657374206170702E5C6E587767
:10141000697265203D5C6E5253343835203D03F5CA
:10142000320010F602FE024D690520690620980080
:1014300000000096344AFFF637FE9816B4389396AB
:1014400030F5390060052014B5F610FB060146336F
:10145000023803985781C093F610FE0120F608FE6B
:101460000907F610FE010D99A000008292ABF40668
:101470001E0000014A0DF636FE87FF1487F40700B0
:10148000000A1470801499F63BFEFF4A0DF636FEF2
:101490000CF637FEF6258214A7F610FB070140462E
:1014A00061696C038014B5F610FB0701405061734D
:1014B000730368052060062014EFF610FB06014652
:1014C00032023803943099A0000082929534F625B8
:1014D0008214E1F610FB0701404661696C03801439
:1014E000EFF610FB0701405061737303680620603C
:1014F00003201505670520670620048215051E00D8
:101500000005801444F5361E00003283192EF610B3
:10151000FB1401405C435254432043616C69627286
:101520006174696F6E03F610FB0D01650227464674
:1015300030303030303003831A5CF610FB11016616
:1015400073797364656661756C742E666F6E03F6ED
:1015500010FB1901405C6E4578697374696E6720F1
:1015600063616C2076616C7565203D20F609FB0790
:1015700000F610FB0103F610FB0E0163320230028D
:101580003202313030250203F610FB03015203F61C
:1015900010FB250140506C6561736520636F6E6EB2
:1015A0006563742074686520475053206F736369C6
:1015B0006C6C61746F722E03F610FB03016303F40D
:1015C00002831A538215EB600320186D8015BFF655
:1015D00010FB18015030020202020202683164312D
:1015E0000202020202020202020203F610FB0E01D4
:1015F00063320230023202313030250203F610FB32
:1016000003015203F610FB19014057616974696EBA
:101610006720666F722073746162696C6974792ED9
:1016200003F610FB030163031E000032F610FB06F5
:10163000014632023003F406F402831A5381150B7B
:10164000F4070000C81638F610FB180150300202EB
:101650000202020268316431020202020202020244
:10166000020203F610FB0E01633202300232023135
:101670003030250203F610FB03015203F610FB2065
:101680000140506572666F726D696E6720525443F7
:101690002063616C6962726174696F6E2E2E2E0315
:1016A000F610FB03016303831A44F402831A4A0110
:1016B000860116AAF610FB0E0163320230023502D3
:1016C000313030250203F610FB03015203F610FB04
:1016D00003016303F610FB0501463202030816E816
:1016E00016AA171A175E179E831A65F610FB1E01BD
:1016F0004043616C6962726174696F6E206F6B2127
:101700005C72475053206379636C65733DF609FB47
:101710000800F610FB01038017D6831A65F610FB4C
:101720001801404E6F204750532031304D487A2CDD
:1017300020636F756E74656420F609FB0800F6106F
:10174000FB195C72507265737320627574746F6EEE
:1017500020746F2072657472792E038017EEF61074
:10176000FB3901404661696C656420746F207772B3
:101770006974652063616C20746F20454550524F39
:101780004D2E5C72507265737320627574746F6E47
:1017900020746F2072657472792E038017EE831A9D
:1017A00065F610FB24014043616E27742063616C71
:1017B00020616E79206265747465722E5C72475088
:1017C00053206379636C65733DF609FB0800F610DE
:1017D000FB01038017D6831A5CF610FB070140203B
:1017E00043616C3DF609FB0800F610FB0103690339
:1017F00020690220F610FB1801503002020202029A
:101800000268306430020202020202020202020393
:10181000F610FB2B0150310234023002332E380215
:10182000392E3802526574727902020202020202F3
:101830002746463130313031300202020E0203F4C5
:1018400002600320186D61022017EEF610FB1501EF
:1018500050310202020230020202020202020202BD
:1018600002020203831A5381157680164783192ECC
:10187000F610FB1501405C4354657374696E672074
:10188000436F6D706C65746503F610FB0D016502A6
:1018900027464630303030303003F610FB460140EA
:1018A0005C6E45697468657220275265746573744F
:1018B00027206F7220274E65787427207361766524
:1018C00020726573756C745C6E616E6420746F2039
:1018D0007374617274207468652064656D6F206133
:1018E00070702E03F610FB2C0150310233023002CF
:1018F000332E3802392E3802526574657374020231
:1019000002020202022746463130313031300202F3
:10191000020E0203F40260022000DB6103201914AE
:101920008F06AA8F07550EF436F402801929690331
:1019300020690220690420F610FB0401530203F61B
:1019400010FB2A015030022D33022D3130023302B8
:101950003130024E6578740202020202020227460A
:1019600046313031303130020202160203F610FBEC
:101970000E0163300230023102313030250203F6AD
:1019800010FB0D01650227464630303030433003EE
:10199000F610FB03015203F610FB0301630309F683
:1019A00010FB130164302E3802302E3202313230F7
:1019B00002333002310309F10500F107044A0099AE
:1019C000000000001E000002EEAE0090AB0C018A89
:1019D0000A19C4982000008293F105088319E3F1E5
:1019E000060809F10800919AF108044AFFF61D3C27
:1019F000934A000968032009680220096804200945
:101A000003F1020ABB4A01BDBF1A0F57801A07F142
:101A1000020BF402F1010AF1010B5206064A0152CF
:101A2000F610FB020140EF4445EF4545F60AFBF690
:101A300010FB0103EF4545F1010B5601F1020B8745
:101A4000801A1209F00000200009F005002000F1C2
:101A5000010009F005012000F1010009F007002054
:101A600000F1060009F007012000F1060009150B3E
:101A70002A0B031A788F0B000E09F4031A89000051
:101A800000F4031AA7000000091E00000294389910
:101A90006666667E929638AE01994CCCCD7B929567
:101AA00038909638801A89170B1AB11B021ACC1A73
:101AB000DFF610FB140164312E3002302E33350274
:101AC000313230023630300203801AF2F610FB0C4D
:101AD0000164302E3102023002300203801AF2F625
:101AE00010FB0C0164312E30020230023002038000
:101AF0001AF2450B1E00001401450B12811AF480E6
:101B00001AA7290B011AA71E000014943899000087
:101B1000007F91993333337E929919999A7D90F68B
:101B200010FB020164F609FB0402F610FB07020237
:101B30003002300203801B02F4031B400000000946
:101B400045154A001206410245154A041206410392
:101B50005D001B5F5D011B6A1E000005801B4028A5
:101B600015001B75831D81801B752815041B75834B
:101B7000350E801B75F610FB07016402020202039A
:101B8000801B4099CCCCCD7AAA1B90994CCCCD7AB5
:101B900090961CAB980000007F833CA6F10504954D
:101BA0001C91992000008292AB980000007F833C3A
:101BB000A6961CF1060409F4031BBF00000009F4FB
:101BC00002801BBF944099F0000083F61D1BE19931
:101BD00048000085F61F1BE16100063C93831BFB58
:101BE0000998F9F99A880999800000849099200051
:101BF000008192AB98100000829309991000008236
:101C000092AB982000008193990000008490099481
:101C1000076000061C299920000082F61C1C3C99D4
:101C200020000084F61E1C3C099948000084F61C24
:101C30001C3C9974000085F61E1C3C099796070908
:101C4000F4031CB4000000F4031C52000000831CC9
:101C50000F09831CAA963C1E000005943C996666F9
:101C6000667E92963C831CAA994CCCCD7B92953C87
:101C700090963C9540919A994CCCCD7BF61C1C5784
:101C8000943C992000008292998000007EAA1C95C5
:101C9000990000007E90AB980000007F833CA699DD
:101CA0004CCCCD7B929640801C57AE00F303025D76
:101CB000833DCF091E00000A831BC4AB9407919992
:101CC0004CCCCD7BF61F1CD499CCCCCD7BF61D1C07
:101CD000E5801CB46101061CDB42056102061CE2C2
:101CE0004204801CB46101061CEC43056102061C21
:101CF000F34304801CB4833BC5F4031D01000000C2
:101D000009831D8162002127BFF610FB0D015302DC
:101D10002746463030303030300369072017151D14
:101D20008622D9314B27DE3513441568072009F682
:101D300010FB0D016670726F7032352E666F6E0388
:101D4000F610FB1601652746464530453045300202
:101D500027464636303630363003F610FB12016324
:101D60003070780230707802310231303025020351
:101D7000F610FB03015203090BF40E094A00801D03
:101D8000294A00801D298F18FF8F19FFF610FB0DBF
:101D900001530227303030303030303003F610FB42
:101DA000080164020202023103F610FB2601500210
:101DB00030707802307078023237327078023438FE
:101DC000307078020268310202020202020202024C
:101DD0001702031E00000A6007201DE883203E83CF
:101DE0001DFA832205801DD3F610FB080164020250
:101DF00002023003801D048022D4F610FB0401612E
:101E00003103F411F41F451812812033F41F4418D4
:101E1000F610FB0E016670726F703231302E666FF5
:101E20006E03F610FB160163307078023070780292
:101E3000313730707802313030250203F610FB164E
:101E400001652746464646464646460227464630F0
:101E5000303030303003F610FB03015203F41BF432
:101E60001DF610FB080146300235707803F610FBB2
:101E70001601652746464646464646460227303006
:101E800030303030303003F610FB020140EF444573
:101E9000EF4446EF45460188091EA0F610FB0130CD
:101EA000EF454601F60AFBF610FB013AEF4545887F
:101EB000091EB8F610FB0130EF4545F60AFBF61097
:101EC000FB0103EF4545F610FB03016303F3030237
:101ED00019F31102F41D9FAB9820000082833C94FB
:101EE0009EF30BF30900F30A0000F31104F3190049
:101EF000F32104F610FB0F01666C656473656733AC
:101F0000352E666F6E03F610FB16016527464646B2
:101F1000463030303002273030303030303030030F
:101F2000F610FB02014697F609FB030097F610FB3B
:101F300003707802F609FB0300F610FB03707803C8
:101F4000F41FF610FB020140EF4445EF45458809B8
:101F50001F57F610FB0130EF4545F60AFBF610FB64
:101F60000103EF4545F610FB0D016670726F703787
:101F7000302E666F6E03F610FB1401630233707827
:101F80000231023130302502313138707803F610D9
:101F9000FB160165274130303030303030022730B9
:101FA0003030303030303003F423F610FB04014081
:101FB0005C43F3030073EF4445EF4545F30BF31126
:101FC00002F30900F31100F630FBF610FB0103EFFA
:101FD0004545F610FB14016302307078023102317E
:101FE00030302502313135707803F610FB1601656B
:101FF00027383030304330453002273030303030F1
:1020000030303003F610FB0401405C43F3030073EF
:10201000EF4445EF4545F30BF31102F30900F311CB
:1020200000F630FBF610FB0103EF4545F610FB030D
:10203000016303F610FB0401613003F40209F41993
:10204000F41F4519120AF41F4419F610FB0301523C
:1020500003F610FB0E01666D6F6E6F3132302E6627
:102060006F6E03F610FB0D01652746464646464651
:1020700046460203F610FB0C0146323730707802F8
:1020800030707803F41F0188092093F610FB0401D7
:10209000402003F610FB020140EF4445EF4545F6B2
:1020A0000AFBF610FB0103EF4545F610FB0D016638
:1020B00070726F7032352E666F6E03F610FB090179
:1020C0004530022D302E3503F41F01860120F90121
:1020D00086022105018603211101861520F901865A
:1020E000162105018617211101861F20F9F610FB24
:1020F00005014074680380211DF610FB0501407343
:10210000740380211DF610FB0501406E64038021DD
:102110001DF610FB05014072640380211DF610FBC3
:102120000D016670726F7033352E666F6E03F61098
:10213000FB1601630230707802393002333035709B
:102140007802323135707803F41DF610FB0401403B
:102150005C52F30300D7EF4445EF4545F30BF31111
:1021600002F30900F31100F630FBF610FB0103EF58
:102170004545F610FB0B0146373070780230707819
:1021800003F41BF610FB0601405C523230EF44456D
:10219000EF45458809219CF610FB0130EF4545F6D7
:1021A0000AFBF610FB0103EF4545F610FB0D016538
:1021B0002746463630363036300203F41DF610FB23
:1021C0000D016670726F7032352E666F6E03F610F9
:1021D000FB0601405C525C52EF4445EF4545F60A70
:1021E000FBF610FB022F03EF4545F610FB0D0165D2
:1021F0002746464646464646460203F610FB03017E
:102200006303F40209F610FB0401613103F610FBCD
:102210001601652746464646464646460227464636
:1022200030303030303003F610FB0D01666D6F6ECC
:102230006F36302E666F6E03F610FB1701630233A4
:1022400033357078023102313436707802323435E9
:10225000707803F610FB03015203831BC499F9C085
:102260000088F61C22C4AA22B3831B83994800006D
:1022700085F61F22B3F610FB020140F609FB0200AF
:10228000F610FB0103F610FB0D01666D6F6E6F33E8
:10229000352E666F6E03F610FB0301402EEF964756
:1022A000941CF609FB0100F610FB02B003EF944703
:1022B0008022C4F610FB020140F609FB0300F61071
:1022C000FB02B003F610FB03016303F610FB0401ED
:1022D000613003094A01801D29F610FB16016527AC
:1022E000464639303930393002274646464646465A
:1022F000464603F610FB0D016670726F7033352E83
:10230000666F6E03F610FB3F0150023070780230AA
:102310007078023133357078023135397078025374
:1023200065745C7254696D650202020202022746FE
:1023300046464646464646022746464430363030F4
:1023400030020202180203F610FB41015002307005
:102350007802313631707802313335707802313598
:10236000397078025365745C7244617465020202CC
:10237000020202274646464646464646022746464B
:10238000393032304330020202190203F610FB48A2
:1023900001500230707802333232707802313335B6
:1023A000707802313539707802436C696D617465FB
:1023B0005C6E436F6E74726F6C020202020202273F
:1023C0004646303030303030022746464646464694
:1023D00030300202021A0203F610FB3901503002BB
:1023E00031333770780230707802313335707802CB
:1023F000313539707802020202020202274646464F
:102400004646464646022746463030303043300284
:1024100002021B0203F610FB0D016670726F70372B
:10242000302E666F6E03F610FB3E015002313337DB
:10243000707802313631707802313335707802337A
:10244000313970780245786974020202020202276B
:1024500046464646464646460227464630303930CE
:1024600030300202021C020383248B690121F4062E
:102470001E00000A6007201D04600121246BF40780
:102480000007D02470831D81802470F610FB140196
:10249000503002020202024261636B6C6967687429
:1024A0005C6E5BF303002DEF4445450BF30BF3111A
:1024B00002F30900F31100F630FBF610FB0D5D028C
:1024C0000202020202020202020203EF454509680B
:1024D0000121831A6E80248BF610FB040161310305
:1024E0008326CBF610FB160165274646363036307C
:1024F00036300227464646464646464603F610FB19
:102500000D016670726F7033352E666F6E03F610B4
:10251000FB27015031023630707802313930707843
:1025200002353470780235347078023102020202CA
:102530000202020202021D0203F610FB27015032C2
:102540000233357078023234357078023534707861
:1025500002353470780232020202020202020202E2
:10256000021D0203F610FB2701503302363070784B
:102570000233303070780235347078023534707838
:102580000233020202020202020202021D0203F6EA
:1025900010FB280150340231313570780231393066
:1025A0007078023534707802353470780234020263
:1025B00002020202020202021D0203F610FB2701C0
:1025C0005035023930707802323435707802353443
:1025D000707802353470780235020202020202027B
:1025E0000202021D0203F610FB28015036023131AF
:1025F00035707802333030707802353470780235B7
:102600003470780236020202020202020202021D45
:102610000203F610FB280150370231373070780280
:102620003139307078023534707802353470780280
:1026300037020202020202020202021D0203F61027
:10264000FB2801503802313435707802323435704D
:10265000780235347078023534707802380202021C
:10266000020202020202021D0203F610FB280150C0
:1026700039023137307078023330307078023534B7
:1026800070780235347078023902020202020202C6
:102690000202021D0203F610FB2801503002323004
:1026A0003070780232343570780235347078023503
:1026B0003470780230020202020202020202021D9B
:1026C0000203F610FB040161300309B900F433F68C
:1026D00010FB020150EF4445BAF60AFBF610FB125C
:1026E000020202300202020202020202020202029C
:1026F0000203EF4545BCBA8B0C26CD09B9001F2259
:1027000000BCBA8A0A26FE4517441609833BDF023D
:10271000014A30F6204413211627218326FC802706
:1027200034B900BCBA451712812734B022BDB1229A
:10273000BC8027234517BBBD4513B122161609F6E9
:1027400010FB0D015302273630303030303030036B
:10275000F610FB20015002300230023130302502E9
:102760003130302502026831020202020202020206
:10277000021E0203F610FB1601652746463330336E
:102780003033300227464645304530453003F61099
:10279000FB0D016670726F7032352E666F6E03F638
:1027A00010FB110163432D3202432D3130023402FC
:1027B00032300203F610FB0301520368002109F4D2
:1027C00006F4026100213C93F4070000FA27C1F4EB
:1027D0000E69002109690021094A03801D298F170C
:1027E000028326FCF610FB0D0153022746464530B6
:1027F0004530453003831D2FF610FB0F01405C432D
:10280000456E746572204461746503F610FB030124
:102810006303F610FB160165274646363036303620
:10282000300227303030303030303003F610FB0DBE
:10283000016670726F7033352E666F6E03F610FB93
:102840003C015032300238307078023470780235F2
:10285000347078023137307078020270316730029C
:10286000020202020227464643304330433002024E
:10287000274646464646464646021F0203F610FBDA
:102880003B015032310231333570780234707802B6
:1028900035347078023137307078020267300202C6
:1028A00002020202274646433043304330020227E9
:1028B000464646464646464602200203F610FB0DB3
:1028C000016670726F7037302E666F6E03F610FB04
:1028D0000C014632343070780234707803F610FB05
:1028E000050140323003F610FB0D016670726F7007
:1028F00033352E666F6E03F610FB3B015032320209
:10290000313930707802383070780235347078029E
:10291000393470780202673002020202020227464E
:102920004643304330433002022746464646464639
:10293000464602210203F610FB160165274646367D
:10294000303630363002274646464646464646032F
:10295000F610FB0D016670726F7033352E666F6E68
:1029600003F610FB2C0150333002363070780233FE
:10297000363670780235347078023130387078022B
:1029800053415645020202020202020202022202E0
:1029900003F610FB2C0150333102313135707802CF
:1029A00033363670780235347078023130387078CA
:1029B00002434C52020202020202020202022302FB
:1029C00003F610FB2B01500231373070780233369A
:1029D00036707802353470780231303870780251B0
:1029E00055495402020202020202020202240203B8
:1029F0004A00F41C4A00F41E4A00F420832ED683B9
:102A00002A0E1E00000A6007201D04802A02F6100C
:102A1000FB1A0150333102020202020268306430B4
:102A20000202020202020202022302038326FC8344
:102A300024D8B900F433F610FB020150EF4445BA34
:102A4000F60AFBF610FB1202020202020202020266
:102A5000020202020202250203EF4545BCBA8B09BD
:102A60002A3409F610FB1901503331020202020226
:102A7000026831643102020202020202020202030F
:102A8000F610FB16016527464636303630363002E2
:102A900027464646464646464603F610FB0D016667
:102AA00070726F7032352E666F6E038326CBF61010
:102AB000FB190150310233357078023139307078AA
:102AC0000235347078023534707802F3030121F353
:102AD0000A0001F31102F30900F31100F630FBF6CE
:102AE00010FB180267310202020202020227464668
:102AF0004530453045300202260203F610FB19012D
:102B00005032023335707802323435707802353401
:102B10007078023534707802F3030121F30A000261
:102B2000F31102F30900F31100F630FBF610FB1865
:102B30000267310202020202020227464645304580
:102B40003045300202260203F610FB190150330211
:102B50003335707802333030707802353470780253
:102B60003534707802F3030121F30A0003F31102F4
:102B7000F30900F31100F630FBF610FB1802673181
:102B80000202020202020227464645304530453025
:102B90000202260203F610FB19015034023930708C
:102BA00078023139307078023534707802353470FB
:102BB0007802F3030121F30A0004F31102F3090080
:102BC000F31100F630FBF610FB1802673102020227
:102BD00002020202274646453045304530020226B1
:102BE0000203F610FB1901503502393070780232B9
:102BF000343570780235347078023534707802F3E9
:102C0000030121F30A0005F31102F30900F3110097
:102C1000F630FBF610FB18026731020202020202D4
:102C2000022746464530453045300202260203F66B
:102C300010FB190150360239307078023330307091
:102C4000780235347078023534707802F30301214C
:102C5000F30A0006F31102F30900F31100F630FB4A
:102C6000F610FB1802673102020202020202274636
:102C7000464530453045300202260203F610FB1A65
:102C800001503702313435707802313930707802B2
:102C900035347078023534707802F3030121F30A79
:102CA0000007F31102F30900F31100F630FBF610F0
:102CB000FB18026731020202020202022746464561
:102CC00030453045300202260203F610FB1A01504F
:102CD0003802313435707802323435707802353448
:102CE0007078023534707802F3030121F30A00088A
:102CF000F31102F30900F31100F630FBF610FB1894
:102D000002673102020202020202274646453045AE
:102D10003045300202260203F610FB1A0150390238
:102D20003134357078023330307078023534707851
:102D3000023534707802F3030121F30A0009F3111C
:102D400002F30900F31100F630FBF610FB180267DE
:102D50003102020202020202274646453045304552
:102D6000300202260203F610FB1B01503130023202
:102D70003030707802313930707802353470780232
:102D80003534707802F3030121F30A000AF31102CB
:102D9000F30900F31100F630FBF610FB180267315F
:102DA0000202020202020227464645304530453003
:102DB0000202260203F610FB1B01503131023230B1
:102DC00030707802323435707802353470780235DC
:102DD00034707802F3030121F30A000BF31102F3BC
:102DE0000900F31100F630FBF610FB180267310200
:102DF00002020202020227464645304530453002B3
:102E000002260203F610FB1B015031320232303031
:102E1000707802333030707802353470780235348F
:102E2000707802F3030121F30A000CF31102F30995
:102E300000F31100F630FBF610FB180267310202B6
:102E40000202020202274646453045304530020262
:102E5000260203F41D010AF610FB020150EF44455F
:102E6000EF4545F60AFBF610FB13020202020202CE
:102E700070310202020202020202020203EF454521
:102E800009F610FB1A0150333102020202020268F5
:102E900030643002020202020202020227020383AD
:102EA00026FC8324D8B900F433F610FB020150EF5E
:102EB0004445BAF60AFBF610FB12020202020202B5
:102EC000020202020202020202280203EF4545BC8E
:102ED000BA8B092EA709F433F610FB0D0166707248
:102EE0006F7033352E666F6E03F610FB1601652783
:102EF00046463630363036300227303030303030CB
:102F0000303003F610FB1401630230707802310296
:102F10003138307078023730707803F610FB0301D7
:102F20005203F41F812F7BF41D812F7BF41B812F13
:102F30007BF423F610FB0401405C43F3030073EFC2
:102F40004445EF4545F30BF31102F30900F311007B
:102F5000F630FBF610FB0103EF4545F610FB1901B7
:102F60005033300202020202026430683002020270
:102F70000202020202020203802F9AF610FB1B01DA
:102F80005033300202020202026431613330250202
:102F900002020202020202020203F610FB030163B4
:102FA00003F610FB160165274646363036303630BC
:102FB0000227464646464646464603F41F01812FF1
:102FC000EDF610FB09015032300202020202EF441A
:102FD00045EF4545F60AFBF610FB0C020202020221
:102FE00002020202020203EF454580300AF610FB9E
:102FF000190150323002020202024461793F02029A
:1030000002020202020202020203F433F41D0181F1
:103010003059F610FB09015032310202020202F36C
:10302000030121EF4445EF4545F30BF31102F3098A
:1030300000F31100F630FBF610FB0128EF4545F6D2
:103040000AFBF610FB0D2902020202020202020232
:10305000020203EF4545803078F610FB1B01503229
:103060003102020202024D6F6E74683F02020202D8
:103070000202020202020203F41B018130B4F610C4
:10308000FB09015032320202020202EF4445EF45D1
:10309000458809309AF610FB0130EF4545F60AFBEA
:1030A000F610FB0C020202020202020202020203FA
:1030B000EF454509F610FB1A0150323202020202B6
:1030C00002596561723F020202020202020202021A
:1030D000020309F41A83273FF610FB080146432D2B
:1030E00031023003F610FB1E01405C434E65772031
:1030F00064617465206861735C6E6265656E2073DF
:10310000617665642E038022D48326FC4A00F42075
:10311000802ED68326FC4A00F41C802ED683270CF2
:103120008334D94513F420F42F802ED6833BDF025D
:10313000F41EF42F802ED683270C8334D94513F444
:103140001CF42F802ED64A02801D298F18FF8F175E
:10315000048326FCF610FB0D01530227464645303A
:103160004530453003831D2FF610FB0C01405C43B6
:1031700053657454696D6503F610FB03016303F630
:1031800010FB0D016670726F7032352E666F6E0324
:10319000F610FB16016527464636303630363002CB
:1031A00027303030303030303003F610FB0B014622
:1031B000353070780230707803F610FB0C01404E09
:1031C00065772074696D653A03F610FB0C01463192
:1031D000393070780230707803F610FB10014043EC
:1031E000757272656E742074696D653A038324D8B4
:1031F000B900F433F610FB020150EF4445BAF60A69
:10320000FBF610FB1202020202020202020202029A
:1032100002020202290203EF4545BCBA8B0931F2D2
:10322000F610FB30015033300236307078023336FE
:103230003670780235347078023130387078025345
:103240004156450268316431020202020202020262
:10325000022A0203F610FB2A015002313135707840
:103260000233363670780235347078023130387077
:103270007802434C52020202020202020202022BB4
:103280000203F610FB2B0150023137307078023305
:103290003636707802353470780231303870780202
:1032A00051554954020202020202020202022402A1
:1032B00003F610FB0D01650227303030303030301E
:1032C00030038333EA1E00000A6007201D048332A6
:1032D000D48032C5F411F41F4518120AF41F4418A3
:1032E000F610FB0D01666D6F6E6F33352E666F6ED7
:1032F00003F610FB16016527464636303630363069
:103300000227303030303030303003F610FB0C0103
:103310004632333070780235707803F41BF41DF6B2
:1033200010FB020140EF4445EF4446EF454601885B
:10333000093338F610FB0130EF454601F60AFBF67B
:1033400010FB013AEF454588093350F610FB013078
:10335000EF4545F60AFBF610FB0103EF4545F61075
:10336000FB0D01666D6F6E6F33352E666F6E03F465
:103370001FF610FB0301403AEF4445EF454588092D
:103380003387F610FB0130EF4545F60AFBF610FBDC
:103390000103EF4545F402098334D94513F41C4574
:1033A00014F41E4A00F420F41283273FF610FB08A1
:1033B0000146432D31023003F610FB1E01405C43F1
:1033C0004E65772074696D65206861735C6E626517
:1033D000656E2073617665642E038022D48326FC9B
:1033E0008333EA0983270C8033EAF610FB0D01666C
:1033F00070726F7037302E666F6E03F610FB160119
:10340000652746463630363036300227464643304A
:103410004330433003F610FB15016302327078022B
:103420003102313830707802313230707803F61062
:10343000FB03015203F610FB020140B900B022BAAF
:1034400087023449F610FB013A01823456F610FB2C
:10345000022020803459F60FFBBCBA8A04343DF6B2
:1034600010FB0103F610FB03016303F610FB1601CA
:103470006527464636303630363002273030303019
:103480003030303003451626160134B98334D9263E
:10349000131734B926143B34B9F610FB1901503315
:1034A00030020202020202683064300202020202AA
:1034B0000202020202038034D8F610FB1B015033D3
:1034C000300202020202026431613330250202023C
:1034D000020202020202020309B9008334E7441324
:1034E000B9028334E744148334FA9F9920000082A0
:1034F00092ABBC8334FA9F909E09B022018A30358A
:103500000B018839350B4A30F622094A00094A0472
:10351000801D29690221F610FB0D01530227464642
:1035200045304530453003F610FB0D016670726F73
:103530007032352E666F6E03831D2FF610FB14015B
:10354000405C43436C696D61746520436F6E7472B7
:103550006F6C03F610FB03016303F610FB160165A5
:10356000274646363036303630022730303030305D
:1035700030303003F610FB17016330707802307082
:10358000780232373270780231343570780203F6BF
:1035900010FB0B0146363770780230707803F61056
:1035A000FB0801405C5246616E03F610FB0C0146BD
:1035B00031323270780230707803F610FB0A014025
:1035C0005C5252656C617903F610FB0C0146313791
:1035D0003770780230707803F610FB1001405C52AF
:1035E00054656D706572617475726503F610FB0C3D
:1035F000014632333770780230707803F610FB0ED4
:1036000001405C5243757272656E746C7903F610FA
:10361000FB160165274646333033303330022746E8
:103620004643304330433003F610FB0D01667072A1
:103630006F7032352E666F6E03F610FB3C0150340E
:103640000233357078023135307078023534707855
:103650000236397078024F6E0267300202020202AF
:10366000020227464646464646464602274646301A
:103670003046463030022C0203F610FB3D01503537
:103680000233357078023232307078023534707817
:103690000236397078024F66660267300202020213
:1036A0000202022746464646464646460227464608
:1036B000303046463030022D0203F610FB3E0150FA
:1036C0003602333570780232393070780235347012
:1036D000780236397078024175746F0267300202E1
:1036E0000202020202274646464646464646022750
:1036F0004646303046463030022E0203F610FB3C80
:103700000150370239307078023135307078023527
:103710003470780236397078024F6E0267310202D7
:10372000020202020227464646464646464602270F
:103730004646303046463030022F0203F610FB3D3D
:1037400001503802393070780232323070780235E8
:103750003470780236397078024F6666026731023B
:1037600002020202020227464646464646464602F4
:1037700027464630304646303002300203F610FB12
:103780003E01503902393070780232393070780297
:10379000353470780236397078024175746F02677B
:1037A00031020202020202022746464646464646C9
:1037B000460227464630304646303002310203F694
:1037C00010FB2B0150300231343570780231353026
:1037D000707802353470780236397078022D0272B2
:1037E0003130020202020202020202320203F61029
:1037F000FB2B015031023134357078023239307090
:103800007802353470780236397078022B027231C2
:1038100030020202020202020202320203F610FB2E
:103820003D015032023230307078023232307078DE
:103830000235347078023639707802B0430267324C
:103840000202020202020227464646464646464613
:103850000227464630304646303002330203F61027
:10386000FB3D015033023230307078023239307013
:10387000780235347078023639707802B0460267C3
:1038800032020202020202022746464646464646E7
:10389000460227464630304646303002330203F6B1
:1038A00010FB160165274646363036303630022783
:1038B000464646464646464603F610FB2B01500256
:1038C000313137707802333636707802353470789B
:1038D000023130387078024558495402020202021F
:1038E00002020202022402038339268339818339CA
:1038F000DC833A17F610FB1601652746463630364C
:1039000030363002273030303030303030031E0057
:10391000000A600720391D833AD180390E610221E7
:1039200039230E801D0460010639664C0582394B2F
:10393000F610FB160150350202020202027031023B
:103940000202020202020202020309F610FB160141
:10395000503402020202020270310202020202022A
:10396000020202020309F610FB160150360202029F
:103970000202027031020202020202020202020389
:103980000960020639C14C048239A6F610FB160103
:1039900050380202020202027031020202020202E6
:1039A000020202020309F610FB160150370202025E
:1039B0000202027031020202020202020202020349
:1039C00009F610FB160150390202020202027031A0
:1039D0000202020202020202020203096000063928
:1039E000FCF610FB16015032020202020202703194
:1039F000020202020202020202020309F610FB1690
:103A0000015033020202020202703102020202027B
:103A100002020202020309F610FB0D016670726FCA
:103A20007033352E666F6E03F610FB160165274660
:103A30004633303330333002274646464646464604
:103A40004603F610FB1901633134377078023232C5
:103A5000327078023530707802363570780203F6AD
:103A600010FB03015203F610FB0901463335707851
:103A70000230036000003A95F610FB0401405C43FD
:103A8000EF96479407F609FB0300F610FB0103EFDE
:103A90009447803AAFF610FB0401405C43EF964731
:103AA0009407F609FB0300F610FB0103EF9447F6B9
:103AB00010FB16016527464633303330333002277A
:103AC000303030303030303003F610FB0301630308
:103AD00009F610FB0D016670726F7033352E666F3C
:103AE0006E03F610FB16016527464633303330333C
:103AF000300227303030303030303003F610FB19D0
:103B000001633230357078023135307078023534E7
:103B1000707802363970780203F610FB0301520305
:103B2000831BC499F9C00088F61D3B3CF610FB02CC
:103B30000140F609FB0401F610FB0103F610FB033C
:103B4000016303096901064205680221096901064A
:103B50004305680221096801066802210969020615
:103B600042046802210969020643046802210968C7
:103B7000020668022109833BDF02823B85998000AF
:103B8000007F803B8A990000007F9407909607830E
:103B90001C0F680221803A17833BDF0286033BB08B
:103BA0006100063C936900069407831BE7803BBDD8
:103BB0006000063C936800069407831BFB96076829
:103BC0000221803A17F00500000AF10100823BD57E
:103BD000F00000000AF10A0000F00100000A094AA2
:103BE00005F636FB86FF3C43F63BFB03F624823C9E
:103BF000439EF639FB87023C43F63BFB03F62482E7
:103C00003C439EF639FB87023C43F63BFB06F62419
:103C1000823C43F639FB87023C43F10500F63BFB4F
:103C200006F624823C43F639FBF1050498000000B7
:103C30000087023C42F63BFB08F624823C43F639FF
:103C4000FB02094A04094A05F636FB86FF3C5CF68E
:103C50003CFB0186003C5D0186013C7C09F639FB9A
:103C600087023C5CF63CFBF639FB87023C5CF63B8A
:103C7000FBFFF639FB87053C5C801D78F639FB8736
:103C8000053C5CF610FB0401530203F00000000A3F
:103C9000801D7C09F10704F10508833CA6F10808A2
:103CA00092F10804910993F105009A990000007EB1
:103CB000F61F3CBA980000000009F10600AA3CC5B6
:103CC000998000007E90F51700F5180009F10704AF
:103CD000979A833CA6ABF106049A92F1080409F185
:103CE0000507F305F10500F313F10204F30CF102EB
:103CF00005F302F10206F1060709F10507F10106D5
:103D0000F301F10600F304F10104F312F10105F3EC
:103D10000BF106070992F10504980000007F9791C6
:103D2000833D3392F1080490833D4F09833D3AF17E
:103D3000060009833D3AF1080009B000F10200B025
:103D400001F10201B002F10202B003F1020309F134
:103D50000500803D5BF10700803D5BF10100B10093
:103D6000F10101B101F10102B102F10103B1030955
:103D7000F10500F30000F30A0000F31104F317004B
:103D8000BBF30701F31900F306F1080092F32100D9
:103D900090BDBE3D8709F10510AB986100008A8394
:103DA0003CA69EF1020C996100008A92F1081091E4
:103DB000F10510AB9870000084833CA69EF1020DC3
:103DC000997000008492F10810919EF1020E09EFA3
:103DD0009647F30000F30A0000F31104EFF3170015
:103DE000EF4445F30701EFF31900F306EF9547920F
:103DF000EFF3210090EF8E453DEA09F616F4024AF2
:103E000004F61386FF3DFDF30000F30302EBF62FEB
:103E100001083DFB3E623E683E6E3E743E7A3E8047
:103E20003E863E8C3E923E983E9E3EA43EAA3EB0CA
:103E30003EB63EBC3EC23EC83ECE3ED43EDA3EE03A
:103E40003EE63EEC3EF23EF83EFE3F043F0A3F10A7
:103E50003F163F1C3F223F283F2E3F343F3A3F4012
:103E60003F468319F8803DFD8319FC803DFD8304A6
:103E70001E803DFD83042E803DFD830436803DFD84
:103E8000830EA6803DFD830EC2803DFD830EDB8048
:103E90003DFD8319F4803DFD831DF7803DFD833199
:103EA00046803DFD8327D9803DFD83350E803DFD55
:103EB0008324CF803DFD831D81803DFD833C938025
:103EC0003DFD8327D5803DFD832A0E803DFD832A5D
:103ED00063803DFD832E81803DFD8330D3803DFD99
:103EE000833109803DFD8322D4803DFD83311D80D7
:103EF0003DFD83312C803DFD833113803DFD8331B9
:103F000037803DFD8333E4803DFD833398803DFD64
:103F10008333DD803DFD833B44803DFD833B4D800D
:103F20003DFD833B56803DFD833B5D803DFD833BF6
:103F300066803DFD833B6F803DFD833B76803DFD8C
:103F4000833B98803DFD833C46803DFD00000000A2
:103F50000000007E0000007F8000007FF03404300D
:103F600004FF54696D657200416D6269656E74008D
:103F70004C6F770048696768000016001C00240039
:103F8000284F6F7073004D6F6E64617900547565D2
:103F900073646179005765646E6573646179005478
:103FA000687572736461790046726964617900535F
:103FB000617475726461790053756E646179000093
:103FC0003A004100490053005C0063006C4A616E96
:103FD00075617279004665627275617279004D6132
:103FE00072636800417072696C004D6179004A75B6
:103FF0006E65004A756C790041756775737400537E
:10400000657074656D626572004F63746F6265728E
:10401000004E6F76656D62657200446563656D6222
:1040200065720000350081008900920098009E00B2
:10403000A200A700AC00B300BD00C500CE4A616E6F
:1040400000466562004D617200417072004D6179F9
:10405000004A756E004A756C0041756700536570C3
:10406000004F6374004E6F760044656300003500B6
:10407000F100F500F900FD010101050109010D0143
:104080001101150119011D4C756E6573004D6172AA
:10409000746573004D69E972636F6C6573004A75EE
:1040A0006576657300566965726E65730053E162EB
:1040B00061646F00446F6D696E676F00656E657255
:1040C0006F006665627265726F006D61727A6F0073
:1040D000616272696C006D61796F006A756E696FFB
:1040E000006A756C696F0061676F73746F00736548
:1040F000707469656D627265006F63747562726574
:10410000006E6F7669656D627265006469636965EA
:104110006D627265004A8000873E000085390000AC
:10412000870C0000863E00008716000085430000D3
:1041300087700000854080008711000086430000E2
:1041400087700000854A800087700000853E00006F
:1041500087020000854A8000877A0000854A800037
:10416000870600008501C901D101D901E101E901FA
:10417000F101F902010209021103FF0007FFFFFF2D
:10418000FFFF006400FFFFFFFF03FF0007FFFFFFCB
:10419000FFFF006400FFFFFFFF03FF0007FFFFFFBB
:1041A000FFFF006400FFFFFFFF05A9255989619506
:1041B000428AF0FEA48A023CBD8AA88E158818BEE9
:1041C00097860E04000F040010040011040012046E
:1041D0000013040014040015040016040017040062
:1041E0001804001904001A04001B04001C04001D1C
:1041F00004001E04001F0400200400210400220407
:1042000000230400240400250400260400270400E1
:104210002804002904002A04002B04002C04002D8B
:1042200004002E04002F0400300400310400320486
:104230000033040006040002760279027C027F0249
:104240008202850288028B028E02910294029702FA
:104250009A029D02A002A302A602A902AC02AF022A
:10426000B202B502B802BB02BE02C102C402C7025A
:10427000CA02CD02D002D302D602D902DC02DF028A
:10428000E202E502E8FFFFFFFFFFFFFFFFFFFFFF86
:10429000FFFFFFFFFFFFFFFFFFFFFFFFFFFFFFFF2E
:1042A000FFFFFFFFFFFFFFFFFFFFFFFFFFFFFFFF1E
:1042B000FFFFFFFFFFFFFFFFFFFFFFFFFFFFFFFF0E
:1042C000FFFFFFFFFFFFFFFFFFFFFFFFFFFFFFFFFE
:020000022000DC
:1000000071B940F21423C1F20003D3ED007AB7EEC8
:10001000007A37EE670A82ED000A4FF00000704761
:100020004FF01400704700BF40F21423C1F20003E8
:1000300018686FEA0000704708B507EE902A4FF085
:1000400001021A70B1B9B7EE007A37EE670A40F2D2
:100050001423C1F2000383ED000A4FF002004FF0B9
:10006000000117EE102A10EE103A03F0CFFE4FF009
:10007000000008BD4FF0000018704FF0140008BDDC
:1000800010B540F21424C1F200044FF030002146B4
:100090004FF0080209F0F8FBFFF7C6FF63688342E0
:1000A00009D14FF002004FF000014FF07E5223685B
:1000B00003F0ACFE0FE04FF002004FF000014FF0F4
:1000C0007E52134603F0A2FE40F21420C1F200005B
:1000D0004FF0804202604FF00C0041F61801C0F270
:1000E000060140F20822C1F2000228F0C9FA10BD50
:1000F00008B54FF00103137011B101291DD110E0B3
:10010000FFF792FF40F21422C1F200025060104645
:100110004FF008014FF0300209F044FC4FF00000AE
:1001200008BD4FF002004FF000014FF07E52134621
:1001300003F06CFE4FF0000008BD4FF0000111709D
:100140004FF0140008BD00BF6FF00200704700BF01
:100150004FF00100704700BF4FF00100704700BF33
:100160004FF00100704700BFC3688B4206D800699A
:100170001A1891428CBF0020012070474FF00000F8
:10018000704700BF48F20C02C4F20802136813F073
:10019000100FFBD148F20C01C4F208010A6812F0FA
:1001A000040F0CD048F20801C4F2080148F20C0216
:1001B000C4F208020B68136813F0040FFAD148F276
:1001C0000C01C4F208010A6812F0020FFBD048F2D9
:1001D0000803C4F20803186048F20C00C4F20800D7
:1001E000016811F0040FFBD048F20802C4F20802C3
:1001F0001368D8B2704700BF82B048F20C02C4F254
:100200000802136813F0100FFBD100BF00BF48F2C3
:100210005800C2F209004FF4000101604FF01402CF
:100220000192019B3BB100BF019800F1FF310191A8
:10023000019A002AF7D102B0704700BF2DE9F041C2
:1002400082B015461C46C368C91A019148F25C0089
:10025000C2F209004FF40002026048F20C01C4F23D
:1002600008010B6813F0020FFBD048F20800C4F23B
:1002700008004FF00B0202609DF8061048F20C00D7
:10028000C4F20800036813F0020FFBD048F2080222
:10029000C4F2080211609DF8051048F20C00C4F287
:1002A0000800036813F0020FFBD048F20802C4F202
:1002B000080211609DF8041048F20C00C4F2080016
:1002C000036813F0020FFBD048F20802C4F20802E0
:1002D00011604FF00000FFF755FF75B34FF00007B6
:1002E00041F68406C0F2060605F1FF3808F0010861
:1002F0003846FFF747FF80EA1461C8B256F820304D
:1003000083EA0424013D1ED117E03846FFF73AFF87
:1003100080EA1463DAB256F8221081EA042405F167
:10032000FF353846FFF72EFF80EA1460C3B256F857
:10033000232082EA0424013DE7D1FFF75DFF204638
:1003400002B0BDE8F081B8F1000FDED03846FFF70B
:1003500019FF80EA1462D1B256F8210080EA042421
:10036000013DD2D1E9E700BF2DE9F04F85B00E463F
:100370001C46C368D21A039248F25C00C2F209001C
:100380004FF40001016048F20C05C4F208052F6823
:1003900017F0020FFBD048F20803C4F208034FF035
:1003A0000B021A609DF80E0048F20C01C4F208011D
:1003B0000D6815F0020FFBD048F20807C4F20807D9
:1003C00038609DF80D0048F20C02C4F20802136870
:1003D00013F0020FFBD048F20801C4F208010860D4
:1003E0009DF80C7048F20C05C4F20805286810F05E
:1003F000020FFBD048F20805C4F208052F604FF049
:100400000000FFF7BFFE41F6AC42C0F206021168E1
:1004100048F22403C4F20803196041F68007C0F2D1
:100420000607386840F28C12C2F20802106040F2EF
:100430006011C2F208010D6040F28013C2F208039D
:1004400041F6B447C0F206071F6040F28410C2F2C2
:100450000800056041F68C45C0F20605D5F800B0ED
:1004600041F64C02C0F206021168019141F66C039C
:10047000C0F20603186840F6FF7940F6F87840F2BB
:10048000641CC2F2080C40F26C1EC2F2080E40F26C
:100490008C17C2F2080740F27012C2F2080240F252
:1004A0009015AA46C2F2080A4C4594BF214641461F
:1004B000CCF800604FEA01534FEA1353DEF80050C6
:1004C00063F30B05CEF800503D6863F30B053D6008
:1004D000C2F800B0019BCAF80030641A761811689F
:1004E0000842FCD1002CDFD14FF0000048F224027A
:1004F000C4F20802106040F27013C2F208031860E0
:1005000040F29011C2F208010860FFF775FE4FF04B
:10051000010005B0BDE8F08F08B548F25C03C2F2F7
:1005200009034FF400021A6048F20C00C4F20800FC
:10053000016811F0020FFBD048F20803C4F208036F
:100540004FF006021A60FFF757FE08BD10B548F2DB
:100550005C03C2F209034FF400021A6048F20C0077
:10056000C4F20800016811F0020FFBD048F2080441
:10057000C4F208044FF0050323601C462046FFF731
:1005800001FE10F0010F02D024F0B4F8F6E7FFF7F7
:1005900033FE10BDF0B583B004461E46089DC0680A
:1005A000884231D302F1FF33CB1898422CD8276907
:1005B00007F1FF37C019814226D8834224D3FFF7C1
:1005C000ABFF48F25C01C2F209014FF400020A607D
:1005D00048F20C00C4F20800036813F0020FFBD0CD
:1005E00048F20801C4F208014FF060020A60FFF708
:1005F00003FEFFF7ABFF0EB1E068306075B1236911
:100600002B604FF001000BE000960195204640F270
:100610002563C0F2020334F0C1F801E04FF001009D
:1006200003B0F0BD10B582B04B68C268981A019053
:100630008968B1F5004F0BD0B1F5803F05D0B1F519
:10064000805F51D14FF0200404E04FF0D80401E066
:100650004FF05204FFF760FF48F25C03C2F2090357
:100660004FF400021A6048F20C00C4F2080001685E
:1006700011F0020FFBD048F20803C4F208031C601B
:100680009DF8060048F20C02C4F20802116811F04D
:10069000020FFBD048F20803C4F2080318609DF86B
:1006A000050048F20C02C4F20802116811F0020FB2
:1006B000FBD048F20803C4F2080318609DF8040058
:1006C00048F20C02C4F20802116811F0020FFBD0CC
:1006D00048F20803C4F208031860FFF78DFDFFF726
:1006E00035FF4FF0010001E06FF0080002B010BDCF
:1006F0002DE9F04F83B015461F461378FF2B1AD112
:10070000002F73D007F1FF3404F001044FF0010310
:1007100012F8016FFF2E6ED00FE003F101042346A3
:1007200012F8016FFF2E08D104F1010312F8014FF6
:10073000FF2C6DD001E04FF00003BB4256D0C068E3
:10074000091A0191CBB2C3F5807B002F4ED048F23D
:100750005C0AC2F2090A4FF4000948F20C04C4F220
:10076000080448F20806C4F208064FF00208FFF732
:10077000D3FECAF80090226812F0020FFBD0C6F830
:1007800000809DF80600216811F0020FFBD0306058
:100790009DF80520236813F0020FFBD032609DF80E
:1007A0000400216811F0020FFBD03060BB4534BF5C
:1007B0005A463A46BF1A4AB1A81815F8013B2168B3
:1007C00011F0020FFBD033608542F6D1FFF714FD24
:1007D000FFF7BCFE4FF000028DF80420019800F5F1
:1007E000807301934FF4807B002FC0D14FF0010044
:1007F00003B0BDE8F08FBB42F8D0002C8DD003F1E0
:10080000010312F8014FFF2C97D1BB4285D1EDE7D0
:10081000BB4282D1EAE700BFF0B585B007460E467D
:1008200015464CF2C402C4F20F02116841F00050A8
:10083000106041F6B844C0F20604206840F230016E
:10084000C2F2080108604CF2C414C4F20F0420681C
:100850006FF38200206021686FF3C30121604FF0C5
:10086000000140F26814C2F20804216040F28810CE
:10087000C2F20800016041F67C04C0F2060424685C
:1008800040F26C10C2F208000460146844F40010D6
:10089000106048F21002C4F208024FF00204146023
:1008A00041F68440C0F2060002684CF25814C4F2CB
:1008B000020422604CF26810C4F2020002604CF2A2
:1008C0006C14C4F20204226041F6B042C0F2060287
:1008D00010684CF25C14C4F2020420604FF4000073
:1008E00048F25802C2F20902106048F24002C2F215
:1008F000090214680443146048F20402C4F20802B6
:10090000146861F34104146041F69041C0F206019D
:100910000C6848F20001C4F208010C604FEA13238E
:1009200045F2C744C0F21E14A4FB03E34FEA93242C
:1009300004F1FF33DCB20B6864F30F230B6041F664
:100940006801C0F206010C681460136843F00201EC
:10095000116048F25C02C2F20902106048F20C0019
:10096000C4F20800046814F0020FFBD048F2080338
:10097000C4F208034FF09F0119604FF00000FFF729
:1009800001FC4FF00000FFF7FDFB4FF00000FFF708
:10099000F9FBFFF731FC48F25C00C2F209004FF4AA
:1009A0000002026048F20C04C4F20804236813F049
:1009B000020FFBD048F20801C4F208014FF05000CA
:1009C0000860FFF719FC48F25C04C2F209044FF416
:1009D0000002226048F20C01C4F208010B6813F017
:1009E000020FFBD048F20800C4F208004FF00104E7
:1009F000046041F68842C0F20602117848F20C0405
:100A0000C4F20804236813F0020FFBD048F2080078
:100A1000C4F208000160FFF7EFFB4FF00002009204
:100A200041F65001C0F20601019141F67003C0F297
:100A300006030293384631462A4641F69443C0F2F3
:100A4000060333F01BFE4FF0010005B0F0BD00BF00
:100A50000B4629B140F22C21C1F20001096819604E
:100A600058B140F22C23C1F20003196840F2202350
:100A7000C1F200031B68C91A01602AB140F22420A8
:100A8000C1F2000003681360704700BF40F200032A
:100A9000CAF200031868B0F1FF3F04D040F2000032
:100AA000CAF2000070474FF00000704790B1026832
:100AB00002F10302801820F0030140F20003CAF2A1
:100AC0008003994209D24A68B2F1333F0CBF08460D
:100AD000002070474FF0000070474FF00000704753
:100AE00038B14268B2F1333F08D1037B4FF00000C8
:100AF00008E04FF002004FF0000303E04FF0020067
:100B00004FF0000301B10B70704700BF18B10068CF
:100B1000A0F1380070474FF00000704710B100F1AD
:100B2000100070474FF00000704700BF08B18068A8
:100B300070474FF00000704710B100F13800704767
:100B40004FF00000704700BF024668B31F4B2049BA
:100B500099422CD240F20000CAF200004368B3F17F
:100B6000333F27D140F20001CAF200018868904269
:100B700026D040F20000CAF2000040F20001CAF2A2
:100B8000800102E0836893421ED0036803F10303EF
:100B9000C01820F0030088420FD24368B3F1333FFE
:100BA000F0D04FF0000070474FF0000070474FF05A
:100BB000000070474FF0000070474FF00000704792
:100BC00040F20000CAF20000704700BF000080A0A1
:100BD000000000A02DE9F8438046284B284A9A429D
:100BE0003CD24FF0000540F20004CAF200044FF678
:100BF000FF7640F20007CAF280076068B0F1FF3F5D
:100C000004D12068B0F1FF3F34D129E0E1892029E7
:100C100030D8B0F1333F2DD1636B6FEA0302206807
:100C2000904227D12046FFF787FF81462046FFF7F5
:100C30006DFF02463046494625F086FF218E8142EF
:100C400018D1A3689D4238BF1D46226802F10302F5
:100C5000A41824F00304BC42CFD301E04FF00005F8
:100C6000B8F1000F04D0C8F800504FF0000401E0C4
:100C70004FF000042046BDE8F88300BF000080A0CC
:100C8000000000A010B540F22823C1F200031C6848
:100C90002CB120461DF078FB2469002CF9D110BD41
:100CA00038B50446154600682018821840F2000343
:100CB000CAF280039A4208D22A463DF0FDFC216820
:100CC0004D1925604FF0010038BD4FF0000038BDD0
:100CD00070B50646294B2A4898421CD240F20004BF
:100CE000CAF200046368B3F1333F19D140F2000443
:100CF000CAF2000440F20005CAF28005206800F143
:100D00000300241824F00304AC420DD26368B3F14D
:100D1000333FF3D008E040F20004CAF2000403E0DD
:100D200040F20004CAF20004611840F20000CAF266
:100D3000800081421ED24FF07735656040F21C2161
:100D4000C1F200010B6803F101030B60A360A281F3
:100D500004F11005284631464FF020023BF0C2FC5A
:100D600028463DF0A9FD00F10100E0814FF0380276
:100D7000226001E04FF00004204670BD000080A01A
:100D8000000000A0F0B583B0044600286CD0436892
:100D9000B3F1FF3F6BD0808910F0010F6AD1216859
:100DA00001F103052A1922F0030540F20006CAF2F8
:100DB0008006B54215D26B68B3F1333F13D12E468E
:100DC00040F20000CAF28000326802F10302B31858
:100DD00023F00306864207D27268B2F1333FF3D0A4
:100DE00002E02E4600E02E4606F1380640F20000F2
:100DF000CAF28000864240D240F22427C1F20007A6
:100E00003B6803F1FF323A6040F22020C1F200005B
:100E10000768791A0160771B204629464FEA970236
:100E200008F052FC2D1BE0194FF0FF314FEA9502FC
:100E30000AF04AFFFFF726FF40F20005CAF200055C
:100E4000631B40F20007C5F20007D819311B01AA45
:100E50006B4633F085FC0198C21B5119009A33F0A0
:100E600047FC4FF000000AE04FF0020007E04FF0AF
:100E7000020004E04FF0030001E04FF0010003B076
:100E8000F0BD00BF70B504464368B3F1773F46D16B
:100E90000068382803D12046FFF774FF70BD4FF07B
:100EA00033316160C0F1000505F0030520184FF0F3
:100EB000FF012A463DF034FC2046FFF73DFE064682
:100EC0002046FFF723FE02464FF6FF70314625F01D
:100ED0003BFE208622686FEA0203636340F2000053
:100EE000CAF20000211A40F20003C5F20003C8183C
:100EF0002146AA1833F0FCFB40F22420C1F2000086
:100F0000026802F10102026040F22023C1F20003F4
:100F100018682168421855191D60FFF7B3FE70BDAF
:100F200070B50546144B154A9A4221D240F2000092
:100F3000CAF200004168B1F1333F19D140F2000418
:100F4000CAF2000440F20006CAF2800604F1100062
:100F500029463BF04DF968B1236803F10303E41817
:100F600024F00304B44203D26268B2F1333FEDD0FF
:100F70004FF00004204670BD000080A0000000A0DB
:100F80002DE9F84F58B940F21C20C1F20000FFF7DC
:100F900021FED0F1010038BF0020BDE8F88F4FF0EE
:100FA000030640F20008CAF2000840F2000BC5F246
:100FB000000B40F2000ACAF2800AC8EB0A0A40F2AB
:100FC0001C29C1F200094FF47A7540465946524631
:100FD00033F0A8FB4846FFF7FDFD074660B14FF030
:100FE000FA04284625F098FD04F1FF34284625F040
:100FF00093FD013CF5D168E040F20000C5F200002D
:1010000040F20001C5F280010A1A40F22C23C1F21D
:1010100000031A604FF0000040F22021C1F20001ED
:10102000086040F22422C1F2000210602F4B3048C9
:1010300098423ED240F20001CAF200014A68B2F181
:10104000333F36D14FF000014FF0010040F2000372
:10105000CAF2000340F20005CAF2800500E0204613
:101060001A68C2F1000404F00304A418091902F17B
:1010700003029B1823F00303AB420AD340F2202261
:10108000C1F20002116040F22421C1F200010860A7
:101090000FE000F101045A68B2F1333FDFD040F2B3
:1010A0002023C1F20003196040F22421C1F20001A3
:1010B000086040F2E800C1F2000005F089F9D7F1BC
:1010C000010038BF0020BDE8F88F013E7FF47DAFFE
:1010D00040F20002CAF28002D31B38464FF0FF31C3
:1010E0004FEA93020AF0F0FD86E700BF000080A0FF
:1010F000000000A040F22823C1F200031A68026138
:101100001860704710B503460068824234BF144629
:101110000446021B0846991822463DF0CDFA2046A7
:1011200010BD00BF10B5044641F61050C0F20600D5
:10113000FFF7F6FEFFF700FD034608B92CB1234682
:1011400040F23022C1F20002136041F62050C0F29A
:101150000600FFF7E5FEFFF7EFFC40F23421C1F295
:1011600000010860C0B940F23020C1F200000368FD
:1011700040F23422C1F2000213606BB941F63051E3
:10118000C0F2060140F23020C1F20000016040F2DE
:101190003423C1F20003196010BD00BF28B940F22A
:1011A0003421C1F200010868FFE7008A704700BFE0
:1011B00028B940F23421C1F200010868FFE7B0F914
:1011C0000C00704728B940F23421C1F200010868D0
:1011D000FFE7B0F90E00704728B940F23421C1F2A0
:1011E00000010868FFE74089704700BF28B940F256
:1011F0003422C1F200021068FFE7438A8B4206D90D
:1012000000EB81025369C31801D0984205D142F224
:101210000B0291420DD0416943185A88D988188829
:1012200001FA82F38342C4BF01F1FF30801882B219
:1012300001E04FF0000210B2704700BF28B940F241
:101240003422C1F200021068FFE7438A8B4206D9BC
:1012500000EB81025369C31801D0984205D142F2D4
:101260000B02914203D041694318188870474FF030
:101270000000704728B940F23421C1F2000108682B
:10128000FFE70068704700BF28B940F23421C1F27F
:1012900000010868FFE78088704700BF28B940F266
:1012A0003421C1F200010868FFE7C088704700BF21
:1012B0002DE9F04F89B0BDF8484028B940F23426F6
:1012C000C1F200063068FFE70693468AA64207D9B6
:1012D00000EB84056D694519029501D0A84207D13C
:1012E00042F20B05AC4200F0C48044690419029438
:1012F0000298B0F902A08A44B0F90410551A029875
:10130000C28802EB0A0601894A19019200F1100015
:1013100000900593C3F3C400C3F38521C3F3C44312
:101320009DF81C2060F304028DF81C20BDF81C0001
:1013300061F34A10ADF81C004FEA102163F3C701B6
:101340008DF81D109DF81B80B8F1FF0F04D0019B94
:101350009D42C0F2818089E001998D422EDB85E0BB
:101360005446CAEB08076FEA0A0C0CEB060E0EF0A7
:10137000010B50462946079A17F80A3001F0BAFDCA
:1013800004F10104A64279DC11E020462946079ABF
:101390003B5D01F0AFFD04F1010420462946079AA8
:1013A0003B5D01F0A7FD04F10104A642EDDCC84459
:1013B00005F101050198A84204DC57E0CAEB0609D3
:1013C000DDF80080B245CBDBF2E75446009FCAEB64
:1013D00007076FEA0A0B0BEB060000F0010B17F88A
:1013E0000A1008FB01F389FB0312D3185046294663
:1013F000079AC3F3C71301F07DFD04F10104A6426F
:101400004BDC1FE0385D08FB00F189FB010253183B
:1014100020462946079AC3F3C71301F06BFD04F178
:101420000104385D08FB00F389FB0312D318204642
:101430002946079AC3F3C71301F05CFD04F10104C8
:10144000A642DFDC009903980A18009205F1010515
:10145000019BAB4207DC09E048F28109C8F2800930
:10146000CAEB06020392B245AFDBEFE7029D288884
:1014700001E04FF0000009B0BDE8F08FBBF1000FB4
:1014800083D020462946079A3B5D01F033FD04F1E5
:101490000104A6423FF779AF89E7BBF1000FB1D055
:1014A000385D08FB00F189FB0102531820462946EC
:1014B000079AC3F3C71301F01DFD04F10104A6420E
:1014C000A0DCBFE770B582B0054664460A2804D1A7
:1014D000DCF814200D2A06D11DE00D280CD1DCF813
:1014E00014100A2917D02369E360A068FFF7C2FE31
:1014F0006168081860600EE0DCF80800DCF80C1089
:10150000DCF80420DCF80030AEB20096FFF7D0FE25
:10151000E3681818E06065614FF0000002B070BD2C
:10152000F0B591B016AD55F8046B08900A9107928A
:1015300010AF47F8283D0CAC41F60053C0F206034B
:101540000FCB84E80F00A76041F2C540C0F2020053
:10155000E060204610A908F0E3FB0A9909914FF0DA
:1015600000020B92059503926FF00043029344F042
:101570000104049401A831462A463DF0D5F911B082
:10158000F0BD00BFF0B4DCF8083093422DD9DCF890
:10159000000000F11800DCF80C3003EB430402FB00
:1015A000040213B34FF000034C784FEA94048E7892
:1015B0004FEAD606CD7811F8040B04F007074FEA7E
:1015C000D00040EA47101070507820F0070040EA41
:1015D000D40066F3C7005070957003F1010302F167
:1015E0000302DCF80C009842DED8F0BC704700BF64
:1015F00070B4DCF80830934225D9DCF8000000F123
:101600001800DCF80C304FEA430402FB0402D3B1AB
:101610004FF000034D784FEA95058C784FEAD404DB
:1016200011F8036B4FEAD606108866F3040065F3E1
:101630004A1064F3CF2022F8020B03F10103DCF817
:101640000C009842E6D870BC704700BF704700BFDE
:10165000704700BF10B56446DCF8080020B10DF0FB
:10166000FBFE4FF00003A36010BD00BF10B5644641
:10167000DCF8000020B10DF0EFFE4FF00003236016
:1016800010BD00BF70B56446DCF8080090B1DCF80E
:101690000430DCF800603568D618AE422CBFC3EBCE
:1016A00005051546C0182A463DF006F861684D1933
:1016B000656070BDDCF80450AD18CCF8045070BD06
:1016C0002DE9F04383B005460E4664460FF00EF850
:1016D000E060284631460FF013F8A06028463146F6
:1016E0000FF022F8207403280DD0062802D002281B
:1016F00054D10BE004F1440848F0010848F2655960
:101700004FF003070AE0284610F0F4FA04F1340021
:1017100040F0010840F265594FF00207E368B3F565
:10172000F07F84BF4FF4F073E360A168B1F5887F68
:1017300084BF4FF48871A160A068E26802FB00F0EA
:1017400007FB00F7636813B107F11801196007F18F
:1017500018000CF087FA206000B3E368A16840F637
:101760001F5262F31F4202602068C0F80490226892
:1017700093602368D96021680F6120684FF00002F0
:101780004261009228461146434610F083F92846EC
:1017900010F0A0FA2846314610F0AEF903B0BDE8CB
:1017A000F08300BF2DE9F04F8DB005460E469146FF
:1017B0001F469DF8644000690B90002D00F00683E1
:1017C00040F61F53C0F61F532A689A4240F0FE822B
:1017D0001799002940F3FA82189B002B40F3F682F8
:1017E000AB68B34240F3F282002E06DA8A191792F0
:1017F00000F1EC82BF1B4FF00006D5F80CA0CA45E3
:1018000040F3E482B9F1000F0FDADDF8608018EBE5
:101810000908CDF8608000F1D982DDF858C0C9EB25
:101820000C09CDF858904FF00009B7F5F07F80F221
:10183000CD82002F07DA1799CA19179200F1C682D4
:10184000F61B4FF0000740F29031C1F20001096829
:101850008F4207DA7A1A179FBF18179700F1B682DE
:10186000B61A0F46DDF85C80B84440F29031C1F200
:1018700000018A6808F1FF3C944507DDC8F10101C9
:10188000521817998A18179200F1A082169AB2F589
:10189000887F80F29B82002A09DA189989181891AA
:1018A00000F19482C2EB09094FF00002169240F257
:1018B0009031C1F200014968DDF8588088450ADAA4
:1018C000C1EB080C189A12EB0C02189200F17E8200
:1018D000CCEB090916911699DDF86080884440F236
:1018E0009032C1F20002D16808F1FF3C8C4507DD5F
:1018F000C8F101028918189A5118189100F16682EE
:101900009E4280F26382D14580F260829B1BC7F5C4
:10191000F0729A42B8BF134617998B42B8BF194666
:101920000091C9EB0A02DDF85880C8F5887393422C
:10193000A8BF134618998B42B8BF194601916A692E
:101940002AB905F118014FF0000003900CE00CF0EB
:1019500089F90390002800F039820BA905F11802DB
:101960006B6917F039FA03996B6840F2655293423C
:1019700040F0C480AB68B3F5F07F12D1EA68B2F5ED
:10198000887F0ED10098B0F5F07F0AD1019AB2F5A8
:10199000887F06D1B84800684FF47F4207F094FE74
:1019A0000FE20098C0EB030AC0F5F07B03FB096669
:1019B00001EB46064FF4F073169903FB0177AE4A2C
:1019C000106800EB4707FA2C53D946EA070414F0D5
:1019D000030F09D04FEA4A0A4FEA4B09009D4FEA2C
:1019E000450CA846019D2EE0009A12F0010FF1D19E
:1019F0004FF0020392FBF3F4DDF804800BE038466D
:101A00003146224607F060FEAA6806EB420607F55B
:101A1000707708F1FF38B8F1000FF0D1D1E101F192
:101A200002044988104620F8021B04F10201648870
:101A3000548000F10202023BF1D1674466445644EF
:101A40004F4405F1FF35002D00F0BB81009B002BBA
:101A5000F5D0A6F10202434608F1FF3101F001047E
:101A6000314652883A8007F10202013B40F0B181D1
:101A7000E3E7042C40F2A5814FEA4A0A4FEA4B0BF8
:101A8000009D33E02A463B8803F01F0003F4FC6C02
:101A900003F47841338803F01F09C0EB090804FB05
:101AA00008F9C9F3042803F4FC69CCEB090909FB24
:101AB00004F94FEA292909F4FC6903F478435B1A15
:101AC00003FB04F34FEA232303F47843CC4440445C
:101AD0004CEA0000591840EA01033B80013AD2D198
:101AE00056445F44019800F1FF310191019B002BA6
:101AF00000F0678100990029C4D1F1E748F26550F0
:101B0000834240F0BB80AB68009D581BC5F5F07266
:101B100003FB09634FF0030606FB03114FF4F07556
:101B2000DDF8588005FB0877534B1D6805EB47032C
:101B30000293019D002D00F0448106FB00F0069009
:101B40004FEA42070897009806FB00F00590009ABC
:101B500002F1FF3506FB05F39F1904974FEA450094
:101B600000F10200099048F28105C8F280050A469A
:101B700065E03146FFE7877804FB07F785FB0786BA
:101B8000F7194FEAE717FEB2042E33D9FA2E02D91D
:101B900006880E802EE00E8806F01F0806F4FC6909
:101BA00006F4784C0688FFB206F01F0BC8EB0B0A50
:101BB00007FB0AFBCBF3042A06F4FC6BC9EB0B0B07
:101BC0000BFB07FB4FEA2B2B0BF4FC6B06F4784660
:101BD000CCEB060606FB07F74FEA272707F4784702
:101BE0000BEB0906D04446EA080607EB0C0946EA67
:101BF00009070F8000F1030001F10201867804FB60
:101C000006F685FB0697BE194FEAE617FEB2042ECC
:101C100040F2AD8178E1DDF810C06244029B099981
:101C200058180290069FD219029BDDF8208003EB22
:101C3000080702970199481E019000F0C2800099A0
:101C40000029EFD0DDF8148002EB0803029910465A
:101C50009E1AA6F1030606F001070797967804FB83
:101C600006F685FB0697BE194FEAE616F7B2042F73
:101C700040F2EF80B9E000BF8003001048F688040E
:101C8000A34240F09E80AD68009BE81AC3F5F07255
:101C900005FB096401EB840B4FF4F071169D01FB09
:101CA0000577D04B1C6804EB4701019B002B00F02B
:101CB00088804FEA800704974FEA4205059500980F
:101CC0004FEA80020292009C4FEA440306930D46BD
:101CD00066E013F8010C042847D9FA2816D953F8FE
:101CE000040C0A90C0F38524C0F3C44604F007072F
:101CF000C0F3C40040EA47101070507820F007008D
:101D000040EAD40466F3C70454702EE0168806F047
:101D10001F0706F4FC6C06F4784653F8044CC4F331
:101D2000C409C7EB090800FB08F9C9F304284FEA06
:101D3000541909F4FC69CCEB090900FB09F94FEAD5
:101D4000192909F4FC694FEA142404F47844A41B0B
:101D500000FB04F04FEA102404F4784409EB0C0073
:101D600047443843A6193043108002F1020201F1C2
:101D7000FF3003F1040313F8011C042940F2F3813E
:101D8000A9E1DDF80880C344DDF818904D44DDF882
:101D900010C0E344059BED18019A501E019010D02D
:101DA000009F002FF3D00BF104033946284607F1BA
:101DB000FF3909F0010C13F8012C042A40F22A81A2
:101DC000DDE0039C14B120460DF046FB0DB0BDE8EC
:101DD000F08F002C3FF423AE31F8024F7C8002F1EB
:101DE0000202013B7FF41BAE27E6FA2F2FD8B1F891
:101DF00000B00BF01F080BF4FC690BF4784C17884B
:101E0000F6B207F01F0AC8EB0A0B06FB0BFACAF37F
:101E1000042A07F4FC6BC9EB0B0B0BFB06FB4FEA28
:101E20002B2B0BF4FC6B07F47847CCEB070707FB75
:101E300006F64FEA262606F47847D944D04449EA04
:101E4000080907EB0C0649EA06070F8001E016882F
:101E50000E8000F1030001F1020698423FF4DBAE70
:101E6000079F002F3FF485AE877804FB07F785FBBB
:101E7000078C67444FEAE7175FFA87F8B8F1040F59
:101E800038D9B8F1FA0F33D8B6F800B00BF01F0903
:101E90000BF4FC6A0BF47848B0F800C0FFB20CF009
:101EA0001F0BC9EB0B0B07FB0BFBCBF3042BCDF884
:101EB0001CB00CF4FC6BCAEB0B0B0BFB07FB4FEAE3
:101EC0002B2B0BF4FC6B0CF4784CC8EB0C0C0CFBC0
:101ED00007F74FEA272707F47847DA44DDF81CC0F4
:101EE000E1444AEA090A47444AEA07074F8001E009
:101EF00007884F8000F1030006F10206984218BFE0
:101F000031467FF438AE86E6FA2E2ED80E8806F0DB
:101F10001F0806F4FC6906F4784A0688FFB206F04A
:101F20001F0BC8EB0B0C07FB0CFBCBF3042C06F4CC
:101F3000FC6BC9EB0B0B0BFB07FB4FEA2B2B0BF4DA
:101F4000FC6B06F47846CAEB060606FB07F74FEA79
:101F5000272707F478470BEB0906E04446EA080612
:101F6000BA4446EA0A060E8001E006880E8000F1B7
:101F7000030001F1020198427FF4FDAD4BE6FA2A1D
:101F800032D82E8806F01F0706F4FC6806F478465F
:101F900053F8044CC4F3C40AC7EB0A0902FB09FA5C
:101FA000CAF304294FEA541A0AF4FC6AC8EB0A0A75
:101FB00002FB0AFA4FEA1A2A0AF4FC6A4FEA1424CE
:101FC00004F47844A41B02FB04F24FEA122404F444
:101FD0007842D04409EB070448EA040492191443F8
:101FE0002C8017E08003001053F8042C0A92C2F3EF
:101FF0008524C2F3C44604F00707C2F3C40242EAD0
:1020000047122A706A7822F0070242EAD40466F383
:10201000C7046C7000F1020203F1040301393FF4BC
:10202000B0AEBCF1000F3FF454AE1E4613F8014CA5
:10203000042C48D9FA2C30D8178807F01F0C07F465
:10204000FC6807F4784753F8046CC6F3C409CCEB7A
:10205000090A04FB0AF9C9F304294FEA561A0AF4DB
:10206000FC6AC8EB0A0A04FB0AFA4FEA1A2A0AF4C5
:10207000FC6A4FEA162606F47846F61B04FB06F4C3
:102080004FEA142606F47844D04409EB0C0648EADB
:102090000606E4193443448015E053F8044C0A94CE
:1020A000C4F38526C4F3C44706F0070CC4F3C40484
:1020B00044EA4C148470507820F0070444EAD600B7
:1020C00067F3C700507002F1020203F10403013903
:1020D0007FF4FFAD55E6FA292FD8168806F01F07C2
:1020E00006F4FC6C06F4784653F8044CC4F3C408B8
:1020F000C7EB080901FB09F8C8F304284FEA541993
:1021000009F4FC69CCEB090901FB09F94FEA19292B
:1021100009F4FC694FEA142404F47844A41B01FB7D
:1021200004F14FEA112404F4784409EB0C0147440C
:102130003943A6193143118015E053F8041C0A9164
:10214000C1F38524C1F3C44604F00707C1F3C401F9
:1021500041EA47111170517821F0070141EAD40496
:1021600066F3C704547002F1020203F10403411E36
:102170007FF4AFAD05E600BF2DE9F0419CB00290C1
:10218000039108920DF11C080CAE41F62864C0F2D0
:10219000060494E80F0086E80F00C6F8088041F2B4
:1021A000C163C0F20203F36010AD3046294607F068
:1021B000B7FD18AF94E80F0087E80F00C7F8088054
:1021C00041F28550C0F20200F86038461CA907F0C1
:1021D000A7FD14AE94E80F0086E80F00C6F808804B
:1021E00041F2F151C0F20201F1603046394607F088
:1021F00097FD94E80F0085E80F00C5F8088041F2CC
:102200006D62C0F20202EA602846314607F088FD9E
:102210004FF0000107910691059141F63860C0F238
:10222000060045F0010241F24D63C0F202030FF0D7
:102230004BFC069028B30DF04FFF059008B30698AD
:102240004EF2A161C0F205014FF070020EF0ECF900
:102250003CF0D8FAA8B94FF000030093069819464D
:102260000CAA42F001020FF015FC06984FF0040191
:102270000A460FF0D9FC06980599029A039B0FF0C5
:10228000EBFB06A805A94FF000020FF049FC0798E8
:102290001CB0BDE8F08100BF2DE9F041ADF5BE6D89
:1022A0000DF5BE6747F82C0D0DF5BA6641F62865A9
:1022B000C0F2060595E80F0086E80F00B76041F20E
:1022C0008563C0F20203F3600DF5BC64304621461D
:1022D00007F026FD95E80F0084E80F00A76041F2A3
:1022E0005560C0F20200E06020460DF5BE6107F0C7
:1022F00017FD4FF00001CDF8C015CDF8BC15CDF895
:10230000C815CDF8CC15DDF8C425106830B10BF038
:10231000A9FCCDF8CC05002800F0CA8041F6386051
:10232000C0F206004FF000010DF5BC6343F001025E
:1023300041F25163C0F2020312F0B2FACDF8C005C7
:10234000002800F0A5800DF0C7FECDF8BC050028E0
:1023500000F09E80DDF8C0054EF2A161C0F20501DB
:102360004FF070020EF060F93CF04CFA002840F09B
:102370008F80DDF8C0054FF000010DF5BA6444F020
:1023800001020B4612F030FA4FF0080500954FF0AD
:10239000020601964FF00007029703970497DDF8B5
:1023A000C005DDF8BC154FF4F0724FF4887312F0DD
:1023B0003BF9DDF8C005DDF8BC1512F047FA40F234
:1023C0000004CAF2800404F57F3706AE4FF0010521
:1023D00023460DF11B0104F57074A04693F800C06C
:1023E0004FEACC0E0EF0F80E5A7802F007004FEAD2
:1023F000C00040EA5C104FEA800002F0F8024EEAAA
:102400005E1C01F803CC40EA901001F8020C42EA8D
:10241000521201F8012C03F1020093F802C04FEAB6
:10242000CC0E0EF0F80EDB7803F007024FEAC20282
:1024300042EA5C124FEA820203F0F8034EEA5E1CA5
:1024400001F803CB42EA921201F8022C43EA53133B
:1024500001F8013C00F1020301F103014345BDD144
:10246000CDF8B865DDF8C0050DF5B7612A4612F064
:10247000BFFABC42ACD10DF5BE6454F8300D4FF03C
:10248000000112F0FBF920460DF2BC5112F0E4FA03
:102490000DF5B8600DF2BC514FF000020FF040FB9B
:1024A000DDF8C415DDF8C8050860DDF8CC0501E0ED
:1024B0004FF000000DF5BE6DBDE8F08130B403466D
:1024C00058B940F29034C1F2000441F64062C0F2C3
:1024D00006020FCA84E80F003FE0B0F9004040F266
:1024E0009032C1F200021460B0F902005060B3F9FA
:1024F0000050B3F904106D1805F1FF319160B3F984
:102500000250B3F90630EB1803F1FF33D360002C0F
:1025100006DA40F29032C1F200024FF0000414607B
:10252000002806DA40F29032C1F200024FF00000BB
:102530005060B1F5F07F06DB40F29032C1F200024C
:1025400040F2DF119160B3F5887F06DB40F29033F3
:10255000C1F2000340F20F10D86030BC704700BFDA
:1025600030B585B040F20005CAF2800528464FF02C
:1025700000014FF47F4209F0A7FB4FF00000FFF786
:102580009DFF40F28034C1F20004256041F6E06016
:10259000C0F206008368C3F5F07101EBD173C26825
:1025A000C2F5887101EBD1724FEA620100916FF0C0
:1025B0000042019202924FF0FF0103914FF000019F
:1025C0000A464FEA6303FFF7EDF8104820604FF02A
:1025D0000003009340F23C22C1F2000201924FF04E
:1025E0005001029141F65060C0F206004FF08701A1
:1025F00043F2E542C0F2020221F050FF40F2A43360
:10260000C1F20003186005B030BD00BF00FC83A01C
:1026100030B440F29032C1F20002146851689568FB
:1026200005F101052D1BD26802F10102521A048046
:1026300041808580C28030BC704700BF70B405689F
:1026400040F29034C1F200042668B54209DAAD1BAD
:1026500014686619166040F29035C1F200052C68C6
:1026600004600E6840F29035C1F200056C68A64225
:1026700009DA351B1E6874191C6040F29035C1F2EE
:1026800000056E680E60006840F29034C1F20004EC
:10269000A4681568451904F10106B54203DD201A46
:1026A00000F101001060096840F29034C1F20004AA
:1026B000E0681D684C1900F10105AC4203DD411AC8
:1026C00001F1010119601268002A05DD186800286F
:1026D000D4BF0020012001E04FF0000070BC704723
:1026E00030B484B00B4699B1B1F900200092B1F931
:1026F0000410541804F1FF320292B3F90210019150
:10270000B3F90630CC1804F1FF3203926B4603E0B4
:1027100040F29033C1F2000301881A680CB294426F
:1027200005DA848809198A1A82801C680480418825
:102730005A680CB2944205DAC48809198A1AC28010
:102740005C684480048821B29A68914203DD4FF0AE
:102750000002828008E0B0F9045049198A4203DC83
:1027600002F10102141B848041880AB2DB689A429C
:1027700003DD4FF00003C38008E0B0F906401219F2
:10278000934203DC03F10103591AC180B0F904201C
:10279000002A06DDB0F906000028D4BF0020012081
:1027A00001E04FF0000004B030BC704708B5B1F54F
:1027B000887F36DC0029BCBF5B180021B3F5887F19
:1027C00088BF4FF48873CA18B2F5887FC8BFC1F5B7
:1027D000887340F28430C1F200000268914204DA4A
:1027E00040F28430C1F200000160CB1803F1FF31E8
:1027F00040F2A832C1F200021068814204DD40F2CA
:10280000A833C1F20003196040F23821C1F200017F
:102810000A6832B940F2A430C1F20000006821F029
:1028200005FE08BD00B583B0C0F3C401C0F3852226
:10283000C0F3C4409DF8043061F304038DF8043004
:10284000BDF8041062F34A11ADF804104FEA1122EA
:1028500060F3C7028DF80520BDF8041040F2803007
:10286000C1F20000006841EA01414FF47F4209F0E3
:102870002BFA4FF0000001464FF0FF321346FFF7EE
:1028800095FF03B000BD00BF08B540F2DF139942C9
:10289000A8BF194621EAE17140F20F139A42A8BF7E
:1028A0001A4622EAE27240F2A033C1F200031B781A
:1028B00083420DD140F28833C1F200031B688B4282
:1028C00006D140F28C33C1F200031B68934216D04C
:1028D00040F2A033C1F20003187040F28830C1F218
:1028E0000000016040F28C31C1F200010A604FF03B
:1028F000000001464FF0FF321346FFF757FF08BDB7
:1029000008B5012808D140F23821C1F200010A6857
:1029100002F101020A601BE090B940F23820C1F2D6
:102920000000016801F1FF32026040F27C33C1F225
:102930000003186803280BD952B921F0DBFE07E029
:1029400040F23823C1F200034FF000021A600FE09A
:1029500040F23823C1F200031868B0F1FF3F01D103
:1029600009F050F940F23821C1F200010A6832B989
:1029700040F2A433C1F20003186821F057FD08BDEE
:1029800010B504464FF00000FFF798FD1CB14FF062
:102990000000FFF747FF4FF00200FFF7B1FF4FF0D5
:1029A000000001464FF0FF321346FFF7FFFE10BD57
:1029B00070B48FB0CCB2C3B2E41A02FB04F448F294
:1029C0008103C8F2800383FB04652E194FEAE47487
:1029D000C4EBE61546198DF80460C1F30725C0F372
:1029E00007242E1B06FB02F483FB04652E194FEA15
:1029F000E474C4EBE616C0F3072555FA86F48DF8A7
:102A00000540C1F30746C0F30745741B04FB02F4FD
:102A100083FB04652D194FEAE474C4EBE514C0F39D
:102A2000074555FA84F48DF806404FEA1064C4EB6C
:102A3000116101FB02F283FB021083184FEAE2727C
:102A4000C2EBE31154FA81F38DF8073001980FB00F
:102A500070BC70470000000000B52DED048B83B002
:102A600008EE100ADFEDC67AB4EEE78AF1EE10FA4E
:102A700024DB9FEDC40AB4EEC08AF1EE10FA1DD833
:102A800032F0FEF94FF000024FF40043C4F27B0332
:102A900032F0CEFA01F1004319464FF000024FF038
:102AA0000003C4F24E0332F0BFFC32F005FA09EE27
:102AB000900AF7EE008A9FEDB49ACCE0DFEDB10A00
:102AC000B4EEE08AF1EE10FA23DB9FEDB01AB4EE1B
:102AD000C18AF1EE10FA1CD818EE100A32F0D0F9C3
:102AE0004FF000024FF40043C4F27B0332F0A0FA2F
:102AF0004FF000024FF00003C4F2490332F094FC9F
:102B000032F0DAF909EE100AF7EE008ADFED9E9A4C
:102B1000A1E0DFED9E1AB4EEE18AF1EE10FA22DBBD
:102B20009FED9B2AB4EEC28AF1EE10FA1BD818EE84
:102B3000100A32F0A5F98AA3D3E9002332F078FA1B
:102B400001F100414FF000024FF00003C4F23403E2
:102B500032F06AFC32F0B0F908EE900AB7EE009A53
:102B6000DFED899A77E0DFED8A2AB4EEE28AF1EEB2
:102B700010FA20DB9FED873AB4EEC38AF1EE10FA2B
:102B800019D818EE100A32F07BF975A3D3E90023A7
:102B900032F04EFA4FF000024FF40043C4F25103FA
:102BA00032F042FC32F088F909EE900ADFED768AC5
:102BB000B7EE009A4FE0DFED773AB4EEE38AF1EE3C
:102BC00010FA26DB9FED744AB4EEC48AF1EE10FAD7
:102BD0001FD818EE100A32F053F94FF000024FF4EC
:102BE0002053C4F2840332F023FA01F10043194662
:102BF0004FF000024FF48043C4F2500332F014FC53
:102C000032F05AF909EE100ADFED5F8AF7EE009A0A
:102C100021E0DFED614AB4EEE48AF1EE10FA0DDB5B
:102C20009FED5E5AB4EEC58AF1EE10FA0DD9DFEDD4
:102C3000568AB0EE689AF0EE689A0CE0DFED528AA0
:102C4000B0EE689AF0EE689A05E0DFED4F8AB0EEDC
:102C5000689AF7EE009ADFED525AB4EEE58AF1EE8B
:102C600010FA24DD18EE100A32F00AF902460B467B
:102C70004FF000004FF4C041C4F2880132F0D8F99F
:102C800039A3D3E9002332F019FB4FF000024FF0D3
:102C90000003C4F2540332F0C7FB35A3D3E9002389
:102CA00032F0C8F932F008F907EE100A28E09FED7B
:102CB0003D6AB4EEC68AF1EE10FA1FD518EE100A7E
:102CC00032F0DEF82CA3D3E9002332F0B1F926A3C9
:102CD000D3E9002332F0F2FA4FF000024FF0000384
:102CE000C4F2440332F0A0FB21A3D3E9002332F065
:102CF000A1F932F0E1F807EE100A01E0B7EE007A30
:102D000069EE876ADFED287A26EEA70AFCEEC00A94
:102D100010EE901A29EE071A61EE271ABCEEE12A8E
:102D200012EE102A68EE872A22EEA73AFCEEC33A8A
:102D300013EE903A4FF00000C9B261F30700D2B22F
:102D400062F30F20DBB263F317409DF8071061F3C5
:102D50001F6003B0BDEC048B00BD00BFAFF300806B
:102D60000000000000E07F40666666666666E63F3B
:102D7000333333333333D33F0000000000C0774098
:102D80000000BE430000DC43000000000000F543EB
:102D90000000FF4300001144004021440000434470
:102DA00000002F440000D24300007F43AFF30080B7
:102DB00082B0ADF8042040F29033C1F200031B68EA
:102DC000834220DC40F29033C1F200039B689842BA
:102DD00019DC40F29033C1F200035B688B4212DCD5
:102DE00040F29033C1F20003DB6899420BDCC1EB87
:102DF000011100EB411040F28033C1F20003196869
:102E000092B221F8102002B0704700BFF0B482B037
:102E1000072B6BD940F29034C1F20004246884423D
:102E200064DC40F29034C1F20004A468A0425DDC8E
:102E300040F29034C1F2000464688C4256DC40F2E7
:102E40009034C1F20004E468A1424FDCC1EB0111EF
:102E500000EB411040F28035C1F200052C6804EB14
:102E60004001EF2B2DD80F8807F01F0507F4FC66F3
:102E700007F47841C2F3C4077F1B03FB07F7C7F3CE
:102E800004274FEA521C0CF4FC6CC6EB0C0C03FB41
:102E90000CFC4FEA1C2C0CF4FC6C4FEA122202F4DE
:102EA0007842521A03FB02F34FEA132202F47843EA
:102EB00066447D193543591845EA010224F810206B
:102EC00014E00192C2F38525C2F3C44605F007035E
:102ED000C2F3C40242EA431304F81030487820F0E9
:102EE000070242EAD50366F3C7034B7002B0F0BC99
:102EF000704700BFF0B482B0ADF80420072B58D95A
:102F000040F29032C1F200021268824251DC40F27B
:102F10009032C1F20002926890424ADC40F2903254
:102F2000C1F2000252688A4243DC40F29032C1F2A0
:102F30000002D26891423CDCBDF80420092B38D94C
:102F4000C1EB011100EB411040F28034C1F20004EA
:102F5000246804EB4001EF2B29D80F8807F01F05E8
:102F600007F4FC6607F4784102F01F077F1B07FB9C
:102F700003F7C7F3042702F4FC6CC6EB0C0C0CFB44
:102F800003FC4FEA1C2C0CF4FC6C02F47842521A3D
:102F900002FB03F34FEA132303F4784266447D19DE
:102FA0003543511845EA010324F8103001E024F8B4
:102FB000102002B0F0BC70472DE9F04F87B00746F3
:102FC0000C4600929B46109DC5F3C400C5F38521B5
:102FD000C5F3C4429DF8143060F304038DF8143037
:102FE000BDF8140061F34A10ADF814004FEA102147
:102FF00062F3C7018DF815104FEA15655C4505DDD4
:1030000022465C4693463B46009F00933846214645
:10301000059A2B46FFF76EFF0098C21B46BF52422F
:103020004FF0FF360126BBEB040A27D1002A00F03F
:103030002781934602F1FF3101F00108BF1938469C
:103040002146059A2B46FFF755FFBBF1010B40F0D7
:103050001A8115E1BF1938462146059A2B46FFF71C
:1030600049FF0BF1FF3BBF1938462146059A2B4615
:10307000FFF740FFBBF1010BECD101E132BB0AF1DC
:10308000FF3606F0010604F1010438462146059A90
:103090002B46FFF72FFFBAF1010A40F00481EFE061
:1030A00004F1010438462146059A2B46FFF722FF1A
:1030B0000AF1FF3A04F1010438462146059A2B46ED
:1030C000FFF718FFBAF1010AEAD1D9E0524529D138
:1030D0000AF1FF3E0EF00108BF1904F10104384661
:1030E0002146059A2B46FFF705FFBAF1010A40F089
:1030F000EA80C5E0BF1904F1010438462146059A6B
:103100002B46FFF7F7FE0AF1FF38BF1904F101045F
:1031100038462146059A2B46FFF7ECFEB8F1010A26
:10312000E8D1ADE0524554DA4FEA022191FBFAF0C2
:10313000C3B20193BAF1010ACDF808A000F09B8058
:1031400048F2810AC8F2800A029A02F1FF3808F0B8
:1031500001099846002B40F0C980C6E0CDF80CB0BC
:10316000DDF808B003E0CDF80CB0DDF808B0019A46
:1031700008EB020E5FFA8EF9C14598BFBF1904F142
:103180000104C9F1FF0305FB03F38AFB0310C11817
:103190004FEAE372C2EBE11338462146059ADBB2EF
:1031A000FFF7A8FE05FB09F08AFB00121318B819F7
:1031B0002146059AC3F3C713FFF79CFE0BF1FF3BB3
:1031C000019909EB010C5FFA8CF8C84500F2E48024
:1031D000E1E04FEA0A4ABAFBF2FA5FFA8AF101919A
:1031E000531E029347D048F28108C8F2800803F1C9
:1031F000FF3000F0010A8946002940F0F580F1E037
:10320000CDF80CB0DDF808B003E0CDF80CB0DDF877
:1032100008B0019A09EB020E5FFA8EFACA4598BF10
:103220000134BF19CAF1FF0305FB03F388FB031048
:10323000C1184FEAE372C2EBE11338462146059A02
:10324000DBB2FFF757FE05FB0AF088FB00121318EC
:10325000384604F10101059AC3F3C713FFF74AFE8C
:103260000BF1FF3B01990AEB01095FFA89F9D1459E
:1032700000F212810EE100985946059AFFF798FD79
:1032800007B0BDE8F08FB8F1000F3FF4E3AEBF190F
:1032900038462146059A2B46FFF72CFEBBF1010B61
:1032A0007FF4D8AEECE7002E3FF4FAAE04F101044F
:1032B00038462146059A2B46FFF71CFEBAF1010A53
:1032C0007FF4EEAEDCE7B8F1000F3FF413AFBF19A7
:1032D00004F1010438462146059A2B46FFF70AFE01
:1032E000BAF1010A7FF406AFCAE7BF1904F101047D
:1032F000C8F1FF0005FB00F08AFB001319184FEA24
:10330000E072C2EBE11338462146059ADBB2FFF7C3
:10331000F1FD05FB08F08AFB00121318B8192146CD
:10332000059AC3F3C713FFF7E5FD0299481E029003
:10333000A1D0B9F1000F3FF411AF019A08EB020CD4
:103340005FFA8CF9C14598BFBF1904F10104C9F1B6
:10335000FF0305FB03F38AFB0310C1184FEAE37276
:10336000C2EBE11338462146059ADBB2FFF7C2FDF6
:1033700005FB09F08AFB00121318B8192146059ABB
:10338000C3F3C713FFF7B6FDC8460299481E029063
:103390007FF4E9AE6FE7BF1904F10104C8F1FF0043
:1033A00005FB00F08AFB001211184FEAE073C3EB33
:1033B000E11338462146059ADBB2FFF79BFD05FB7A
:1033C00008F08AFB00121318B8192146059AC3F3B6
:1033D000C713FFF78FFDBBF1010B7FF4C8AEDDF81B
:1033E0000CB048E704F10104BF19C9F1FF0305FB64
:1033F00003F388FB0312D1184FEAE370C0EBE1132B
:1034000038462146059ADBB2FFF774FD05FB09F04B
:1034100088FB00121318384604F10101059AC3F322
:10342000C713FFF767FD0299481E02903FF423AFD0
:10343000BAF1000F3FF4E4AE019A09EB020C5FFA17
:103440008CFACA4598BF0134BF19CAF1FF0305FBC6
:1034500003F388FB0310C1184FEAE372C2EBE113D8
:1034600038462146059ADBB2FFF744FD05FB0AF01A
:1034700088FB00121318384604F10101059AC3F3C2
:10348000C713FFF737FDD1460299481E02907FF41B
:10349000BCAEF0E604F10104BF19C9F1FF0005FB61
:1034A00000F088FB001211184FEAE073C3EBE11340
:1034B00038462146059ADBB2FFF71CFD05FB09F0F3
:1034C00088FB00121318384604F10101059AC3F372
:1034D000C713FFF70FFDBBF1010B7FF49AAEDDF8C8
:1034E0000CB0C8E62DE9F04383B040F23827C1F2B2
:1034F000000740F27C35C1F20005DFF8B88120F00A
:1035000063FF3B6823B12C6804F101042C60F6E7EB
:103510004FF00000286040F28431C1F200010A68D7
:10352000002A06DA40F28434C1F200044FF00006AB
:10353000266040F2A833C1F200031868B0F5887F16
:1035400006DB40F2A831C1F2000140F20F120A601E
:1035500040F28434C1F200042668C6EB061040F243
:10356000A833C1F2000319688A1B02F10102C2EB01
:1035700002144FEA84164FEA96064FEA801404EBD1
:103580008600B0F57F3F01D908F03CFB40F2000314
:10359000CAF28003181908EB0401324606F094F8C9
:1035A00040F2A031C1F200010A78002A72D040F244
:1035B0008036C1F2000640F20004CAF28004346092
:1035C00040F28C30C1F20000046840F28433C1F252
:1035D00000031E68B4422BDB40F2A831C1F20001A7
:1035E0000A68944224DC4FF0FF3000904FF0000056
:1035F000214640F2DF122346FFF7DEFCB4F5877F59
:10360000D4BF013404F1FF3440F28C33C1F2000323
:103610001C6040F28C34C1F2000423684FF07F41FB
:1036200000914FF00000194640F2DF12FFF7C4FC92
:1036300040F28832C1F20002146840F2A830C1F2B0
:103640000000D0F800904FF0FF3300932046314641
:1036500022464B46FFF7B0FCB4F5EF7FD4BF0134F0
:1036600004F1FF3440F28831C1F200010C6040F2F5
:103670008832C1F2000212684FF07F440094104675
:1036800031464B46FFF798FC40F28036C1F2000607
:10369000C6F8008040F28430C1F200006FF00043B1
:1036A000036040F2A831C1F200014FF000020A604D
:1036B00025E700BF00FC83A02DE9F04F8BB00790F9
:1036C000069105920493149C0894C4F3C40AC4F3AD
:1036D00085260196C4F3C4454FEA14649DF854301E
:1036E000002B00F0888007A806A905AA04ABFEF706
:1036F000A5FF002800F09881069F029704997B1887
:103700009F4280F29181C7EB07164FEA4610039063
:1037100040F280329346C1F2000B019ECDF804B016
:10372000079B05995818834257DADDF80CB00BEB6C
:1037300003024FEA42029DF824106AF304018DF857
:103740002410BDF8240066F34A10ADF824004FEAB7
:10375000102165F3C7018DF82510BDF82410092C40
:1037600032D9DDF804C0DCF800008718EF2C2AD825
:103770003F8807F01F0C07F4FC6807F4784701F056
:103780001F0BCCEB0B0904FB09FBCBF3042901F461
:10379000FC6BC8EB0B0B04FB0BFB4FEA1B2B0BF476
:1037A000FC6B01F47841C91B04FB01F14FEA1121C4
:1037B00001F47841D844CC4448EA0C0CCF194CEAC7
:1037C0000701815200E0815203F1010302F102027C
:1037D0000599079841189942ADDC029800F1010063
:1037E0000290039B03F5F07203920499069B5A180A
:1037F000824295DC18E1069804994218904280F2C2
:10380000898040F29031C1F2000140F28037C1F26C
:1038100000070297D1464B6883426EDCCA68824239
:103820006BDB079B059FDA19934266DAC0EB001643
:1038300003EB46174FEA47020E689E4254DC8F683E
:103840009F4251DB9DF8246069F304068DF82460E3
:10385000BDF82470DDF804B06BF34A17ADF824709E
:103860004FEA172665F3C7068DF82560BDF824607A
:10387000092C39D9DDF808C0DCF8007007EB020A22
:10388000EF2C30D8BAF800B00BF01F080BF4FC6A2C
:103890000BF4784C06F01F0BC8EB0B0B04FB0BFB77
:1038A000CBF3042BCDF80CB006F4FC6BCAEB0B0B7E
:1038B00004FB0BFB4FEA1B2B0BF4FC6B06F4784666
:1038C000CCEB060604FB06F64FEA162606F478460D
:1038D000DA44DDF80CB0D8444AEA080A66444AEAF9
:1038E0000606BE5200E0BE5203F1010302F10202DD
:1038F000059E079FBE199E429EDC049A012A08D0AD
:1039000002F1FF33C018069FD219824283DCCA46F7
:1039100000E0CA46079F05997B189F4280F2848089
:1039200040F29031C1F2000140F28030C1F200005B
:103930000390CDF808A00A68BA426BDC8B68BB42E2
:1039400068DB069B04981A18934263DAC3EB0316EC
:1039500007EB46104FEA40024E689E4251DCC868B1
:1039600098424EDB9DF82460DDF808C06CF3040635
:103970008DF82460BDF82400019E66F34A10ADF86E
:1039800024004FEA102065F3C7008DF82500BDF82C
:103990002400092C35D9DDF80CB0DBF8006006EB0B
:1039A000020CEF2C2CD8BCF800B00BF01F080BF465
:1039B000FC690BF4784C00F01F0AC8EB0A0B04FBFF
:1039C0000BFACAF3042A00F4FC6BC9EB0B0B04FBE3
:1039D0000BFB4FEA1B2B0BF4FC6B00F47840CCEB99
:1039E000000004FB00F04FEA102000F47840D944B6
:1039F000D04449EA0809604449EA0000B05200E0B6
:103A0000B05203F1010302F570720498069E30185B
:103A10009842A1DC059A012A06D002F1FF33FF1873
:103A200007981218BA4286DC0BB0BDE8F08F00BFD1
:103A30002DE9F0472DED028B82B005460C460C9F18
:103A40000D9E002A61DD002B5FDD00EB020808F10E
:103A5000FF3801EB0309184631F020F802460B4607
:103A60003AA1D1E9000131F0DFFC31F025FA08EE8E
:103A7000900A4C4549DA6FEA040A0AEB090000F0A3
:103A8000010A9FED318A38EE288AFCEEC87A17EEDB
:103A9000902A38463146D2B2FEF78AFF0090284677
:103AA000214642462346FFF787FA04F10104A14567
:103AB00030DC2AE038EE288AFCEEC80A10EE902AA4
:103AC00038463146D2B2FEF773FF009028462146B1
:103AD00042462346FFF770FA04F10104A24638EE8D
:103AE000288ABCEEC81A11EE103A38463146DAB2CE
:103AF000FEF75EFF00902846214642462346FFF728
:103B00005BFA04F10104A145D4DC02B0BDEC028BE8
:103B1000BDE8F087BAF1000FCCD038EE288ABCEEB1
:103B2000C80A10EE103A38463146DAB2FEF740FFC6
:103B300000902846214642462346FFF73DFA04F10D
:103B40000104A145B6DCE0E7000000000000000031
:103B500000E06F40AFF3008010B340F2AC33C1F22D
:103B6000000393ED001AB5EEC01AF1EE10FA06D874
:103B700040F2B432C1F2000292ED000A704740F206
:103B8000EC30C1F2000090ED000A40F2E831C1F2E1
:103B90000001D1ED001A31EEC02A01EE020A704791
:103BA00040F2B833C1F20003D3ED007AF5EEC07AEB
:103BB000F1EE10FA06D840F2B432C1F2000292EDF2
:103BC000000A704740F2EC30C1F2000090ED000AAC
:103BD00040F2E831C1F2000191ED007A77EE400A3F
:103BE00007EEA00A704700BF08B540F2E433C1F207
:103BF00000031868B0B140F2F401C1F20001087886
:103C000040F2B432C1F20002116805F0F9F84FF049
:103C1000000000F0CDF940F2B033C1F200034FF0E4
:103C20000000187008BD00BF10B582B040F2BC3370
:103C3000C1F20003186850B340F2F401C1F2000170
:103C40000C784FF00000FFF787FF204610EE101AA7
:103C500005F0D6F840F2B033C1F200034FF0010294
:103C60001A7040F2E430C1F20000016879B14FF0FF
:103C700000030093019340F2C030C1F200004FF006
:103C8000FF0243F6E933C0F2020321F0A9F902B0C2
:103C900010BD00BF10B4044628B140F2AC30C1F2F0
:103CA00000000068206029B140F2B830C1F2000085
:103CB000006808602AB140F2BC31C1F20001086816
:103CC00010602BB140F2E432C1F2000211681960B9
:103CD00010BC70470246C8B140F2B033C1F20003D5
:103CE0001878012808D002280DD140F2AC33C1F277
:103CF00000031868106009E040F2B831C1F2000119
:103D00000B68136002E04FF00001116040F2B03226
:103D1000C1F200021078704730B583B040F2F4036E
:103D2000C1F200031878032853D040F2B031C1F239
:103D300000010C781CB94FF0010000F039F940F295
:103D4000F402C1F2000215784FF00100FFF704FF02
:103D5000284610EE101A05F053F840F2B033C1F2C5
:103D600000034FF00200187040F2BC31C1F20001B4
:103D7000096881B14FF000000090019040F2C0301E
:103D8000C1F200004FF0FF0243F62943C0F20203E4
:103D900021F026F91FE040F2E432C1F2000211687E
:103DA00081B14FF000030093019340F2C030C1F2A3
:103DB00000004FF0FF0243F6E933C0F2020321F0A6
:103DC0000FF908E040F2C030C1F2000021F062F8C3
:103DD00001E04FF00004204603B030BD10B540F2C2
:103DE000AC34C1F20004206040F2B830C1F20000EF
:103DF000016040F2BC31C1F200010A6040F2E432DD
:103E0000C1F200021360FFF787FF10BD10B540F24A
:103E1000F404C1F20004207040F2E830C1F2000066
:103E2000016040F2B431C1F200010A6040F2EC32AC
:103E3000C1F2000213604FF07E5049F69A11C3F6AA
:103E400099614FF078024FF41673FFF7C7FF10BD6A
:103E500010B548F21C02C2F20902136843F01000C8
:103E6000106048F20004C2F20904216841F0100316
:103E7000236041F66C60C0F2060001684CF210034A
:103E8000C4F202031960106840F480731360226862
:103E900042F4807020604CF22004C4F202042160DD
:103EA00048F23C01C2F209014FF400330B604CF2BE
:103EB000C400C4F20F00026842F00104046041F63D
:103EC0006861C0F20601086848F20803C2F20803FC
:103ED000186041F66062C0F2060214684CF2B81134
:103EE000C4F20F010C604CF28810C4F20F0003689A
:103EF000C3F38102C3F38124944208DC02F101027E
:103F000062F38B234CF28811C4F20F010B6041F66F
:103F10006460C0F20600046841F67461C0F20601F4
:103F2000A1F1040301F1680103F104025B681C6064
:103F30005068046002F10803926814608B42F3D168
:103F40004CF20814C4F20204216841F400702060AD
:103F500041F67063C0F206031A6848F20004C2F228
:103F60000804226041F65861C0F20601086848F270
:103F70000403C2F20803186048F21004C2F20804F5
:103F800040F20002CAF28002226041F65C61C0F297
:103F90000601086848F21804C2F2080420604CF2D6
:103FA000503022F0B9FD236843F40062226010BD56
:103FB00010B580B148F21804C2F20804216841F03B
:103FC000010222604FF0640022F0A6FD236843F452
:103FD0000060206010BD48F21804C2F20804236893
:103FE0006FF3CB2323604FF0640022F095FD20682F
:103FF0006FF30000206010BD51B148F21801C2F209
:1040000009014FF480130B604FF480020A6070477F
:1040100048F21C03C2F209034FF480121A604FF4F5
:1040200080001860704700BFF0B583B04FF01C00EF
:1040300001A94FF0040205F027FC4FF08503C8F2F8
:104040006813019A9A4234D040F20000CAF200008C
:1040500040F20001CAF2001102F09EFED0B94FF00A
:1040600008054FF001074AF22014C0F207044FF090
:104070000006284639463A4624F0BEFC204622F087
:104080004BFD28463146324624F0B6FC204622F04D
:1040900043FDEEE74FF08501C8F2681102A840F831
:1040A000041D4FF004014FF01C0205F07BFC07F0EB
:1040B0009DFD03B0F0BD00BF08B540F20003C5F29E
:1040C000000340F2F430C1F20000194640F2000251
:1040D000C5F28002D21A4FF46063C0F22773FCF776
:1040E0009BFB4FF00100FCF74BFF43F27050C0F216
:1040F0000600FDF717F84FF005004FF0000144F2FD
:104100009912C0F2020206F041FE4FF0030043F69E
:10411000F971C0F2020144F28912C0F2020206F003
:1041200035FE45F6D820C0F2060021F0D5FA4FF052
:1041300040004FF0010105F0D1FC4FF003004FF0BB
:1041400001010A464FF0120306F0C0F840F2184091
:10415000C1F200004FF60001CAF287014FF480322D
:104160004FF002032EF094FA40F23040C1F200000A
:1041700044F24401C4F202014FF014024FF0030371
:104180002EF086FA08BD00BF08B519B94FF005003A
:1041900030F0B6F908BD00BF08B5012903D14FF0D2
:1041A000030030F0ADF908BD002817DD40F2F03112
:1041B000C1F200010A68831846F6E800CAF28900D5
:1041C00040F20001CAF20011091A8B4212D880187D
:1041D00040F2F032C1F200021360704700280CDA9E
:1041E00040F2F033C1F200031A68801818604FF0F3
:1041F000000070474FF0FF30704746F6E800CAF203
:104200008900704708B507F0FDFC08BD4FF0280095
:10421000704700BF08B50368196B4068884740F2D3
:104220004840C1F200004FF0000280F8642008BD51
:104230002DE9F04F87B005468B4601929A4640F231
:10424000B043C1F200031C68E4B14FF00007B84668
:10425000B9464FF6FF76B54203D020680188A942DF
:104260000CD1226893684BB105A804A903AA98470A
:104270000598814404998844039ABF186468002C07
:10428000E9D103E04FF00007B846B946BBF1000F93
:1042900001D0CBF80090019B0BB1C3F80080BAF1BC
:1042A000000F01D0CAF8007007B0BDE8F08F00BF62
:1042B0002DE9F04105460F46904640F2B043C1F269
:1042C00000031C68A4B14FF000024FF6FF76B54220
:1042D00003D020680188A94206D12368996A19B1E0
:1042E00038468847024628B96468002CEFD101E0BF
:1042F0004FF00002B8F1000F01D0C8F800202046AE
:10430000BDE8F08108B54FF0020045F64441C0F227
:10431000060146F20932C0F2020221F00FFA08BD8E
:10432000F0B591B004468569436943B14FF000018F
:1043300041616A68002A00F0C9809047C6E0C06801
:10434000002800F0C3804FF00001E160206869465A
:104350004FF0400221F006FD0246AB681BB120463B
:1043600069469847B2E0A569BDF80400012840F00D
:10437000AD8000998A4240F0A9804FF0000EC5F848
:1043800004E0C5F81CE0C5F820E0C5F80CE005F134
:1043900024066F460FCF0FC697E80F0086E80F0080
:1043A000C5F844E042F20102A5F84A2005F15000A8
:1043B00071464FF014023AF0B3F96B8D41F20900E7
:1043C000834277D01CD841F204018B423ED009D8F9
:1043D00041F20202934275D076D802F1FF30834257
:1043E00054D159E041F206018B4233D030D301F170
:1043F00001018B4230D001F101018B4246D12DE009
:1044000049F60102934237D012D841F20C008342A0
:1044100026D004D800F1FF318B4237D14CE041F275
:104420000D02934221D002F1070293422ED121E0E6
:1044300049F603018B4223D020D301F102018B42C4
:1044400020D001F10B018B4220D11DE020492BE04F
:10445000204929E0204927E0204925E0204923E0A0
:104460002048A8604FF0000127E01F4BAB604FF0E1
:10447000000122E01D4917E01D4915E01D4913E028
:104480001D4911E01D490FE01D490DE042F20502F2
:10449000A5F84A201B4907E01B4905E042F2190034
:1044A000A5F84A00174900E081B12068224621F0B2
:1044B000FFFB0BE0154900E0154995F86430002B2F
:1044C000ECD1F1E71349EFE71349EDE711B0F0BD87
:1044D000C94B0200115C020061450200154A02004E
:1044E000355A020049500200994F0200715F0200E4
:1044F000C9470200CD4C020051590200FD5602008E
:10450000D14602001D4502007960020031490200D7
:10451000955F0200414602003146020070B5064632
:10452000946904F14405636C03F10C0363644FF078
:10453000030284F848204FF0000084F84900E26A42
:10454000E2648B4201D907F05DFB30462946626C7C
:104550003AF0B2F84FF00001E162606C70BD00BF4C
:104560002DE9F04383B0804689461746966940F2AC
:104570001D53C1F200031878F8B1326B40F220519C
:10458000C1F200010B8843F480318A421ED040F210
:104590002054C1F200044FF0000310F0010F34D09A
:1045A00003F101052B46854205D234F8021F41F480
:1045B0008031914232D1834208D1306BB0F1FF3F5C
:1045C00004D042F20803A6F84A3016E0726B02F1FA
:1045D000FF3313F1030F04D842F21402A6F84A2065
:1045E0000BE0308E4FF000010A4601ABFFF720FED2
:1045F0004FF00401716401983065404649463A46DF
:10460000FFF78CFF03B0BDE8F08303F1010334F83A
:10461000021F41F480319142C2D1CCE705F1010380
:1046200034F8021F41F480319142B9D1C3E700BF91
:1046300010B593694FF000041C60FFF76FFF10BDC9
:1046400038B593691C682CB142F21E05A3F84A5094
:104650001C6501E01C6B1C60FFF760FF38BD00BFEC
:104660002DE9F84380460E4691460A9D2C686CB3AE
:104670000F6800682218974203D80899CA19904217
:1046800004D30898C7193760BDE8F883C71B08989A
:10469000C11B8C4228BF0C46099A32B1D9F80000E0
:1046A0001018D91922463AF007F82B68191B29600F
:1046B000D8F800201019C8F80000D9F800301919EE
:1046C000C9F800103268BF183C193460BDE8F8839F
:1046D000F0B58DB005460591164694694FF000037C
:1046E0000B93E3614FF6FF70216B07AAFFF7E0FD24
:1046F000079848B942F20903A4F84A3028460599B8
:104700003246FFF70BFF35E04FF0100108914FF0F4
:104710000202ADF8242049F61006ADF82660E76ADB
:104720000A9704F1200704F11C064FF00C030093D4
:10473000019505A80290384631460BAA08ABFFF751
:104740008FFF0599A9B14FF0000206924FF00403C4
:104750000093019505A80290384631460BAA06AB96
:10476000FFF77EFF059921B144F65D72C0F20202A7
:1047700062600B980DB0F0BDF0B5A5B01C78ADF837
:1047800011406CB14FF0000404F1010413F8015F13
:1047900024AF07EB440626F87F5C002DF4D101E03E
:1047A0004FF0000404F1010424AB03F8804D4FEAFC
:1047B000440404F1010400942A9C01942B9C02946B
:1047C000FFF74EFF25B0F0BDF0B58BB00746059161
:1047D00094694FF000030693E3614FF01C000790CB
:1047E0004FF00201ADF8201049F60102ADF8222089
:1047F000E56A099504F1200604F11C054FF00C034D
:104800000093019705A802903046294606AA07ABF7
:10481000FFF726FF0599002900F086804FF0060279
:1048200007924FF004030093019705A802903046C9
:10483000294606AA07ABFFF713FF0599002973D095
:104840004DF60142ADF81C204FF002030093019792
:1048500005A802903046294606AA07ABFFF700FFDD
:104860000599002960D04DF60242ADF81C204FF0AA
:1048700002030093019705A802903046294606AA34
:1048800007ABFFF7EDFE059900294DD04DF6034229
:10489000ADF81C204FF002030093019705A8029089
:1048A0003046294606AA07ABFFF7DAFE059900292C
:1048B0003AD04DF60442ADF81C204FF002030093AD
:1048C000019705A802903046294606AA07ABFFF7D4
:1048D000C7FE059941B34DF64142ADF81C204FF09B
:1048E00002030093019705A802903046294606AAC4
:1048F00007ABFFF7B5FE0599B1B14DF64442ADF8EF
:104900001C204FF002030093019705A80290304647
:10491000294606AA07ABFFF7A3FE059921B144F685
:104920005D72C0F20202626006980BB0F0BD00BF7B
:10493000F0B58BB00646059194694FF000030993DA
:10494000206A0B283BD84FF6FF70216B04F114024C
:10495000FFF7AEFC2061656925B10268516A09B1B3
:1049600093693BB942F20901A4F84A104FF00003E1
:10497000A36108E028469847A061206905686A6A33
:10498000606990476061A06900F10C0006904FF0EB
:104990000205ADF81C5041F20902ADF81E20E16A93
:1049A00008914FF00C030093019605A8029004F1C2
:1049B000200004F11C0109AA06ABFFF751FE65694E
:1049C000ADB1059F236AA3F10C03A2690092019681
:1049D00005A9029104F1200004F11C0109AAEB18B9
:1049E000FFF73EFE05983F1AA369DA1BA2610999F9
:1049F00009B1059850B123691A68D16B09B1606992
:104A0000884744F65D70C0F20200606009980BB000
:104A1000F0BD00BF2DE9F04F8DB0074605919569B7
:104A20004FF000030B93EB61D5F830C01FFA8CF404
:104A300040F21D50C1F2000090F800E0BEF1000FFE
:104A40001CD040F22051C1F200010B88A34221D0BA
:104A500040F22051C1F200014FF000031EF0010F9F
:104A600000F0A28003F101000346704504D231F842
:104A7000026FA64240F0A08073450BD1BCF1FF3F0E
:104A800008D042F20800A5F84A0038460599FFF719
:104A900045FD86E0696B01F1FF3313F1030F08D880
:104AA00042F21401A5F84A1038460599FFF736FD81
:104AB00077E020464FF000010A4607ABFFF7B8FB4E
:104AC000079A02F104024FEA820008904FF00201B7
:104AD000ADF8241041F20703ADF82630EA6A0A92D5
:104AE00005F1200805F11C094FF00C00009001971A
:104AF00005A90291404649460BAA08ABFFF7B0FD55
:104B0000059B002B4CD04FF004020092019705A8A2
:104B10000290404649460BAA07ABFFF7A1FD059955
:104B200000293DD040F2B046C1F200063668002EA2
:104B30002DD04FF0040BA2464FF6FF739A4503D0D9
:104B40003268108850451FD13168CB68E3B198476F
:104B5000044617E03268116A204688470690CDF86F
:104B600000B0019705A80290404649460BAA06AB43
:104B7000FFF776FD059B9BB13268116921B1204694
:104B800088470446002CE5D17668002ED4D10B98D6
:104B900008B1059B23B144F65D72C0F202026A605F
:104BA0000B980DB0BDE8F08F03F1010331F8020F4F
:104BB000A0427FF457AF5FE700F1010331F8020F25
:104BC000A0427FF44FAF57E72DE9F04F8BB08146FD
:104BD000059196694FF000030693F36140F21D5072
:104BE000C1F20000017801F104014FEA810207924D
:104BF0004FF00207ADF8207041F20403ADF8223007
:104C0000F06A099006F1200706F11C084FF00C012C
:104C10000091CDF8049005AA02923846414606AAB2
:104C200007ABFFF71DFD059B002B49D040F21D503F
:104C3000C1F20000017807914FF004020092CDF814
:104C4000049005AB02933846414606AA07ABFFF72E
:104C500007FD0598002833D040F21D51C1F2000134
:104C60000A7822B3184D4FF000044FF0010B40F2C8
:104C70001D539A46C1F2000A35F8020FADF81C0028
:104C8000ADF81EB04FF004010091CDF8049005AAD4
:104C900002923846414606AA07ABFFF7E1FC059BA6
:104CA00073B104F101049AF80000A042E4D8069917
:104CB00009B1059A22B144F65D73C0F20203736034
:104CC00006980BB0BDE8F08F1E0500102DE9F041ED
:104CD0008EB00546059194694FF000030693E36199
:104CE000208EA0F55C4101F1FF33432B4BD8DFE868
:104CF00013F05300F400F400F7004A004A004A00A1
:104D00004A004A004A0053004A004A004A004A004A
:104D10004A004A004A004A004A004A004A004A0043
:104D20004A004A004A004A004A004A004A004A0033
:104D30004A004A004A004A004A004A004A004A0023
:104D40004A004A004A004A004A004A004A004A0013
:104D50004A004A004A004A004A004A004A004A0003
:104D60004A004A004A004A004A004A004A004A00F3
:104D70004A0044004A004A0047004FF01A060DE07E
:104D80004FF00B060AE04AF60101A4F84A10284643
:104D90000599FFF7C3FBA6E04FF00E0606F10C02E3
:104DA00007924FF00207ADF8207007F51840ADF8F4
:104DB0002200E16A099104F1200804F11C074FF078
:104DC0000C030093019505AA02924046394606AAB3
:104DD00007ABFFF745FC059800287CD0218EA1F594
:104DE0005C4303F1FF30432864D8DFE800F0222B56
:104DF00037406363636363635B63636363636363DA
:104E00006363636363636363636363636363636372
:104E10006363636363636363636363636363636362
:104E2000636363636363636363636363636349636C
:104E3000635207A845F6B841C0F20601324639F080
:104E40003BFC37E007A845F6C841C0F206013246F0
:104E500039F032FCA28EADF821202BE007A845F6F0
:104E6000C831C0F20601324639F026FC22E007A81C
:104E700045F6FC21C0F20601324639F01DFC19E06E
:104E800007A845F68C41C0F20601324639F014FC01
:104E900010E007A845F67041C0F20601324639F02D
:104EA0000BFC07E007A845F6A841C0F20601324610
:104EB00039F002FC0096019505A902914046394659
:104EC00006AA07ABFFF7CCFB059B23B144F65D7048
:104ED000C0F202006060069805E04FF00C065DE746
:104EE0004FF012065AE70EB0BDE8F0812DE9F84305
:104EF00080460E4691460A9D2C686CB30F68006888
:104F00002218974203D80899CA19904204D30898E6
:104F1000C7193760BDE8F883C71BD9F80010089897
:104F2000421A944228BF1446099820B1C019591852
:104F3000224639F0C1FB2B68191B2960D8F80020E4
:104F40001019C8F80000D9F800301919C9F8001074
:104F50003268BF183C193460BDE8F88310B5846925
:104F6000626C02F10C0262644FF0030384F8483073
:104F70004FF0000184F84910E36AE364006804F12B
:104F8000440120F0B9FE94F8640000B9E0624FF0EB
:104F90000002A260626010BDF8B5064684693F2A2F
:104FA0008CBF00270127E36923B901F10C01A2F1AD
:104FB0000C0500E0154620690268936B60692A467B
:104FC000984768B922691368196B6069884742F28B
:104FD0000C00A4F84A00E2695319E36127B329E001
:104FE000002F2BD02269136899696069884740F2C5
:104FF000B442C1F20002136A984209D023691868CA
:10500000016B6069884742F20702A4F84A2004E075
:1050100020690168CA6B606990474FF000036361C3
:10502000E0694119E16105E0B4F84A1042F201007B
:10503000814207D03046FFF791FFF8BDE16948197A
:10504000E061F1E7F8BD00BF2DE9F04F8BB00590AE
:105050008A46164684694FF00003099345F61039D5
:10506000C0F2060940F2D84BC1F2000B40F2B44046
:10507000C1F20000049048E0E2684FEA021009EB38
:1050800000054FF00003079319F8001002297AD0A9
:1050900001290BD19BF800204FEA42000890696873
:1050A000884205D9431A0793089101E06F68089771
:1050B000AA68B2F1FF3F14BF5A44002204F120084D
:1050C00004F11C070096019208A802904046394658
:1050D00009AA5346FFF70AFF00964FF0000101911D
:1050E00007AB02934046394609AA5346FFF7FEFE36
:1050F0000898079A111841B9EB6813B143F0010001
:105100000047E36803F10103E36009998E42B3D8D5
:10511000402E38D1CCE0DBF8082004990A62F0E791
:10512000BBF8010040B34FF00003FF2888BF3F20C9
:10513000049A985403F10103BBF80310002940F0CE
:10514000BA801BE0FF2988BF3F21195403F10102F7
:1051500013460BEB4201B1F8011079B1FF2988BF6A
:105160003F21815402F101030BEB4302B2F801101D
:10517000002940F0A28001E04FF000034FF0000052
:10518000049AD054BDE74FF000036361208E06A956
:105190001A46FFF74DF840F2B441C1F20001086A27
:1051A000069A904204D942F20C03A4F84A307CE0FB
:1051B000268E04F1140840F2B045C1F200052D68B6
:1051C0009DB14FF0000140F2B447C1F200072B68D7
:1051D0001888B04205D1DA6A1AB1384690470146BC
:1051E00028B96D68002DF2D101E04FF00001B8F14F
:1051F000000F00D06161616921B142F21D01A4F884
:105200004A1052E0268E40F2B445C1F20005D5F8AE
:1052100020A040F2B043C1F200031D68B5B14FF0C9
:10522000000140F2B449C1F200090F462868028823
:10523000B24207D1436B2BB1484651463A46984794
:10524000014628B96D68002DF0D101E04FF0000152
:10525000B8F1000F00D061612561606920B942F2A8
:105260000C02A4F84A2020E029680A6A02B190479B
:10527000B4F84A1042F20103994216D1228EA4F8E2
:1052800050204FF000014FF0010384F8523084F8B1
:10529000531084F8541084F8551084F8561084F88C
:1052A0005710A0654FF00C0060640598FFF756FE9C
:1052B0000BB0BDE8F08F049844E71F2B7FF442AF9A
:1052C0005CE700BF2DE9F04188B0804640F2B04570
:1052D000C1F200054FF0000440F21C57C1F2000774
:1052E0004FF001062B6853B11A7A1AB11C72186874
:1052F000016C19B95B68002BF6D100E03BB940F2B4
:105300001C51C1F200014FF000020A7028E03E700B
:105310001A68136C0DF1030001A998479DF803006A
:10532000012809D010B10228DCD102E044F20303C5
:1053300004E044F2070301E044F202034FF01002DC
:1053400002924FF00401ADF80C10ADF80E304FF0A2
:10535000FF300490019B0593404602A920F0CCFC4D
:1053600008B0BDE8F08100BF08B543692BB14FF02C
:10537000000141610078FFF7A5FF08BD10B5144694
:105380004DF6044398422BD009D84DF6024188428D
:105390001CD020D801F1FF3290423DD111E04DF6F2
:1053A0004143984221D004D84DF60B41884233D175
:1053B0002AE04DF6444290421CD0B0F1FF3F2BD181
:1053C00030E04FF001034FF0040028E04FF00103FC
:1053D0004FF0020023E04FF001034FF002001EE007
:1053E0004FF001034FF0080019E04FF001034FF0B8
:1053F000100014E0084639F05FFA4FEA400000F16F
:1054000003004FF001030AE04FF00003184600F1DB
:10541000040003F1010302E04FF0000318465CB101
:10542000236010BD084639F047FA4FEA400000F10A
:1054300023004FF00603EAE710BD00BF2DE9F0435B
:105440008BB007460E4690469946A0F55C4404F1A1
:10545000FF34432C75D8DFE804F0222C31407474FB
:1054600074747474717474747474747474747474FF
:1054700074747474747474747474747474747474EC
:1054800074747474747474747474747474747474DC
:10549000747474747474747474745174745F0A6979
:1054A00013681888ADF818004FF00101ADF81A1014
:1054B00047E04FF44051ADF8181042E00869016828
:1054C0004A691AB170690DF1170190479DF81730BC
:1054D00003F00100ADF8180033E00D692C68A369F2
:1054E0002BB14869984704464FF0000503E04FF0A0
:1054F00000044FF00005CDE9064522E006A84FF074
:1055000000014FF0100239F00BF933691868016A95
:1055100070698847069014E00B691868C169706962
:1055200088470346CDF80090129A019206F12000B8
:1055300006F11C014246FFF71FF918E04FF0000288
:105540000692384646F67C71C0F206014FF0000222
:10555000FFF714FF0090CDF80490129A029206F122
:10556000200006F11C01424606ABFFF779F80BB0AC
:10557000BDE8F083F0B585B005466446CCF8001070
:10558000A080A0F55C4303F1FF30432861D8DFE839
:1055900000F022272C3160606060606040606060D5
:1055A00060606060606060606060606060606060FB
:1055B00060606060606060606060606060606060EB
:1055C00060606060606060606060606060606060DB
:1055D00060603660603B4FF00601ACF806101CE0DE
:1055E0004FF00400ACF8060017E04FF00403ACF8ED
:1055F000063012E04FF00807ACF806700DE04FF0EF
:105600000A02ACF8062008E04FF6FF71ACF806106D
:1056100003E04FF00606ACF80660216A04F11C06B0
:1056200004F114074FF008020092A3690193029756
:1056300001F1200001F11C0132462346FFF710F86A
:10564000606930B1216AA369009728463246FFF7A6
:10565000F5FE05B0F0BD00BF38B56446DCF820307B
:105660001A691068016A58698847054623699A686B
:10567000B2F1FF3F09D1606968B938BDA4464DF663
:105680000B402946FFF776FF38BDA44690B2294665
:10569000FFF770FF38BDA4464DF601402946FFF7DD
:1056A00069FF616941B3A4464DF602402946FFF700
:1056B00061FF636903B3A4464DF603402946FFF733
:1056C00059FF6269C2B1A4464DF604402946FFF76E
:1056D00051FF606980B1A4464DF641402946FFF76D
:1056E00049FF616941B1A4464DF644402946FFF7A0
:1056F00041FF6369002BC1D138BD00BF70B590B0C8
:1057000015460C900B9193690E934FF000040D9485
:10571000DC610E9B03F130020A921A6A0B2A03D94C
:105720004FF00C01D961C3E0DA6B3AB14AF60702D7
:10573000A3F84A202A46FEF7F1FE07E11A6C3AB1B7
:105740004AF60802A3F84A202A46FEF7E7FEFDE0E3
:105750005A6B3AB142F21402A3F84A202A46FEF7E5
:10576000DDFEF3E0986B46F67C71C0F2060105AAF7
:10577000FFF704FE059850B94AF601000E9BA3F806
:105780004A000C980B992A46FEF7C8FEDEE04FF05F
:1057900000010E9B99610A9A116819B34FF6FF70C8
:1057A0000E9A02F11402FEF783FD0E9A10610E9B11
:1057B000586948B942F20902A3F84A200C980B999B
:1057C0002A46FEF7ABFEC1E00A9CA46819690A6884
:1057D000D36998470146204605AAFFF7CFFD0E99E9
:1057E000886141E04FF00000059040F2B041C1F205
:1057F00000010A680E9B1A610E980069002833D0D8
:105800004FF000040168CA68002A25D090470E9B1B
:1058100058611DE095690A9EB66811690B68DA69DE
:1058200090470146304604AAFFF7A8FD40190E999B
:105830008861049B059AD01805900E990B691A6827
:10584000136923B1486998470E99486100E04C619B
:105850000E9A50690028DDD10E98026953680361E1
:105860000E9908690028CDD10E99059800F1020221
:105870008B6903EBC20006904FF00202ADF81C20CA
:1058800049F60503ADF81E30C86A08904FF00C02C7
:1058900000920C9B01930BA8029001F1200001F1F2
:1058A0001C010DAA06ABFEF7DBFE0B9900294CD0BC
:1058B000059806900E994FF0040300930C9A0192FC
:1058C0000BA8029001F1200001F11C010DAA06AB0A
:1058D000FEF7C6FE0B99002937D00A9B1A683AB129
:1058E0000DF1180CFFF7B8FE0B9A002A2DD022E01C
:1058F00040F2B040C1F2000001680E9B19610E9A9F
:105900001369C3B11868C16869B188470E9B5861B3
:1059100005E00DF1180CFFF79FFE0B99A9B10E9A47
:1059200050690028F5D10E9B1A69506818610E99CC
:105930000B69002BE6D10D9808B10B9929B144F6FB
:105940005D720E9BC0F202025A600D9810B070BDDD
:10595000F0B58DB006460591154694694FF00001EB
:105960000B91E161226A0B2A4CD84FF6FF70216B34
:1059700004F11402FEF79CFC2061616939B942F21E
:105980000900A4F84A004FF00002A26115E0A78EBA
:105990000068C26908469047014638464FF0000249
:1059A000FFF7ECFCA06140B94AF60103A4F84A30C5
:1059B0004FF00001A161616101E063692BB93046DC
:1059C00005992A46FEF7AAFD32E0A16901F10C0112
:1059D00006914FF00200ADF81C0049F60302ADF845
:1059E0001E20E36A08934FF00C010091019605A870
:1059F000029004F1200004F11C010BAA06ABFEF793
:105A00002FFE02E04FF00C03E36162693AB1A08E11
:105A100005AB009321460BAA3346FFF70FFD0B9809
:105A200008B1059921B144F65D72C0F202026260CC
:105A30000DB0F0BD2DE9F04796B00646059117462A
:105A400094694FF0000315938DF81B30E3614FF616
:105A5000FF70216B07AAFEF72BFC0546079848B993
:105A600042F20900A4F84A00304605993A46FEF78A
:105A700055FDCAE02A68D169884781462868476988
:105A80001FB107980DF11B01B847484638F014FFC5
:105A900000F123004FEA400308934FF00202ADF8F3
:105AA000242041F20801ADF82610E06A0A9004F1C2
:105AB000200804F11C074FF00C030093019605AA7F
:105AC00002924046394615AA08ABFEF7C9FD059972
:105AD000002900F099802868B0F800A09DF81B50BC
:105AE00005F00105836913B10798984701E04FF06D
:105AF0000000ADF820A04FF00102ADF822204FF4D5
:105B00004051ADF82410ADF826500A904FF0000037
:105B1000ADF82C00ADF82E00ADF83000ADF8320035
:105B2000ADF83400ADF83600ADF83800ADF83A0005
:105B3000ADF83C00ADF83E00ADF84000ADF84200D5
:105B4000ADF84400ADF84600ADF84800BDF84A3065
:105B500060F30F03ADF84A30139014904FF0340205
:105B60000092019605A902914046394615AA08AB54
:105B7000FEF776FD0598002846D0009605AB019308
:105B80004046394615AA4B46FEF7F6FD059A002A0F
:105B90003AD04FF000018DF820104FF00100009036
:105BA000019605AB02934046394615AA08ABFEF7AD
:105BB00057FD059A42B34FF000018DF820104FF0C9
:105BC00001000090019605AB02934046394615AAA4
:105BD00008ABFEF745FD059AB2B14FF000018DF814
:105BE00020104FF001000090019605AB0293404653
:105BF000394615AA08ABFEF733FD059A22B144F6E3
:105C00005D71C0F202016160159816B0BDE8F087C1
:105C10002DE9F04190B00546059194694FF00003DD
:105C20000F93E36140F21D50C1F2000090F800E0D4
:105C3000BEF1000F21D0266B40F22051C1F20001CD
:105C40000B8843F48030864220D040F22051C1F2CC
:105C500000014FF000031EF0010F00F0B38003F1CC
:105C600001000346704506D231F8027F47F48037C1
:105C7000B74240F0B180734508D142F20800A4F861
:105C80004A0028460599FEF749FC98E0B6F1011F45
:105C900014D040F2B042C1F2000213689BB1B6B218
:105CA0001F683988B14201D17F6887B95B68002BD2
:105CB000F6D145F6FC37C0F2060708E045F6FC379A
:105CC000C0F2060703E045F6FC37C0F20607384687
:105CD00038F0F2FD00F101020D9200F11F004FEAD1
:105CE000400006904FF00206ADF81C6041F205013D
:105CF000ADF81E10E36A089304F1200804F11C06B5
:105D00004FF00C020092019505A8029040463146E2
:105D10000FAA06ABFEF7A4FC059900294ED0208EF1
:105D20000EA90DAA4FF00003FEF782FA4FF0000310
:105D30004FF00302ADF818204FF00100ADF81A0043
:105D4000ADF81C300D99CDF81E10CDF822300E9A0A
:105D5000CDF82620CDF82A304FF0FF33ADF82E30A5
:105D6000ADF830304FF01A000090019505A902916E
:105D7000404631460FAA06ABFEF772FC059AEAB11F
:105D8000009505AB0193404631460FAA3B46FEF70E
:105D9000F3FC059890B1009505A901914046314664
:105DA0000FAA45F63843C0F20603FEF7E5FC059A54
:105DB00022B144F65D73C0F2020363600F9810B025
:105DC000BDE8F08103F1010331F8020F40F48030A7
:105DD000B0427FF444AF4EE700F1010331F8020F07
:105DE00040F48030B0427FF43AAF44E7F0B58DB074
:105DF00005460591164694694FF000030B93E06841
:105E000000287BD1E061216AC1B945F61040C0F29B
:105E10000600FBF785F8606148B942F20A00A4F871
:105E20004A00284605993246FEF778FB9BE0FAF7D0
:105E30006DFEA0616069FAF77FFE6061A26902F100
:105E40001A0208924FF00206ADF8246041F21407DE
:105E5000ADF82670E36A0A9304F1200704F11C06EA
:105E60004FF00C000090019505A90291384631468B
:105E70000BAA08ABFEF7F4FB059A002A6AD04DF294
:105E80000543ADF8203044F20200ADF822004FF097
:105E900000018DF824104FF005020092019505AB2A
:105EA0000293384631460BAA08ABFEF7D9FB05989A
:105EB00000284FD04FF0000107914FF004020092EC
:105EC000019505AB0293384631460BAA07ABFEF7A6
:105ED000C7FB059800283DD04FF0040100910195C3
:105EE00005AA0292384631460BAA04F11803FEF7C0
:105EF000B7FB059B002B2DD01C4EE660059F079736
:105F000004F1200704F11C066369A1690091019561
:105F100005AA0292384631460BAAFEF7A1FB059866
:105F2000079B1A1A079261698B186361A1698A1A23
:105F3000A26178B14FF000008DF820004FF001030E
:105F40000093019505A90291384631460BAA08AB8A
:105F5000FEF786FB0B9808B1059A22B144F65D73F3
:105F6000C0F2020363600DB0F0BD00BFFC5E020032
:105F700038B593691C6B4DF20545AC4202D1FFF771
:105F800035FF38BD42F21B04A3F84A40FEF7C6FABB
:105F900038BD00BFF0B587B007460E461546946978
:105FA0004FF000038DF80F30216BB1F1FF3F04D1AA
:105FB00042F20600A4F84A003DE042F20902A4F8C9
:105FC0004A204FF6FF7004F11402FEF771F9014602
:105FD000606980B311B10B681A6B62B32161096803
:105FE0004B691BB10DF10F01984700BB9DF80F00E5
:105FF000E8B921690B680493606905904FF00802C5
:10600000009245F61840C0F206004FF0070144F236
:106010001522C0F2020204AB1EF054FB42F2010151
:10602000A4F84A104FF0010384F8643003E042F210
:106030000D02A4F84A20384631462A46FEF76EFA89
:1060400007B0F0BD10B582B00C4640F20012C0F2AD
:10605000000292F8463092F84720009245F624421A
:10606000C0F2060236F07EF800F10100A04228BF1F
:10607000204602B010BD00BF2DE9F04399B005469F
:10608000059194694FF000030793E361206A0B28A0
:106090002AD89B4838F010FC06464FF000004FF01D
:1060A0004001FFF7CFFF32184FEA420606F1C5065E
:1060B00008964FF00203ADF8243041F20100ADF82C
:1060C0002600E16A0A914FF00C020092019505AB9F
:1060D000029304F1200004F11C0107AA08ABFEF7AB
:1060E000BFFA059818B907E14FF00C01E16145F6D8
:1060F000F426C0F2060608AA3068716803C204F1EB
:10610000200804F11C064FF008010091019505AB31
:1061100002934046314607AA08ABFEF7A1FA05985C
:10612000002800F0E9804FF000098DF820904FF032
:1061300001070097019505AF02974046314607AA2F
:1061400008ABFEF78DFAADF820904FF002020092F6
:10615000019502974046314607AA08ABFEF780FA40
:106160000599002900F0C88018AF4FF0120347F8D6
:10617000403D09A845F6D431C0F206014FF0240293
:1061800038F09AFA4FF028000090019505AA029283
:106190004046314607AA3B46FEF762FA05990029B8
:1061A00000F0AA8018AF4FF0030347F8403D09A85C
:1061B00040F2F801C1F200014FF0060238F07CFA1B
:1061C0004FF00A000090019505AA02924046314620
:1061D00007AA3B46FEF744FA0599002900F08C8097
:1061E00018AF4FF0010347F8403D09A845F6F831D4
:1061F000C0F206014FF0020238F05EFA4FF00600DE
:106200000090019505AA02924046314607AA3B46F6
:10621000FEF726FA059900296ED0CDF820904FF0B0
:1062200004000090019505AA02924046314607AA53
:1062300008ABFEF715FA059900295DD018AF4FF0AD
:10624000040347F8403D09A845F6C031C0F20601F5
:106250004FF0080238F030FA4FF00C000090019532
:1062600005AA02924046314607AA3B46FEF7F8F9D6
:106270000599002940D0009505AB01934046314671
:1062800007AA45F66043C0F20603FEF775FA0598C3
:10629000002831D0009505AA01924046314607AA50
:1062A000174BFEF769FA059931B308A84FF0400182
:1062B000FFF7C8FE009505AB01934046314607AA9B
:1062C00008ABFEF759FA0598B0B108A84FF02001C5
:1062D0004A461FF04BFD18AA111801F8409C009582
:1062E00005A801904046314607AA08ABFEF744FADC
:1062F000059A0AB103496160079819B0BDE8F083B7
:10630000160100005D4F020000B583B00378A12B99
:106310004AD1407866284AD0672820D0642802D025
:106320004FF002004EE0062A44D10A8844F20103ED
:106330009A4242D1D1F8021040F24840C1F2000026
:10634000C26A91423CD1204B4FF0000159601F4876
:106350001FF020FA1FF02AFC4FF0010032E040F25B
:106360004840C1F20000C26A6AB940F24843C1F233
:10637000000393F8641042F2190042F2010300296D
:1063800018BF034601E042F219034FF00402ADF8D2
:106390000420ADF806304FF000000DEB02011FF0B5
:1063A000ABFC4FF003000DE04FF002000AE04FF0AD
:1063B000010007E04FF0020004E04FF0020001E0AE
:1063C0004FF0020003B000BD48040010D45C06008A
:1063D00010B5044640F2B043C1F200031B68002B25
:1063E00031D002681188186802888A4214BF0022DE
:1063F0000122A34208D110BD186802888A4214BF46
:10640000002201229C4226D05B68A2B9002BF3D166
:1064100019E005F0F7FB40F21D53C1F200031A78B2
:106420002068008840F22051C1F2000121F81200DA
:1064300002F101021A7040F2B043C1F200031A687F
:1064400062601C6010BD40F21D51C1F200010A786B
:10645000032AE0D9DDE710BD08B54FF00103037250
:1064600040F21C50C1F20000017839B945F67C4079
:10647000C0F206001FF08EF9FEF724FF08BD00BF32
:1064800040F23053C1F200031868A0F103007047D6
:1064900045F62850C0F20600704700BF4FF6FD7069
:1064A000704700BF4FF6FD7398420CBF184600209E
:1064B000704700BF4FF6FD73984214BF02200020C2
:1064C000704700BF4FF6FD730B604FF00001017085
:1064D000704700BF08B540F20010C1F20000FFF79E
:1064E00077FF08BD08B540F20010C1F20000FFF7C9
:1064F000B3FF45F63C50C0F206004FF0070146F2EC
:106500000D52C0F202021EF0E9F808BD2DE9F04775
:10651000C2B041F288301EF01FF94FF00000FAF7C8
:10652000A9FE05464FF00000FAF7B8FE00EB050A99
:1065300040F22853C1F200031868C1787E290ED0BA
:1065400045F65453C0F2060300934FF00000014695
:1065500052464FF0FF33FAF7E3FFAA44BAE045F69C
:106560007852C0F2060200924FF0000001465246F7
:106570004FF0FF33FAF7D4FF4FF0000001464FF021
:10658000FF321346FCF712F90AEB0504A2461EF08F
:10659000B1F821F091FF98B945F69452C0F2060285
:1065A0000092014622464FF0FF33FAF7B9FF4FF051
:1065B000000001464FF0FF321346FCF7F7F889E080
:1065C00045F6A453C0F2060300934FF000000146C5
:1065D00022464FF0FF33FAF7A3FF4FF000000146C9
:1065E0004FF0FF321346FCF7E1F804EB050A1EF00A
:1065F00081F840F23050C1F200000168042925D929
:106600004FF482744FF0040340F22858C1F200089E
:106610004FF040073E4E40F23059C1F2000900E011
:106620000446D8F8002002A8D1183A4603F04CF8E6
:1066300002A831194FF4807203F00EFB30B904F553
:1066400080702346D9F80010A142E9D840F22852C0
:10665000C1F20002106800F1040040F20001C0F233
:10666000010140F23053C1F200031A6835F08AFA92
:10667000B0B145F6C451C0F2060100914FF00000E0
:10668000014652464FF0FF33FAF74AFF4FF0000041
:1066900001464FF0FF321346FCF788F8AA4419E090
:1066A00045F6D450C0F2060000904FF000000146BD
:1066B00052464FF0FF33FAF733FF4FF00000014628
:1066C0004FF0FF321346FCF771F84FF0010023F052
:1066D000E7F81AE045F6E050C0F2060000904FF0EF
:1066E0000000014652464FF0FF33FAF719FF4FF012
:1066F000000001464FF0FF321346FCF757F842F214
:1067000010701EF029F805F07DFA42B0BDE8F08760
:10671000FCFE000038B5144640F22853C1F20003D5
:106720001B68D3B140F23052C1F200021068251844
:1067300040F22C52C1F200021268954210D818188B
:10674000224637F0B9FF40F23051C1F200010B6828
:10675000E4180C604FF0010038BD4FF0000038BD68
:106760004FF0000038BD00BF00B583B040F22853A1
:10677000C1F200034FF000021A604FF02E0136F014
:10678000D3F8002848D045F60061C0F2060135F084
:106790002FFD002840D123F083F840F20000C0F222
:1067A0000100214B181A40F22C52C1F20002106075
:1067B00007F058FA40F22851C1F20001086058B3BE
:1067C0004FF00100FCF7DCF84FF00000FAF766FD2F
:1067D000024645F60860C0F2060000904FF0000047
:1067E00001464FF0FF33FAF79BFE40F22C53C1F203
:1067F00000031A6840F22851C1F2000108684FF006
:10680000FF314FEA920205F05FFA40F23050C1F2D8
:1068100000004FF00303036040F22852C1F200026F
:10682000106803B000BD00BF080002004FF0FF3346
:1068300003600B604FF000001060704740F234536B
:10684000C1F200031868704745F67060C0F2060098
:10685000704700BF4FF6FE70704700BF4FF6FE73E3
:1068600098420CBF18460020704700BF4FF6FE73D9
:10687000984214BF02200020704700BF2DE9F00F9E
:1068800084B040F24453C1F200031868002800F0BD
:10689000018140F23453C1F20003186810181860E7
:1068A000002A00F0FA8040F24454C1F20004256846
:1068B00002950E46891840F23853C1F200034FF09A
:1068C000000245F62877C0F20607009740F200095B
:1068D000C0F2000940F2000AC5F2000A40F20000CE
:1068E000C5F28000019040F20004CAF20004039453
:1068F00016F8015B1C79A5F14107F8B2052803D809
:10690000A5F13700C7B208E0A5F13007FFB2092FA3
:1069100003D9002C40F08F80174693F809C047EA4E
:106920000C105FFA80FC83F809C0D87900F10100EF
:10693000C0B2D87110F001080AD193F808B0E3444E
:1069400083F808B093F806B00BF1FF3B83F806B06C
:10695000062C05D8DFE804F0060D1B2440565E0027
:10696000104663E0532D58D14FF0010018711046C6
:106970005FE0DDF800C01CF8070000285BD05F7105
:106980001A721A604FF002001871104651E0022886
:1069900045D183F806C04FF003001871104648E057
:1069A0001D6847EA05171F605D79DDF800B01BF828
:1069B0000550B0EB450F34D19879012804D14FF040
:1069C00005001871104634E04FF004051D7107F101
:1069D000FF371F60104629E0B8F1000F23D11D6872
:1069E00005F101051D60587900F1FF35E8B2022874
:1069F0008CBF002001209D79012D17D14FF0050497
:106A00001C7116E0022810D1187AFF2813D11A71D0
:106A100010460EE04FF0020008E0104606E0104677
:106A200004E0104602E0104600E010461D79A54241
:106A30000BD0DA7109E040F23851C1F200014FF099
:106A400006030B714FF000002CE0022828D001282B
:106A50001AD1186848450DD340F20004C0F208046A
:106A6000A04207D85C7AC9EB0000DDF808C00CF83A
:106A7000004009E0504507D3019CA04204D8CAEB6E
:106A800000005C7A039D44558E427FF431AF4FF095
:106A9000010007E04FF0000004E04FF0010001E0CA
:106AA0004FF0000004B0BDE8F00F704708B540F2A9
:106AB0000C10C1F20000FFF78BFC08BD08B545F6CD
:106AC0008060C0F206004FF0070146F6D922C0F2FE
:106AD00002021DF003FE08BD2DE9F04184B002AFB3
:106AE00041F2C862C0F2060241F61803C0F2060382
:106AF000981A20F0030101F10A0121F00702ADEB21
:106B0000020D0DF1080841F288301DF025FE1EF03F
:106B1000D3FD4FF00000FAF705FB41F61050C0F22C
:106B20000600FAF7FDF9002800F0AE804FF00000F3
:106B3000FAF7A0FB04464FF00000FAF7AFFB051987
:106B40002E4640F20003C0F2000340F20010C0F2F3
:106B50000000C21A40F24451C1F2000108684CF62C
:106B6000DE63CEF6A55382589A4274D14FF00000EE
:106B7000FAF706FA00286ED045F69866C0F20606C7
:106B800000964FF0000001462A464FF0FF33FAF717
:106B9000C7FC4FF0000001464FF0FF321346FBF7F1
:106BA00005FE2E191DF0A6FD40F20003C5F20003FC
:106BB000184640F20001C5F28001C91A07F104022B
:106BC0003B462DF0CDFD45F6B460C0F206000090C6
:106BD0004FF00000014632464FF0FF33FAF7A0FCB9
:106BE0004FF0000001464FF0FF321346FBF7DEFD89
:106BF00036191DF07FFD786840F20001CAF20001ED
:106C00003A682DF075FD45F6D062C0F2060200929A
:106C10004FF00000014632464FF0FF33FAF780FC98
:106C20004FF0000001464FF0FF321346FBF7BEFD68
:106C300036191DF05FFD41F2C863C0F206034046FD
:106C4000194641F61802C0F20602D21A37F034FD96
:106C500008F10108C04745F6E051C0F20601009175
:106C60004FF00000014632464FF0FF33FAF758FC70
:106C70004FF0000001464FF0FF321346FBF796FD40
:106C800042F210701DF068FD04F0BCFF07F1080728
:106C9000BD46BDE8F08100BF70B58AB004463D4DE9
:106CA00003A845F6E861C0F206012A4635F070FAFD
:106CB000204603A935F09CFA064603A845F6F06184
:106CC000C0F206012A4635F063FA204603A935F0E2
:106CD0008FFA08B1002E55D14FF0000022F0E0FDF0
:106CE00040F23850C1F200004FF000014FF00C02AA
:106CF00037F016FD40F20003C0F2000340F200043A
:106D0000C0F20804E41A204606F0ACFF40F24451F9
:106D1000C1F200010860A8B34FF00100FBF730FE9C
:106D20004FF00000FAF7BAFA024645F6F860C0F2F2
:106D3000060000904FF0000001464FF0FF33FAF7D5
:106D4000EFFB40F24452C1F2000210684FF0FF31F5
:106D50004FEA940204F0B8FF40F20000CAF20000CB
:106D600040F20003CAF280031A1A4FF0FF314FEAD3
:106D7000920204F0A9FF40F23451C1F200014FF039
:106D80000000086040F24453C1F2000318680AB0E2
:106D900070BD00BF160100002DE9F00F82B04FF06A
:106DA000000301930093019B4FF0010201920260E6
:106DB0006FF0010343600268012A0BD14FF0020318
:106DC00003606FEA0302426002689A4204D15300F2
:106DD000F6D101E04FF001030093009A002A40F041
:106DE000CD804FF002070197091A21FA07F707F142
:106DF000FF3212F0010F00F0D3804FF001034FF08B
:106E0000AA3440F823404FEA43031342F9D1BBE0D0
:106E100003F1FF3440F8245000EB830650F8234080
:106E2000B4F1AA3F04D023E04FF001034FF05535F1
:106E30004FEA43031A42EBD1B9E000EB850640F874
:106E400025800368B3F1AA3F12D1634650F823406E
:106E5000B4F1AA3F01D09D420AD14FEA4303134245
:106E6000F4D1C6F800904FEA45051542E5D102E09D
:106E7000002E40F086804FF003020192C1F17F495D
:106E800009F58019002F6ED009EB07084B466FEA11
:106E9000090404EB080202F00102044644F8049BD2
:106EA00003F10103434540F0C5800CE0224642F85F
:106EB000043B03F101031D46636003F1010302F18A
:106EC00004044345F2D1036899454FD100F1040A07
:106ED00052464D4603464FF0000617F0010F09D108
:106EE0008BE01346144654F804CBA346AC4500F09F
:106EF00092803EE06FEA05041C6005F1010506F191
:106F00000106BE42EDD102686FEA090991452FD111
:106F10004FF00103CFF61073591A6FEA01016FEABF
:106F2000080803464FF00000C8EB010212F0010F01
:106F300013D055E05346524652F8046B154601F102
:106F4000FF348E4215D1CAF800001346DAF8045017
:106F500002F1040AA5424DD00BE018604145E9D189
:106F60004FF0000305E04FF0000302E0034600E0AD
:106F70000346D3F1010038BF00202DE04FF00000A0
:106F80002AE04FF0000027E04FF055330360036024
:106F90004368B3F1AA3F18BF061D7FF469AF43E70A
:106FA0004FF0553303604FF0AA32026063E70646A4
:106FB0004FF0AA3346F8043B4FF055334360036863
:106FC000B3F1AA3F7FF454AF4FF00105AC464FF048
:106FD000AA394FF0553838E702B0BDE8F00F7047D6
:106FE000186053465AF8044B01F1FF328C42C0D16D
:106FF0001146B2E704F1FF31AFE76FEA090404601C
:1070000009F1010406F10106534652F8045BA5425A
:107010003FF470AFADE76FEA0C0515600CF1010CA1
:1070200006F101062346556804F1040265453FF464
:1070300061AF9EE7002A3FF439AF44F8043B03F107
:10704000010343457FF432AF3DE700BF11B1012991
:1070500016D108E040F21811C1F200010B7813704C
:107060004FF00000704748F29400C2F20900016836
:1070700081F48033C3F3004010704FF0000070477C
:107080004FF01400704700BF11B1012926D118E05C
:1070900044F24001C4F202010B6813F4003F44F2D1
:1070A0004000C4F202000168C1F3100318BF5B4244
:1070B00007EE103AF8EEC70AC2ED000A4FF00000E2
:1070C000704740F24C50C1F20000D0ED007AB8EEAB
:1070D000670A82ED000A4FF0000070474FF014007D
:1070E000704700BF684620F007018D4601B440F2AA
:1070F0000002C4F209021368136003F01000C1B269
:1071000000293ED040F25852C1F20002136883B900
:1071100040F22C00C4F20900016840F24852C1F26A
:107120000002116040F24C53C1F200034FF0000026
:10713000186040F25851C1F200010A68B2F5006FC0
:107140000FD140F22C03C4F20903186840F24851F1
:10715000C1F200010A68801A40F24C53C1F20003E8
:10716000186040F25851C1F200010A68B2F5006F90
:1071700007D840F25850C1F20000036803F1010340
:10718000036001BC8546704708B54FF4005045F6D2
:107190006871C0F2060140F25C52C1F2000221F0B7
:1071A0006FFA08BD38B514464FF00003137000297C
:1071B00040F0978040F25050C1F200000168002971
:1071C00040F092804FF0000000F004FC4CF2C40547
:1071D000C4F20F052A6842F480032B6045F6407024
:1071E000C0F2060001684CF2C815C4F20F05296010
:1071F0004CF2EC03C4F20203186840F25452C1F29C
:107200000002106045F63471C0F206010D681D6081
:1072100045F65C73C0F20603186840F27002C4F2CF
:107220000902106045F64471C0F206010D684CF287
:107230003C13C4F202031D6045F63870C0F206002C
:10724000026840F22801C4F209010A6045F660753F
:10725000C0F2060528684CF23813C4F20203186025
:107260004FF0000540F20C02C4F20902156040F232
:107270001401C4F209010D6040F20400C4F20900D7
:1072800045F66473C0F206031A68026045F63C7165
:10729000C0F206010B68036045F64870C0F20600B4
:1072A0004FF0070147F24932C0F202021DF016FA10
:1072B00040F25052C1F20002106047F2E500C0F205
:1072C00002004FF00F014FF0030204F0B9FD4FF040
:1072D000010040F21811C1F2000108702070284628
:1072E00038BD4FF0140038BD4FF0000038BD00BF6E
:1072F00070B540F25853C1F200034FF000021A601B
:107300001DF020FF054643F2D30440F25856C1F267
:1073100000061DF017FF401BA04209D940F21810CB
:10732000C1F200004FF0050202704FF0000070BD86
:107330001DF0E0F93168B1F5006FEAD940F24C5325
:10734000C1F20003186870BD70B54FF0000001462F
:1073500003F088F9FFF7CCFF064640F21813C1F29C
:1073600000031878012840F0EA8030462DF0B6FB83
:1073700004460D4684A3D3E900232EF0E3F938B97F
:107380002046294682A3D3E900232EF0F7F938B12D
:1073900040F21811C1F200014FF002030B70CEE071
:1073A000FFF7A6FF044640F21811C1F200010A7867
:1073B000012A40F0C480864294BFC6EB0006C0EBB1
:1073C0000606012E55D9FFF793FF054640F2181324
:1073D000C1F200031878012840F0B180AC4294BF9C
:1073E000C4EB0504C5EB0404012C3FD9FFF780FF73
:1073F000044640F21811C1F200010A78012A40F057
:107400009E80854294BFC5EB0005C0EB0505012DAC
:107410002FD9FFF76DFF054640F21813C1F20003A4
:107420001878012840F08B80AC4294BFC4EB05046F
:10743000C5EB0404012C1BD9FFF75AFF044640F2A8
:107440001811C1F200010A78012A78D1A84234BF8C
:10745000C0EB0505C5EB0005012D0AD940F2181453
:10746000C1F200044FF00203237068E02C4600E0F4
:107470002C4620462DF032FB04460D4646A3D3E9A8
:1074800000232EF05FF9D0B143A1D1E900012246DB
:107490002B462DF0CDFD02460B46204629462DF009
:1074A000C3FF4FF000024FF00003C3F6E0732DF06E
:1074B000C1FD2DF0ABFC04464FF001051AE020465B
:1074C000294635A3D3E900232DF0B2FD02460B4631
:1074D00031A1D1E900012DF0A7FF4FF000024FF0DC
:1074E0000003C3F6E0732DF0A5FD2DF08FFC0446DC
:1074F0004FF00005B4F5003F0AD340F21813C1F273
:1075000000034FF004021A704FF000052C460AE009
:107510002846214603F0A6F840F21810C1F20000F8
:107520004FF0000101702846214603F0B1F830B950
:1075300040F21814C1F200044FF0030020704FF025
:10754000000440F22802C4F20902146020464FF001
:107550000F014FF0030204F073FC40F25450C1F2EB
:10756000000001684CF2EC03C4F20203196040F21F
:107570005052C1F2000214604FF0010000F02AFAEC
:1075800070BD00BFAFF3008000000000EE0D63414E
:1075900000000000B217634100000000D0126341F8
:1075A00070B515461C464FF00003237031BB40F206
:1075B0005050C1F20000016819BB10462EF0FCF8D3
:1075C00007EE905ABCEEE70A10EE106AD0F1010007
:1075D00038BF002010EE101A03F05AF828462EF09B
:1075E000EBF8D0F1010038BF0020314603F03AF843
:1075F0004FF0010222704FF0000070BD4FF01400F8
:1076000070BD4FF0000070BD4FF0000303600B60D1
:107610004FF001001060704740F28453C1F2000344
:107620001868A0F58030704740F28453C1F200031F
:107630001A68A2F58033984206D141B14FF000009C
:1076400008704FF0030070474FF0020070474FF092
:107650000300704740F28053C1F20003186870477E
:1076600040F28453C1F200031868A0F580307047DF
:1076700040F28453C1F200031968A1F580328242BE
:1076800018BF0020704700BF4FF00000704700BFD8
:1076900008B540F21C10C1F20000FEF799FE4FF44D
:1076A0007D43C0F2020340F28052C1F20002136037
:1076B00008BD00BF08B540F28453C1F200031A6848
:1076C000A2F580330B6040F27851C1F200010B78D3
:1076D0000370BBB902F10102B2F57A7F40F2845027
:1076E000C1F2000028BF0022026040F27851C1F2CE
:1076F00000014FF001020A7040F21C10C1F20000BC
:10770000FEF7AAFE08BD00BF08B540F27C53C1F2E7
:107710000003186808B107F09FFE4FF47D40C0F2E7
:10772000020040F28052C1F20002106040F2785133
:10773000C1F200014FF000030B7040F21C10C1F2C7
:107740000000FEF789FE08BD08B540F28050C1F286
:1077500000004FF47D43C0F202030360FAF79CFD82
:1077600040F27C51C1F20001086008BD10B540F242
:107770006854C1F2000420464FF00D0145F6E07256
:10778000C0F2060240F28453C1F200031B6834F0D9
:10779000E9FC204610BD00BF48F23403C2F20903E1
:1077A000196811F0020F17D040F29551C1F2000193
:1077B0000A78002A4BD138B148F2B801C2F2090167
:1077C0004FF002020A60704748F2BC00C2F20900A2
:1077D0004FF002030360704740F29552C1F200027D
:1077E0001378A3BBD0B140F29451C1F200010A78E2
:1077F00042BB45F6FC73C0F20603196840F23C0236
:10780000C4F20902116045F6F873C0F20603196864
:1078100040F20402C4F20902116013E046F234019E
:10782000C0F206010A6840F20403C4F209031A60B8
:1078300046F24001C0F206010A6840F23C03C4F27D
:1078400009031A6040F29453C1F2000318707047A4
:1078500040F29453C1F200031878704707EE902A63
:10786000002949D140F29550C1F200000178002969
:107870003CD140F20402C4F20902107820F0010168
:1078800011709FED207AF4EEC77AF1EE10FA17DD51
:107890009FED1D0AF4EEC07AF1EE10FA10D577EEE6
:1078A000A70A9FED1A1AC1EE201ABCEEE12A40F297
:1078B0002401C4F2090181ED002A4FF0000108E023
:1078C00040F22402C4F209024CF2867010604FF0BC
:1078D000160140F20402C4F20902107840F00100DF
:1078E0001070107840F00200107001E04FF00001BD
:1078F00019704FF0000070474FF000021A704FF0FF
:10790000140070470000C8420000FA45C0E1E44C92
:1079100010B584B048F23403C2F20903186810F0BD
:10792000020F3FD14CF2C401C4F20F010A6842F4C5
:1079300080040C6046F24403C0F20603186840F26B
:107940007001C4F20901086046F23C02C0F206026E
:10795000146840F21403C4F209031C604FF00004E1
:10796000009401944FF0030202924FF005004FF093
:107970000101234601F07CFC40F22400C4F209001E
:107980004CF28671016040F20C02C4F209021460EC
:1079900046F23803C0F20603186840F20401C4F24C
:1079A0000901086004B010BD08B5FFF7B1FF45F646
:1079B000F070C0F2060021F037FE4FF0140046F2DE
:1079C0000001C0F2060140F28852C1F2000220F02C
:1079D00057FE08BD08B548F23403C2F2090319681E
:1079E00011F0020F1AD140B140F29550C1F20000DF
:1079F00002789AB1FFF78CFF08BD40F29550C1F2B2
:107A00000000027852B94FF00000FFF7C5FE40F2C7
:107A10009553C1F200034FF00101197008BD00BF7A
:107A200030B400F2671292B240F2CE239A4210D9DB
:107A300046F2B704CBF20B6484FB00452B184FEAE7
:107A4000E074C4EB23254FF4B47303FB150423B295
:107A500000E00346002BBCBF03F5B4731BB2A3F1D7
:107A60005B05ACB2B3F5877F08DDA3F5877346F2FB
:107A70004C05C0F2060535F8133015E0B42B08DDCF
:107A8000C3F5877346F24C05C0F2060535F813308E
:107A90000AE05A2BCCBF5A3BC3F15A0346F24C05BD
:107AA000C0F2060535F81330B22C9CBF5B429BB286
:107AB000CB800B8040F2CE239A420FD946F2B70218
:107AC000CBF20B6282FB00231B184FEAE072C2EB81
:107AD00023234FF4B47202FB130000B20028BCBF92
:107AE00000F5B47000B2B0F5877F0ADDC0F5B4725E
:107AF00046F24C03C0F2060333F81220B42816DC19
:107B000018E0B42808DDA0F1B40046F24C02C0F23F
:107B1000060232F810200AE05A28C8BFC0F1B400AB
:107B200046F24C03C0F2060333F8102002E0C2F123
:107B3000000082B24A80C2F100038B8030BC7047E3
:107B400070B4039C1D88491B5E88B21A0DB216B230
:107B5000B0F90210B0F9062002FB06F201FB052283
:107B600002F18002B0F90010B0F9040006FB00F643
:107B700005FB016101F180014FEA212121804FEADB
:107B8000222262801888091821805B889A1A6280F4
:107B900070BC70472DE9F04186B007460E4614468A
:107BA0001D46B2F90010B2F9022005AB009333462E
:107BB000FFF7C6FFA18820880918B4F9022004AB9A
:107BC0000093384609B23346FFF7BAFFB4F9001004
:107BD000E2886088121803AB0093384612B233462D
:107BE000FFF7AEFFA18820880918E288648812197F
:107BF00002AB0093384609B212B23346FFF7A0FF3A
:107C0000BDF91070BDF914108F42B4BF3846084654
:107C1000BDF90C60B042A8BF3046BDF90840A04293
:107C2000A8BF204680B28F42ACBFB8468846BDF997
:107C300012C0BDF91670BC45B4BF63463B46BDF9E2
:107C40000E108B42A8BF0B46BDF90A209342A8BF75
:107C500013469BB2BC45A8BF674628806B80B045E1
:107C6000A8BF4646A642ACBFC0EB0600C0EB04006E
:107C7000A8808F42A8BF39469142ACBFC3EB010335
:107C8000C3EB0203EB8006B0BDE8F0812DE9F04FB5
:107C9000ABB005461646349C9DF8D480CDF83C80A8
:107CA000B3F90000B2F90020871A0D97B3F902006A
:107CB000B6F90230C21A1592B1F800A0CDF808A0AA
:107CC000B1F80680CDF80C80B1F802A0B1F804B08C
:107CD0004FF00007ADF8A070ADF8A270A868ADF83D
:107CE000A400EB68ADF8A6300846314628AA26ABBA
:107CF000FFF750FF002C50D0BDF89810DDF83490FD
:107D000009FA81F2BDF89A80DDF854C00CFA88F3C4
:107D1000B4F800C00FFA8CF0824209DA871ABFB2B9
:107D20007918ADF89810BDF89C10CF1BADF89C7079
:107D3000678839B28B420CDAC3EB01091FFA89F963
:107D4000C844ADF89A80BDF89E80C9EB0809ADF82B
:107D50009E90B4F8048000FA88F0BDF99C9091449C
:107D6000484504DAC444C2EB0C02ADF89C20E2881A
:107D700001FA82F1BDF99E00C018814203DAD219DE
:107D8000D31AADF89E30BDF99C10002940F333841E
:107D9000BDF99E00002840F32E84BDF89A703BB2D6
:107DA000BDF99E20D118994240F32584DDF8088062
:107DB0000FFA88F4DDF80CC00FFA8CF00FFA8AFA8B
:107DC0000FFA8BFB00FB04F20BFB1A2141F30F228D
:107DD0000B924FEA00201C90CBF100084FEA082CD0
:107DE000CDF87CC0CAF1000A4FEA0A2BCDF878B072
:107DF0004FEA04241D9448F28108C8F28008CDF8A7
:107E0000388046F24801C0F206011B910297AA464B
:107E10003546BDF898400FFA84FBBDF99C200BEB6A
:107E20000200834580F294831C9EDDF82C9096FB23
:107E3000F9F739B203911F9A92FBF9F006B2059651
:107E40001E9F97FBF9F10AB206921D9890FBF9F676
:107E500037B20797DDF8548043440C9357462A887D
:107E60006888A11A0BB2029EC6EB000C0FFA8CF1C7
:107E7000DDF814A001FB0AF9039E03FB069808F144
:107E8000800ADDF81C8008FB01FC069E06FB03C38C
:107E900003F1800312B20AEB022900B2C3EB002AFD
:107EA000C9F30F23CAF30F2219B2B1F1FF3FC0F299
:107EB000418310B2B0F1FF3FC0F23C8318B2B96801
:107EC000884280F237830FFA82F8CDF80480FE688A
:107ED0000496B04580F22E835FFA89F95FFA8AF63C
:107EE000C9F5807EC6F5807808FB0EFCCCF30F2A1E
:107EF000CDF820A00FFA89F909FB08F8C8F30F2C78
:107F0000CDF824C036B206FB0EFECEF30F2ACDF814
:107F100028A006FB09F94FEA19291FFA81FAD7F8B8
:107F200004C048F68808C44540F0AD8007F1180E3B
:107F30000FFA8AFC019E0CFB060C0EEB8C0813F466
:107F4000004F0BD112F4004F40F02D835EF82C60EF
:107F5000219600F1010088420BDB0EE04FF0000E8D
:107F6000CDF884E000F10100814206DD12F4004FFB
:107F700003D1D8F80460229602E04FF0000222926A
:107F800013F4004F0BD1019B03F10103049A9A42B1
:107F900005DD0FFA8AF358F82320239202E04FF010
:107FA0000006239681420DDD019800F1010004993D
:107FB000814207DD0FFA8AF303F1010358F8232009
:107FC000249202E04FF00006249608980FFA80FAF7
:107FD000DDF824C00FFA8CF0DDF828800FFA88F164
:107FE0000FFA89F39DF887609DF88B2000FB02F261
:107FF0000AFB06229DF88F6001FB06229DF8936024
:1080000003FB06224FEA22268DF897609DF88460D4
:108010009DF8882002FB00F206FB0A229DF88C6086
:1080200006FB01229DF8906006FB03224FEA222600
:108030008DF894609DF885609DF8892002FB00F220
:1080400006FB0A229DF88D6006FB01229DF89160D7
:1080500006FB03224FEA22268DF895609DF88620C4
:108060009DF88A6006FB00F002FB0A029DF88E0074
:1080700000FB01219DF8926006FB03134FEA2322C7
:108080008DF896207BE248F26556B44540F02A818F
:1080900007F1180C0FFA8AFEDDF804800EFB0806C3
:1080A00006EB460E0CEB0E0813F4004F1ED112F433
:1080B000004F40F05C821CF80E6006F01F0CCDF8FB
:1080C0004CC098F8012002F0070E4FEACE0C4CEAA3
:1080D000561ECDF850E04FEAD20298F802C0CDF813
:1080E00048C000F1010088420CDB62E200F10100AF
:1080F000814244DD12F4004F4FD14FF00002149240
:108100001392129298F803C00CF01F06189698F874
:1081100004E00EF007064FEAC60646EA5C1CCDF8FE
:1081200068C04FEADE0ECDF840E098F805C0CDF803
:1081300064C013F4004F3ED1019B03F10103049E80
:108140009E4241DD0FFA8AF303EB430608EB060378
:1081500018F806C00CF01F0ECDF858E093F801E0B7
:108160000EF007064FEAC60646EA5C1CCDF844C08E
:108170004FEADE0ECDF85CE093F802E02CE04FF021
:10818000000214921392129210921A92189219925B
:1081900096461792119216921EE04FF0000214922A
:1081A0001392129210921A9218921992964617925E
:1081B0001192169210E04FF0000ECDF85CE0CDF871
:1081C00044E0CDF858E007E04FF0000ECDF85CE059
:1081D000CDF844E0CDF858E081421FDD019901F16E
:1081E0000101049888421FDD0FFA8AF303F10103AD
:1081F00003EB430108EB010618F8013003F01F08F8
:10820000707800F0070A4FEACA0C4CEA531ACDF80E
:1082100004A04FEAD0010491B6780AE04FF00006BE
:1082200004960196B04604E04FF0000604960196CD
:10823000B046089B0FFA83FA099800B2DDF828C00F
:108240000FFA8CF10FFA89F3DDF8649000FB09F95D
:10825000DDF848C00AFB0C9901FB0E9E03FB06E605
:108260004FEA26268DF89760DDF860C00CFB00F61B
:10827000DDF84CE00EFB0A66DDF858C00CFB016629
:1082800008FB03664FEA26264FEAC6068DF894607F
:10829000DDF8688008FB00F6DDF850E00EFB0A66AA
:1082A000DDF844C00CFB0166DDF8048008FB0366C2
:1082B0004FEA26264FEA86068DF89560109E06FB4B
:1082C00000F002FB0A02DDF85CA00AFB0120DDF8E9
:1082D00010E00EFB03014FEA21234FEAC3068DF89D
:1082E00096604CE140F265518C4540F01F8107F1EA
:1082F00018010FFA8AFE019E0EFB060801EB480CDE
:1083000013F4004F0FD112F4004F40F05D8131F8AB
:108310001820ADF8842000F10100B96888421FDB05
:108320004FF0FF082AE09DF884106FF304018DF8E8
:108330008410BDF884606FF34A16ADF884604FEA8C
:1083400016216FF3C7018DF8851000F10100BE689A
:10835000B0420EDA12F4004F0ED14FF0000801E0E7
:108360004FF0FF08BCF80260ADF888604FF0FF0ED8
:1083700018E04FF0000801E04FF000089DF8886019
:108380006FF304068DF88860BDF888206FF34A12F9
:10839000ADF888204FEA12216FF3C7018DF88910DC
:1083A0004FF0000E13F4004F0FD1019A02F10102B9
:1083B000FB689A4209DA0FFA8AF13CF81160ADF8CD
:1083C0008C604FF0FF02049214E09DF88C106FF364
:1083D00004018DF88C10BDF88C606FF34A16ADF86F
:1083E0008C604FEA16226FF3C7028DF88D204FF094
:1083F00000030493BB68834210DD019800F1010083
:10840000F96888420ADA0FFA8AF000F101003CF8B4
:108410001010ADF890104FF0FF0213E09DF890603F
:108420006FF304068DF89060BDF890206FF34A1248
:10843000ADF890204FEA12236FF3C7038DF8913007
:108440004FF00002089E0FFA86FA099B18B2DDF879
:1084500028C00FFA8CF10FFA89F300FB0EF60AFB25
:108460000866DDF8108001FB086603FB02624FEA34
:1084700022268DF897609DF8842002F01F069DF853
:10848000882002F01F0202FB00F206FB0A269DF87C
:108490008C2002F01F0202FB01629DF8906006F042
:1084A0001F0606FB03224FEA22264FEAC6028DF87A
:1084B0009420BDF88460C6F34516BDF88820C2F349
:1084C000451202FB00F206FB0A26BDF88C20C2F31F
:1084D000451202FB0162BDF89060C6F3451606FB2B
:1084E00003224FEA22264FEA86028DF895209DF856
:1084F00085604FEAD6029DF889604FEAD60606FBF2
:1085000000F002FB0A029DF88D004FEAD00606FB40
:1085100001219DF891204FEAD20000FB03134FEA9E
:1085200023264FEAC6018DF8961028E01B9B1A6897
:10853000259224E004F10104A4B20FFA84FBBDF9F2
:108540009820BDF99C0011188B45FFF688ACBA46FF
:10855000029B03F101039AB2029213B2BDF99A0091
:10856000BDF99E1042189342FFF653AC43E000F170
:1085700001004FF0000214921392129219E09DF83C
:1085800097000F9901FB00F0DDF838E08EFB0086C4
:1085900033180D9E06EB0B000C99259AC3F3C713F5
:1085A000FAF734FCC6E74FF00002219200F1010017
:1085B000E3E44FF0000ECDF840E0CDF868E0CDF8F0
:1085C00060E0CDF864E0B7E59DF884206FF3040225
:1085D0008DF88420BDF884106FF34A11ADF8841033
:1085E0004FEA11266FF3C7068DF8856000F1010090
:1085F0004FF00008C2E62BB0BDE8F08F40F2A45364
:10860000C1F20003196846F20C10C0F2060082683D
:108610000A6040F2A053C1F200031A6846F2081142
:10862000C0F206010B68136040F29852C1F20002DA
:108630001168C068086040F29C53C1F200031968D9
:1086400046F20412C0F206021068086048F2000305
:10865000C2F2090319686FF3D751196048F21C0080
:10866000C2F209004FF080620260704708B54FF017
:108670001C014FF0000201F095F908BD08B5014654
:108680004FF000004FF01C0201F0FEF840F2A4533E
:10869000C1F200034CF26002C4F202021A6040F21E
:1086A0009850C1F200004CF26401C4F20201016072
:1086B00040F2A053C1F200034CF25C02C4F2020289
:1086C0001A6040F29C50C1F200004CF26801C4F202
:1086D00002010160FFF792FF08BD00BFF8B5044634
:1086E0000D4648F21403C2F20903186810F4000F93
:1086F00040F0D780002C00F0D780002900F0D78010
:1087000040F2A451C1F200010F6846F20412C0F217
:10871000060216683E6040F2A053C1F200031868DA
:10872000066040F29851C1F200010F6846F20C1247
:10873000C0F20602D3683B6040F29C50C1F20000D8
:1087400001680E6048F20007C2F209073A686FF349
:108750009A623A603B6843F400003860396841F03F
:1087600080723A6048F21807C2F209074FF080732E
:108770003B6048F21C00C2F209004FF400010160A6
:108780004FF019001BF0E8FF4FF0000222604FF09D
:10879000030000F0F1FB074620604FF0030000F0FB
:1087A000EBFBC71927604FF0030000F0E5FBC7198A
:1087B00027604FF0030000F0DFFBC31948BF03330D
:1087C0004FEAA307276040F2A454C1F200042068D6
:1087D00046F20C11C0F206018A68026040F2A05312
:1087E000C1F200031C68266040F29850C1F20000FC
:1087F00001680E6040F29C52C1F2000213681E60D4
:1088000048F20004C2F2090420686FF3D7502060D8
:10881000216841F000722260236843F0806020608C
:1088200048F21804C2F209044FF00071216048F2C6
:108830001C03C2F209034FF080621A604FF0190066
:108840001BF08AFF4FF0000028604FF0020000F09C
:1088500093FB044628604FF0020000F08DFB0419E2
:108860002C604FF0020000F087FB04192C604FF0E1
:10887000020000F081FB011948BF03314FEAA10457
:108880002C60FFF7BBFE4FF019001BF065FF48F2AC
:108890001403C2F209031A6882F40000C0F3C05046
:1088A000F8BD4FF00000F8BD4FF00100F8BD4FF0EB
:1088B0000100F8BDF8B540F20403C4F202031A68DF
:1088C00042F400211960044628B34FF47A751E461D
:1088D00000F1FF3000F0010728461EF01DF9336853
:1088E00003F00812082A19D11BE028461EF014F9DB
:1088F000336803F00812082A10D104F1FF34284627
:108900001EF00AF9316801F00810082806D117E0B6
:108910004FF00100F8BD4FF00100F8BD4FF000002E
:10892000F8BD013CF4D0002FDFD028461EF0F4F84B
:10893000316801F008100828F0D1013CD5D1E7E7F3
:10894000013CD2D1E4E700BF684620F007018D4624
:1089500019B548F2B803C2F209034FF002021A60D7
:108960004FF47A742046FFF7A5FF0028FAD003F0F1
:108970003DF9BDE819408546704700BF10B54CF27F
:10898000C803C4F20F031A6842F00800186046F2E8
:108990001C11C0F206010C6840F20003C4F202038D
:1089A0001C604FF064001EF0B7F846F22012C0F2CF
:1089B0000602106840F20401C4F2020108604CF2A1
:1089C00050301EF0A9F84FF03200FFF773FF88B95E
:1089D00000F0CCFC48F2B804C2F209044FF00203E4
:1089E00023604FF4FA742046FFF764FF0028FAD0A2
:1089F00003F0FCF84FF0170003F06EFA48F6491444
:108A0000C0F2020420464FF00F014FF0170203F0AE
:108A100017FA40F20400C4F20200026842F4002196
:108A200001604FF0290003F057FA20464FF00F0184
:108A30004FF0290203F004FA10BD00BF41B940F223
:108A4000B453C1F20003186810604FF00000704783
:108A50004FF01400704700BF40F2B453C1F200035E
:108A600018686FEA0000704708B54FF001001870F1
:108A700051B940F2B453C1F200031A60114600F03C
:108A8000BFF94FF0000008BD4FF000021A704FF020
:108A9000140008BD10B540F2B454C1F200044FF008
:108AA000200021464FF0080200F0EEFEFFF7D4FF51
:108AB0006368834205D14FF00100216800F0A0F9FE
:108AC0000EE04FF001004FF07C5100F099F940F2B8
:108AD000B450C1F200004FF00002CBF68072026089
:108AE0004FF00B0046F22411C0F2060140F2A852EA
:108AF000C1F200021FF0C4FD10BD00BF08B54FF069
:108B00000103137081B9FFF7A7FF40F2B451C1F21E
:108B10000001486008464FF008014FF0200200F0C5
:108B200041FF4FF0000008BD4FF0000010704FF003
:108B3000140008BD02469CF8043043B1DCF8000084
:108B400040B140F2E451C1F2000141F82200DCF8EA
:108B5000000050B940F2E453C1F2000353F8220080
:108B600049F64042002808BF104670474FF4606342
:108B7000C0F22773B3FBF1F110B1012819D10CE059
:108B800044F21802C4F20102116044F20C00C4F273
:108B900001004FF000030360704748F21800C4F270
:108BA0000100016048F20C03C4F201034FF0000120
:108BB0001960704710B582B000918DF80420032829
:108BC00014D1EC464FF00000FFF7B4FF01464FF020
:108BD0000000FFF7CBFFEC464FF00100FFF7AAFFC4
:108BE00001464FF00100FFF7C1FF0CE046F2F01321
:108BF000C0F206031C5CEC462046FFF79BFF0146D3
:108C00002046FFF7B3FF02B010BD00BF10B446F21C
:108C10009413C0F2060300EB80004FEA80001A189C
:108C2000148A1B5C012B1CD169B18C420ED944F211
:108C30001800C4F20100006804F1FF3300FB0131A9
:108C4000B1FBF4F404E04FF0000401E04FF6FF74D0
:108C50005068046093681968D26841EA020018609D
:108C600026E0022B24D103F57F70844218D849B145
:108C70008C420AD9C1EB812104F1FF304318B3FBC8
:108C8000F4F404E04FF0000401E040F2FF344CF251
:108C90000001C4F208010A6864F38F120A6007E059
:108CA0004CF20003C4F208031A6861F38F121A60D1
:108CB00010BC704708B54FF000000146FFF7A6FF53
:108CC0004FF001004FF00001FFF7A0FF4FF002004E
:108CD0004FF00001FFF79AFF4FF0030343F4807158
:108CE0004CF23002C4F2020211604CF23403C4F2BE
:108CF000020319604FF0010141F480704CF26002F0
:108D0000C4F2020210604CF26401C4F20201086075
:108D100046F2EC10C0F2060003684CF28802C4F27E
:108D2000020213604CF28C01C4F202010B604CF29F
:108D30009400C4F20200036008BD00BF10B54CF2FD
:108D4000C404C4F20F04236843F0200020602168AB
:108D500041F040022260FFF7ADFF4FF003004FF0FB
:108D600000010A46FFF726FF44F21403C4F2010390
:108D7000186840F00201196048F21403C4F20103BC
:108D80001A6842F00200186046F2F411C0F20601BF
:108D90000A6844F24C03C4F201031A6048F24C0022
:108DA000C4F201004FF00001016046F2E412C0F28B
:108DB0000602136844F20400C4F20100036048F2A2
:108DC0000401C4F201010B60226842F48053236065
:108DD00046F2E810C0F20600016844F20002C4F254
:108DE0000302116040F2BC50C1F2000046F2FC11D7
:108DF000C0F2060117F04AF910BD00BF00000000E4
:108E000070B52DED028B08EE101A44F21803C4F26F
:108E10000103196846F29413C0F2060300EB8000C8
:108E20004FEA80029E189B5C012B5FD108462BF015
:108E300055FE02460B464FF000004FF00001C3F60E
:108E4000F0712CF0F1FA4FF000024FF00003C3F67E
:108E5000E0732CF033FA2CF02FF808EE900AF4EEC1
:108E6000C88AF1EE10FA33DC18EE100A2CF008F87C
:108E700004460D4618EE900A2CF002F802460B4606
:108E80004FF000004FF00001C3F6F0712CF0D0F865
:108E900002460B46204629462CF038FCD8B944F24D
:108EA0001800C4F20100D0ED000AB8EE601A61EEBD
:108EB000081A11EE900A2BF0E3FF4FF000024FF07A
:108EC0000003C3F6E0732CF0B5F82BF09FFF04E02D
:108ED0004FF0000001E04FF6FF7073681860B06853
:108EE0000168F26841EA0203036035E0022B33D1E6
:108EF00018EE100A2BF0C4FF04460D4619A3D3E95F
:108F000000232CF01FFCD0B92046294617A3D3E933
:108F100000232CF0FBFBA8B9DFED117A28EE270A1D
:108F200010EE100A2BF0ACFF4FF000024FF00003E0
:108F3000C3F6E0732CF07EF82BF068FF04E04FF0EE
:108F4000000001E040F2FF304CF20001C4F20801E1
:108F50000A6860F38F120A60BDEC028B70BD00BF1F
:108F600000C07F449A9999999999A93F6666666667
:108F70006666EE3FAFF3008010B50446032839D88B
:108F800040F2BC50C1F200004FF0000117F096F81B
:108F900044F20001C4F203010B6846F25812C0F219
:108FA000060204EB44004FEA80041019125944F2FF
:108FB0000404C4F2030424681468406860F30703DF
:108FC0004FF0010464F31A630B601168002907DB9A
:108FD00044F20000C4F2030003681368002BFBDABC
:108FE0001268C2F30B1440F2BC50C1F2000017F03B
:108FF00075F901E04FF0FF34204610BD10B504466E
:10900000FFF7BAFF04EB440146F25813C0F206031F
:1090100003EB8104228902FB00F040F20111C0F24F
:109020001001A1FB0023C01A03EB5002C2F3CF20B2
:1090300010BD00BF08B5FFF79FFF07EE900AB8EE1E
:10904000677A9FED030AC7EE000A10EE900A08BD8A
:1090500000F07F450000000008B546F29413C0F20E
:10906000060300EB80004FEA80015A185B5C012B7D
:109070000FD1526892ED007A44F21803C4F2010352
:1090800093ED000AF8EE470AB8EE401AC0EE817A76
:1090900016E0022B12D14CF20000C4F20800016865
:1090A000C1F389102BF0FAFC08A3D3E900232CF0BC
:1090B000BBF92BF001FF07EE900A01E0DFED027A29
:1090C00017EE900A08BD00BF00000000000000007D
:1090D00000F88F40AFF300804FF0000303604FF0C3
:1090E00000007047F8B572B642F210701DF014FD22
:1090F00046F20C23C0F206031A684EF63470CEF224
:109100000000026046F21421C0F206010C684EF61F
:109110008855CEF200052C604CF2A016C4F20F0662
:10912000377847F0200333703246106810F0400F54
:10913000FBD04CF20004C4F20F0425684FF0050187
:1091400061F30F35256046F20826C0F2060637683F
:109150004CF20411C4F20F010F6046F20023C0F27A
:10916000060318684CF20812C4F20F02106046F2AF
:109170001824C0F2060425684CF28006C4F20F06DB
:1091800035604CF28C03C4F20F034FF0AA041C604C
:109190004FF0550018604CF20C15C4F20F052F6803
:1091A00047F001072F6046F21025C0F206052F6830
:1091B0004CF28405C4F20F052F6046F20425C0F27C
:1091C00006052D6835601C60186046F21C26C0F24A
:1091D000060636684CF2A403C4F20F031E604CF27C
:1091E000A003C4F20F031D604CF2AC03C4F20F03E2
:1091F0001C60186008684FF0010363F30400086006
:1092000011684FF0020060F3040111604CF2A812E3
:10921000C4F20F0213604CF28801C4F20F010B6814
:1092200013F4806FFBD04CF2A800C4F20F00026868
:1092300012F4806FFBD04CF20411C4F20F010B68E2
:1092400043F4807008604CF20813C4F20F031A68EC
:109250004FF0020161F309221A604CF20000C4F2DF
:109260000F0003684FF0040262F30F330360F8BD90
:10927000F0B49DF810609DF814504FF00004032ADC
:1092800011D1069A62F3020446F2B832C0F2060225
:10929000925D62F3C40444F02004003518BF012538
:1092A00065F3492416E06FF3020446F2B837C0F2C2
:1092B0000607BE5D66F3C40444F02004003518BF01
:1092C000012565F34924022A04D16FF3C71444F43D
:1092D000803401E044F08004012B14BF00230123FB
:1092E00063F38A2446F22823C0F2060353F82000D1
:1092F00040F82140F0BC704746F25C23C0F2060300
:1093000053F820100A6846F2BC23C0F2060353F853
:1093100020100A4046F2C433C0F2060353F820007E
:10932000824214BF00200120704700BF46F2A423F0
:10933000C0F2060353F820004069704746F2BC2390
:10934000C0F2060353F8203039B146F27431C0F24E
:10935000060151F820201360704746F21C32C0F21B
:10936000060252F820000360704700BF70B546F255
:10937000A023C0F2060319684CF20010C4F20200E8
:10938000C16246F21432C0F2060214684CF20025A3
:10939000C4F202052C6546F2C036C0F206063368F8
:1093A000EB6446F24021C0F206010A686A6546F2A3
:1093B0005424C0F2060426684CF20003C4F20203EF
:1093C0005E6546F21031C0F206010A68AA6646F2EE
:1093D000BC34C0F206042668DE6446F25021C0F2B6
:1093E00006010A684CF28006C4F20206B26446F234
:1093F0000434C0F206042168296446F27032C0F2D7
:1094000006021468746046F22421C0F206010A685C
:109410009A6446F24824C0F206042168A96546F21F
:109420001832C0F206021468EC6546F26431C0F2EC
:1094300006010A685A6446F20C44C0F20604216828
:10944000716346F24422C0F206021468EC6646F2EA
:109450000C35C0F206052968F16146F26832C0F2A7
:1094600006021468446046F24C20C0F2060005680B
:109470004CF28021C4F202014D6046F20032C0F28B
:1094800006021468DC6546F26C30C0F2060005681E
:109490009D6646F20831C0F206010A681A6646F275
:1094A0005824C0F206042068586646F22025C0F20F
:1094B00006052968716446F26036C0F20606326815
:1094C0001A6546F20844C0F20604206898654FF019
:1094D00000000146FFF732FF48F20004C2F209041F
:1094E000236843F4802525604FF001004FF0000110
:1094F000FFF724FF48F28006C2F20906316841F402
:10950000800232604FF002004FF00001FFF716FFBB
:10951000306840F4000333604FF003004FF0000167
:10952000FFF70CFF256845F4003121604FF004007F
:109530004FF00001FFF702FF48F22005C2F20905D3
:109540002A6842F4005028604FF005004FF00001F7
:10955000FFF7F4FE336843F0006131604FF006001E
:109560004FF00001FFF7EAFE2A6842F08000286011
:109570004FF007004FF00001FFF7E0FE48F2400314
:10958000C2F20903196841F002021A604FF00800A4
:109590004FF00001FFF7D2FE48F2A000C2F209002E
:1095A000036843F0020101604FF009004FF0000131
:1095B000FFF7C4FE226842F4000020604FF00A006A
:1095C0004FF00001FFF7BAFE236843F0806121608D
:1095D0004FF00B004FF00001FFF7B0FE226842F0A1
:1095E000807020604FF00C004FF00001FFF7A6FEE6
:1095F000236843F0007121604FF00D004FF000012F
:10960000FFF79CFE2A6842F4003028604FF00E00FD
:109610004FF00001FFF792FE236843F480112160B0
:109620004FF00F004FF00001FFF788FE226842F470
:10963000800020604FF0010015F0C6FA70BD00BF39
:1096400008B5FFF793FE08BD46F2BC23C0F206033F
:1096500053F8203046F25C22C0F2060252F8201085
:109660000968194046F2C432C0F2060252F82020BE
:10967000914207BF46F21C32C0F2060246F2743233
:10968000C0F2060252F820000360704708B54CF2A1
:10969000C403C4F20F031A6842F00050186046F287
:1096A0001441C0F206010A6840F23003C2F2080316
:1096B0001A6040F2EC50C1F2000046F22841C0F2BC
:1096C000060116F0E3FC08BD2DE9F843074688467D
:1096D0001646002A52D040F2EC50C1F200004FF082
:1096E000000116F0EBFC40F22813C2F208034FF021
:1096F00000021A6046F23040C0F20600016840F2F3
:109700002C14C2F20804216046F21045C0F206058E
:10971000D5F8009046F23443C0F206031D6840F6C7
:10972000FF7C40F2201EC2F2080E40F22410C2F26A
:10973000080040F22C11C2F2080140F23014C2F2CB
:109740000804664534BF33466346CEF800800760A0
:109750000A6863F30B020A60C4F80090F61A4FEA35
:1097600083039844FF1822681542FCD1002EE8D1EB
:1097700040F2EC50C1F2000016F0B0FDBDE8F883F5
:10978000F0B41746002A41D046F21C42C0F206024D
:10979000166840F21015C2F208052C682642FCD16A
:1097A00040F20012C2F20802116040F20411C2F24B
:1097B0000801086040F20810C2F208004FF00002F1
:1097C000026046F22441C0F20601086840F20C1221
:1097D000C2F208021060116867F30B01116046F2D3
:1097E0002040C0F20600016840F21012C2F20802E6
:1097F00011605BB146F21843C0F20603186840F2EC
:109800001011C2F208010A681042FCD1F0BC704786
:109810004FF000034FF0020262F307034FF007001E
:1098200060F30F234FF0050161F3174340F29002FC
:10983000C0F22002136040F29403C0F220034FF400
:10984000A0701860704700BF03685868C0F57C605E
:10985000704700BFF0B405686C688768C66806FB8F
:1098600007454768ED1969181960B1F57C6F07D293
:10987000521804F57C64A2428CBF0020012001E054
:109880004FF00000F0BC70472DE9F04F91B0074653
:109890000D469046002A6BD040F2840BC0F2200B9C
:1098A00040F2800AC0F2200A46F23C43C0F20603AE
:1098B000D3F8009040F28C04C0F2200407F03F017E
:1098C000781AC1F14006464528BF4646CBF800004D
:1098D000CAF80090402E26D0226800922368019397
:1098E0002068029022680392236804932068059000
:1098F00022680692236807932068089022680992DC
:1099000023680A9320680B9022680C9223680D93B9
:1099100020680E9022680F92284600AB59183246F4
:1099200034F0CAFE1FE022682A6023686B60216859
:10993000A9602068E86022682A6123686B61216859
:10994000A9612068E86122682A6223686B62216845
:10995000A9622068E86222682A6323686B63216831
:10996000A9632068E863BF19AD19B8EB0608A5D153
:1099700011B0BDE8F08F00BF30B583B015461C466E
:109980001A4601ABFFF766FF38B101982946224617
:10999000FFF77AFF4FF0000001E04FF01F0003B027
:1099A00030BD00BF2DE9F04F93B0804616460D46FE
:1099B00000297AD040F2840AC0F2200A46F2404BD5
:1099C000C0F2060B40F28003C0F22003019306F0C0
:1099D0003F07C7EB0609C7F14004AC4228BF2C463D
:1099E000402C05D0484602A94FF04002FFF74CFF3B
:1099F00002AAD71938464146224632F0C3F8C0B20F
:109A000000284ED038464146224634F055FECAF86A
:109A10000090DBF80010019B196040F28800C0F252
:109A20002000029A026003990160049B0360059A7A
:109A3000026006990160079B0360089A0260099919
:109A400001600A9B03600B9A02600C9901600D9BF8
:109A500003600E9A02600F990160109B0360119AD7
:109A6000026040F6E870C0F220004FF0FF31016064
:109A70004FF032001DF050F8CAF8009046F238431B
:109A8000C0F206031868019A10604FF032001DF012
:109A900043F840F6E071C0F220010B6813F0805FDC
:109AA000FBD03619A0442D1B91D113B0BDE8F08F27
:109AB00030B583B015461C461A4601ABFFF7CAFE07
:109AC00038B128462146019AFFF76CFF4FF000009D
:109AD00001E04FF01F0003B030BD00BF08B50346E2
:109AE0000A4640F21460C1F2000046F24441C0F25E
:109AF00006011EF08BFE08BD10B540F22464C1F2D1
:109B000000044FF03A03236041F6F172C1F6FF7290
:109B1000204621469047206848B940F23860C1F29B
:109B2000000004F104014FF0100234F0C5FD10BD37
:109B300008B572B646F2DC43C0F206031A684CF26E
:109B40000410C4F20F00026046F2D841C0F20601D0
:109B50000A684CF20813C4F20F031A6046F2504030
:109B6000C0F2060001684CF28002C4F20F021160DC
:109B70004CF28C03C4F20F034FF0AA0018604FF0B0
:109B8000550119604CF20C13C4F20F031A686FF3FD
:109B900000021A604CF2A010C4F20F00017821F00C
:109BA0002003037040F22461C1F200014FF039023A
:109BB0000A6041F6F173C1F6FF730846984708BD85
:109BC00070B572B640F28003C0F220034FF000027D
:109BD0001A6046F25444C0F20604256840F6E8765E
:109BE000C0F22006356046F25843C0F206034FEA41
:109BF00010301E5C4FEA11315D5C40F22464C1F20A
:109C000000044FF0320222606660A56041F6F173F5
:109C1000C1F6FF73204621469847206880B9214647
:109C20004FF0340222606660A5604DF2C043C0F27E
:109C30000103E36041F6F172C1F6FF7220469047DE
:109C400062B640F22461C1F200010868002814BF26
:109C50000220002070BD00BFF8B507460D4616462D
:109C600072B646F25843C0F206034FEA1132985CCE
:109C700089194FEA11341B5D40F22464C1F20004DB
:109C80004FF0320222606060A36041F6F173C1F6CA
:109C9000FF73204621469847206888B921464FF037
:109CA000330222606560A760E6604DF2C043C0F2F7
:109CB0000103236141F6F172C1F6FF72204690471D
:109CC00040F22461C1F200010878002814BF02208C
:109CD000002062B6F8BD00BF08B540F23861C1F29D
:109CE00000014FF0100234F0E7FC4FF0100008BD07
:109CF00008B547F6E430C1F2000047F6E472C1F25D
:109D00000002131A4FF0FF314FEAA30201F0DCFF0B
:109D100015F024FD02F0AEFB4FF0000008BD00BFBF
:109D2000BFF36F8F704700BF032826D8DFE800F02D
:109D3000020B141D4CF2C400C4F20F00026842F082
:109D40000201016070474CF2C400C4F20F000168C8
:109D500041F00403036070474CF2C401C4F20F01E8
:109D60000B6843F480020A6070474CF2C403C4F2EB
:109D70000F031A6842F400001860704711B10129FE
:109D80002CD116E040F25863C1F200031968022991
:109D900009D040F25860C1F200000368042B14BFE0
:109DA0000023012301E04FF0010313704FF0000086
:109DB000704740F25861C1F200010B68012B07D1D6
:109DC00040F26460C1F2000003684FF00001996046
:109DD0004FF0010010704FF0000070474FF000008E
:109DE00010704FF014007047684620F007018D4650
:109DF00001B446F2E043C0F20603186840F2501284
:109E0000C2F2080211680842FCD140F25C63C1F260
:109E1000000318680268026040F24C13C2F20803A3
:109E200018684FF0010161F30B00186040F2501305
:109E3000C2F208031A680A431A6040F24862C1F28B
:109E40000002106840F25463C1F200031968401A1E
:109E500040F24C61C1F20001086012681A6040F2E1
:109E60005863C1F200034FF00200186001BC854640
:109E7000704700BF684620F007018D4601B440F2EC
:109E80006463C1F2000318680268026040F2606116
:109E9000C1F200010B681A690AB1006B00E0C06AE8
:109EA00040F25861C1F200010B683BB940F25862C0
:109EB000C1F200024FF00303136011E040F254625C
:109EC000C1F200021168431A40F24C62C1F2000272
:109ED000136040F25863C1F200034FF004011960AF
:109EE00040F25461C1F20001086001BC8546704730
:109EF00010B540F25863C1F200031968022904D07A
:109F0000042916D0012947D12BE040F25863C1F251
:109F100000034FF0000440F24C60C1F200001C60EE
:109F200001681A68002AFAD102EE101AB8EE420A45
:109F300010BD40F25863C1F200034FF0030440F239
:109F40004C60C1F200001C6001681A68032AFAD153
:109F500000EE901AB8EE601ADFED111A81EE210AB8
:109F600010BD78B140F26463C1F2000319684FF08C
:109F7000000001F1080101F049FE07EE900AB8EE79
:109F8000670A10BD40F26460C1F20000026892ED01
:109F9000020AB8EE400A10BD9FED020A10BD00BFD4
:109FA000C0E1E44C0000000010B5144611B10129D5
:109FB00012D108E04FF00000FFF79AFF84ED000A8D
:109FC0004FF0000010BD4FF00100FFF791FF84ED4E
:109FD000000A4FF0000010BD4FF0140010BD00BF8C
:109FE00070B584B040F26463C1F200031A6846F2AF
:109FF0006051C0F206010D68556040F25C63C1F229
:10A0000000031A6855600546002800F03F8140F2C1
:10A010006060C1F200000368187999684FF000048D
:10A0200000940194DA6802924FF003022346FFF78E
:10A030001FF940F25861C1F200010C6040F2546017
:10A04000C1F200000460042D23D140F26461C1F22A
:10A050000001086823464FF0020262F3010340F258
:10A060006061C1F200010A68116961F3830303674B
:10A0700044618462C46046F2F442C0F20602116890
:10A08000416040F25860C1F200004FF001030360EC
:10A09000FCE0052D3DD140F26465C1F200052C685D
:10A0A00040F26065C1F200052868036849F67560F2
:10A0B000C0F202004FF00F0146F2F042C0F2060279
:10A0C000D25601F0BDFE46F2E441C0F20601086836
:10A0D00020674FF0000363612A68116911B10129FB
:10A0E0000DD106E046F24452C0F206021168A162A8
:10A0F00005E046F24850C0F206000368A3624FF044
:10A100000000E06046F2F843C0F206031A6862609D
:10A11000BCE040F26464C1F20004236840F25C6673
:10A12000C1F2000634684FF000024FF0020161F303
:10A13000010240F26060C1F200000668316961F31B
:10A1400083021A674FF000025A619A62DA601A615C
:10A1500046F2E840C0F2060006685E6040F2501128
:10A16000C2F208010A6040F24810C2F20800026020
:10A1700046F25C52C0F20602116840F24C10C2F284
:10A180000800016003F1080340F24012C2F2080225
:10A19000136040F24413C2F2080340F24861C1F276
:10A1A0000001196046F24050C0F20600026840F219
:10A1B0005063C1F200031B68032B2FD8DFE803F0C4
:10A1C000020D18234CF2C411C4F20F01086840F0CC
:10A1D000010008604FF0000122E04CF2C411C4F20B
:10A1E0000F01086840F0040008604FF0020117E01A
:10A1F0004CF2C411C4F20F01086840F0100008606E
:10A200004FF004010CE04CF2C411C4F20F010868D5
:10A2100040F4804008604FF00E0101E04FF0000173
:10A2200061F3450240F25010C2F20800026049F6A4
:10A23000E950C0F202004FF0000146F2F042C0F2D5
:10A240000602D25601F0FCFD46F28C53C0F2060322
:10A250001968216746F2EC40C0F2060002686261AC
:10A260004FF00003A36246F24C51C0F2060101EB2D
:10A27000850595ED007ADFED067A27EE270AFCEEDC
:10A28000C00AC4ED060AE3602361666004B070BDD5
:10A29000C0E1E44C10B54FF000041C7049B9052A28
:10A2A0000AD84FF0010119701046FFF799FE2046B9
:10A2B00010BD4FF0140010BD4FF0160010BD00BFD0
:10A2C00008B54FF00000FFF78BFE08BD38B5044617
:10A2D0000D4640F26061C1F2000146F26450C0F2E6
:10A2E00006000860012D03D1012A01D1122B01D0F3
:10A2F00001F088FC40F25063C1F200031C6046F29A
:10A300003050C0F2060050F8252040F26461C1F2DE
:10A3100000010A6050F8240040F25C63C1F20003BF
:10A3200018602846FFF700FD2046FFF7FDFC4CF2C1
:10A33000020046F2FC41C0F2060140F26862C1F23E
:10A3400000021EF09DF938BD4CF28013C4F20F03D9
:10A35000186840F27462C1F200024FF000011170FF
:10A36000C3B203F00400C2B23AB140F27461C1F268
:10A3700000014FF020020A702DE003F01001C8B276
:10A3800038B140F27463C1F200034FF0010018705D
:10A3900021E013F0010F07D040F27461C1F2000117
:10A3A0004FF080020A7016E003F00202D1B239B118
:10A3B00040F27463C1F200034FF0400018700AE0ED
:10A3C00003F00803D8B230B140F27461C1F2000169
:10A3D0004FF002020A704CF28013C4F20F034FF0E8
:10A3E000FF30186047F6D831C1F200010A6840F228
:10A3F0007863C1F200031A60704700BF40F27463D3
:10A40000C1F200031878704730B444F21402C4F269
:10A41000020244F21805C4F2020513682C681168A0
:10A420008B42FAD129688C42F7D103F03F020260D7
:10A43000C3F305214160C3F304428260C3F30263A6
:10A44000836104F01F01C160C4F3032202F1FF33F2
:10A450000361C4F30B44A4F26C74446130BC7047D4
:10A4600000B58BB0014601A84FF0240234F024F966
:10A4700001A833F02BFA44F20803C4F202031A785D
:10A4800022F001001870197841F002021A7044F2AB
:10A490002000C4F202000199016044F22400C4F2D9
:10A4A0000200029A026044F22801C4F202010398F9
:10A4B000086044F23001C4F20201079A0A6044F2D3
:10A4C0002C00C4F2020004990160059A02F1010215
:10A4D00044F23800C4F202000260069901F26C7284
:10A4E00044F23C00C4F202000260197841F001021B
:10A4F0001A70187820F0020119700BB000BD00BF6F
:10A5000010B582B04CF2C403C4F20F031A6842F4CF
:10A510000070186044F20801C4F202010B6813F0E5
:10A52000010F00F0888044F20802C4F202021068B1
:10A5300010F0020F7FD144F20C01C4F202010A684C
:10A5400046F2B853C0F206031868824273D144F24F
:10A550001001C4F202010A68002A6CD144F23C03E3
:10A56000C4F20203186840F2D971884251D862E0FF
:10A5700001996FEA0104A0420FD146F2C052C0F225
:10A580000602136844F20801C4F202010B6044F2AF
:10A590004004C4F20204206010E046F2C452C0F24B
:10A5A0000602106844F20803C4F20203186044F281
:10A5B0004001C4F202014FF000040C604FF00004AF
:10A5C00044F20C00C4F20200046044F21002C4F22F
:10A5D0000202146046F29450C0F20600FFF740FFFA
:10A5E00044F24403C4F202031C6044F24801C4F282
:10A5F00002010C6044F24C00C4F20200046044F218
:10A600005002C4F20202146044F25403C4F2020382
:10A610001C6044F20001C4F202014FF0FF300860F8
:10A6200046F2B852C0F20602116844F20C03C4F2BA
:10A630000203196014E046F2BC54C0F2060422681A
:10A6400044F20803C4F202031A60F9F7DFFD694619
:10A650004FF00802FFF718F90098002888D19CE70E
:10A6600002B010BD4FF0000361F3100360F35143DB
:10A6700044F24002C4F20202136046F29050C0F26B
:10A680000600016844F20803C4F20203196070472F
:10A6900000B583B04FF00003009360F341038DF8E1
:10A6A0000230009861F3100000906FEA0001019100
:10A6B000F9F7ACFD024668464FF00801FFF772F962
:10A6C0004FF0010003B000BD46F2C853C0F20603CC
:10A6D000195C46F2AC62C0F206024FF02C0000FB9F
:10A6E0000123996846F29C62C0F206021068086075
:10A6F000704700BFF8B546F2AC67C0F2060746F2F5
:10A70000C854C0F20604255C4FF02C0606FB05FE7B
:10A7100007EB0E0547F2E004C0F27204B4FBF1F15E
:10A720004FF08004EE68346057F80E608FB23760E7
:10A730006E68C1F307213160E9694FF0F0060E60E1
:10A740006FF3C714A3F1050363F301049DF81830F8
:10A7500013F1FF3118BF012161F38204131C18BFEC
:10A76000012363F3C30446F2D051C0F206018A5CB0
:10A7700062F30514EB681C60FFF7A6FFF8BD00BF8D
:10A7800038B546F2C853C0F206031B5C03EB8304E2
:10A7900040F27C62C1F2000202EBC40282F8211096
:10A7A00014693CB140F27C65C1F200051346D269E0
:10A7B0009B69A04738BD00BFF8B506460F4646F274
:10A7C000C853C0F206031D5C05EB850040F27C64B3
:10A7D000C1F2000404EBC004D4F810C0BCF1000FB7
:10A7E00007D0E2698A4204D030464FF00001A369E5
:10A7F000E047E76163695BB105EB850040F27C628D
:10A80000C1F2000202EBC002304639469269984715
:10A8100094F8201079B127696FB105EB850540F2F6
:10A820007C63C1F2000303EBC505304694F82110A8
:10A83000E269AB69B847F8BD38B5054640F27C62BD
:10A84000C1F2000200EB80034FEAC30014184FF07E
:10A85000000184F8221013584BB146F29462C0F202
:10A860000602505DA169984794F8220040B96368D8
:10A8700033B146F29461C0F20601485DA169984780
:10A8800038BD00BF2DE9F8430446074646F2AC65E3
:10A89000C0F206054FF02C0303FB0055A8680268C0
:10A8A00012F0010F42D104EB840140F27C68C1F246
:10A8B000000808EBC1082E693168C2F3420646F26F
:10A8C0009469C0F20609CBB2C3F3800203F008001A
:10A8D000C1B211B142F00202D2B203F00203D8B207
:10A8E00008B142F0040206F1FF33052B1ED8DFE861
:10A8F00003F01A03031D1D03D8F808C0BCF1000FB4
:10A9000008D02868036819F80700D9B2D8F81830B9
:10A91000E04701E029680B682A69116811F0010F0E
:10A92000D1D1BDE8F8832046FFF786FFBDE8F88364
:10A93000684620F007018D4601B54FF00400FFF78F
:10A94000A1FFBDE801408546704700BF684620F082
:10A9500007018D4601B54FF00300FFF793FFBDE8F7
:10A9600001408546704700BF684620F007018D46CC
:10A9700001B54FF00200FFF785FFBDE801408546B5
:10A98000704700BF684620F007018D4601B54FF0C3
:10A990000100FFF777FFBDE801408546704700BF23
:10A9A000684620F007018D4601B54FF00000FFF723
:10A9B00069FFBDE801408546704700BF10B582B011
:10A9C0008DF8071046F2C853C0F20603185C46F231
:10A9D000AC61C0F206014FF02C0202FB00142169A9
:10A9E0000B6813F0200FFBD0246802A911F8012D89
:10A9F000226000EB800040F27C63C1F2000303EBB5
:10AA0000C004A08C4FF001021CF09EF8A08404F159
:10AA1000200402B010BD00BF30B583B08DF8071020
:10AA200046F2C853C0F206031B5C46F2AC61C0F2AA
:10AA300006014FF02C0202FB03F2881803EB83059A
:10AA400040F27C64C1F2000404EBC5044FF0010540
:10AA500084F822500069046814F0200F1DBF8A5842
:10AA60009DF807101160002503EB830340F27C6121
:10AA7000C1F2000101EBC304A08C0DF107014FF0FE
:10AA800001021CF061F8A08404F12004284603B000
:10AA900030BD00BF38B5054601F062F9044646F204
:10AAA000C853C0F20603585DFFF7C6FE204601F00A
:10AAB00061F938BD2DE9F041064646F2C853C0F2AF
:10AAC00006031C5C04EB840040F27C65C1F20005C7
:10AAD00005EBC00501F044F9804695F820100029E7
:10AAE00000F08F8046F2AC67C0F206074FF02C02F0
:10AAF00002FB0474236A4FF000071F606068076060
:10AB00003846394694F9242001F09AF9216A0A68F6
:10AB100067F3C7120A6030463946FFF731FE06F187
:10AB2000FF33042B63D8DFE803F0031B33624B00D1
:10AB30004CF2C403C4F20F0318686FF3C30018602B
:10AB400046F29862C0F2060211684CF20803C4F2A1
:10AB5000020319604CF20C00C4F20200016046E0EE
:10AB60004CF2C400C4F20F0001686FF35961016038
:10AB700046F29863C0F2060318684CF20002C4F271
:10AB8000020210604CF20401C4F2020108602EE0DF
:10AB90004CF2C403C4F20F031A686FF304121A6074
:10ABA00046F29860C0F2060001684CF23C03C4F221
:10ABB000020319604CF24002C4F20202116016E076
:10ABC0004CF2C400C4F20F0001686FF31861016019
:10ABD00046F29862C0F2060213684CF22800C4F2F2
:10ABE000020003604CF22C01C4F202010B60EB681E
:10ABF0001BB13046E969AA6998474FF0000285F811
:10AC00002020404601F0B6F8BDE8F0812DE9F0477C
:10AC100082B006468A469146984646F2C853C0F22C
:10AC20000603185C00EB800140F27C64C1F2000472
:10AC300004EBC10446F2AC65C0F206054FF02C02ED
:10AC400002FB005501F08CF8074606F1FF33042B98
:10AC500068D8DFE803F0031B33674B004CF2C400F5
:10AC6000C4F20F00036843F00801016046F29072DD
:10AC7000C0F2060210684CF20803C4F20203186026
:10AC80004CF20C01C4F2020108604BE04CF2C40328
:10AC9000C4F20F03196841F000721A6046F2A06016
:10ACA000C0F2060003684CF20001C4F202010B601E
:10ACB0004CF20402C4F20202136033E04CF2C4010D
:10ACC000C4F20F010A6842F01000086046F2907367
:10ACD000C0F2060319684CF23C02C4F20202116091
:10ACE0004CF24000C4F2020001601BE04CF2C400D0
:10ACF000C4F20F00016841F08072026046F2A46362
:10AD0000C0F2060318684CF22801C4F20201086080
:10AD100046F29072C0F2060210684CF22C03C4F2A4
:10AD2000020318609DF8282000929DF82C000190E5
:10AD3000304651464A464346FFF7DCFC2B6A196809
:10AD400041F080021A600C9820600E9BA3600D9960
:10AD500061600F9AE2601098A061A86A4FF00F013D
:10AD600095F9242001F06CF86B6846F2A861C0F2F6
:10AD700006010A681A604FF0010084F82000384686
:10AD800000F0F8FF02B0BDE8F08700BF46F2C853FC
:10AD9000C0F20603185C00EB800340F27C60C1F255
:10ADA000000000EBC30319615A61704746F2C853B3
:10ADB000C0F20603185C00EB800340F27C62C1F233
:10ADC000000202EBC3008160704700BF46F2887347
:10ADD000C0F20603185C00EB400146F2D452C0F208
:10ADE000060202EB01107047062812D846F2C8533B
:10ADF000C0F20603185C00EB800140F27C62C1F2F5
:10AE0000000202EBC1034FF6FF7098844FF001007F
:10AE100070474FF00000704706280ED846F2C8531E
:10AE2000C0F20603185C00EB800140F27C62C1F2C4
:10AE3000000202EBC103988C70474FF0000070478E
:10AE400008B54AF6CD60C0F202004FF00F014FF096
:10AE5000010200F0F5FF4CF2C403C4F20F031A68BC
:10AE600042F00200186046F29C71C0F206010A68C6
:10AE700044F27003C4F200031A6046F2A070C0F2FC
:10AE80000600016844F21402C4F20002116044F2A8
:10AE90001803C4F2000345F6C050186044F20C01D8
:10AEA000C4F200014FF000020A6046F29873C0F24B
:10AEB0000603186844F20401C4F20001086046F277
:10AEC0009472C0F2060213680B6008BD684620F059
:10AED00007018D4601B544F20003C4F200031A785D
:10AEE00042F0010018701AF03DF9BDE801408546B6
:10AEF000704700BF0B4601B3032816D8DFE800F007
:10AF0000020B0211082913D9102914D920298CBF4A
:10AF10004023202311E040F2FF32934228BF134622
:10AF20000BE0402B28BF402307E04FF0000304E074
:10AF30004FF0080301E04FF010031846704700BFC0
:10AF40004FF000034CF20822C2F208024FF0100149
:10AF500011604FF0050262F30F2360F317434CF2C8
:10AF60001020C2F2080003604CF20021C2F2080176
:10AF70000B6813F0100FFBD0704700BF38B50D46BB
:10AF80004FF00004FFF7DCFF4CF20823C2F2080385
:10AF90004FF010021A604FF0010060F30F2465F3C8
:10AFA00017444CF21021C2F208010C604CF200224E
:10AFB000C2F20802136813F0100FFBD038BD00BFB7
:10AFC00038B505464FF00004FFF7BAFF4CF20823EE
:10AFD000C2F208034FF020021A604FF0020060F343
:10AFE0000F2465F317444CF21021C2F208010C60E3
:10AFF0004CF20022C2F20802136813F0200FFBD0BB
:10B000004CF21420C2F20800006838BD2DE9F84F58
:10B010004CF20023C2F20803D3F800B04CF2302007
:10B02000C2F208000768002F53D041F2FC11C1F2B0
:10B0300000010A78012A4CD94FF000044FF00105B5
:10B040004CF2382AC2F2080A41F25829C1F200092A
:10B0500041F28C28C1F200083D4233D0CAF80050BA
:10B060004FEA540619F806304FF04C0000FB0386F7
:10B070004CF20021C2F208010A6812F0200FFBD046
:10B080004CF21423C2F208031868C0F3800114F0D4
:10B09000010F0BD0F36B2BB1306A4FF000011AF0A7
:10B0A000A5FD07E04FF00100706303E04FF00102DF
:10B0B000F2623163F16A09B9726B1AB106F11000DC
:10B0C00013F062F904F10104E4B24FEA4505202CC3
:10B0D000C2D14CF20823C2F20803C3F800B00BF04F
:10B0E0000800C1B2002971D04FF0FE00FFF768FFE1
:10B0F000C4B204F01002D3B26BB141F25420C1F2D9
:10B1000000004FF00101017041F26822C1F200021B
:10B11000106819F08BF914F0010F36D004F0080014
:10B12000C1B2002952D004F00402D3B2B3B141F24B
:10B13000ED41C1F200014FF001030B7041F2FD102F
:10B14000C1F200004FF00002027041F26821C1F22A
:10B150000001086819F06AF9BDE8F88F41F2ED4086
:10B16000C1F200004FF00001017041F2FD13C1F285
:10B1700000034FF001021A7041F26820C1F2000092
:10B18000006819F053F9BDE8F88F04F00203D8B253
:10B19000E0B141F2FC11C1F2000191F90020002A56
:10B1A00014DB41F2ED43C1F200034FF001001870CF
:10B1B00041F2FD11C1F200014FF000020A7041F2AC
:10B1C0006823C1F20003186819F030F9BDE8F88F60
:10B1D000684620F007018D4689B500AFFFF716FFDE
:10B1E000BD46BDE889408546704700BF70B50B4637
:10B1F000A1B34CF20822C2F208024FF48071116030
:10B200004CF24424C2F2080425684FF0010606FA05
:10B2100000F646EA050222604CF24821C2F208011B
:10B2200008604CF24C20C2F20800036019F08AFF5B
:10B230004CF20024C2F20804C0F10405236813F4A0
:10B24000807F04D119F07EFF2A18F92AF6D94CF232
:10B250003421C2F20801086806430E6070BD00BFC9
:10B2600010B54FF04C0303FB00F041F28C21C1F20A
:10B2700000014418405828B3226A4FEA420303F001
:10B28000FE00E168FFF7B2FF216A4FEA410000F1DA
:10B290000102D0B2A168FFF7A9FF41F2FC13C1F28D
:10B2A00000031978081F18BF012060624FF00102E7
:10B2B000A2624FF00003E3622363636304F11000B2
:10B2C00013F062F810BD00BF4CF2C013C4F20F03BC
:10B2D0001A6860F3DF721A60704700BF10B541F260
:10B2E0005823C1F200031A5C40F24473C1F2000318
:10B2F0001B8843FA00F010F0010F30D041F28C238C
:10B30000C1F200034FF04C0000FB023311B198680A
:10B3100018B927E0DA68002A27D01C6A4FEA4403EC
:10B3200000290CBF1946591C4CF2C014C4F20F047A
:10B3300022686FF3DF722260C8B2FFF741FE236814
:10B3400043F000412160C0B200F00202D3B27BB9E9
:10B3500000F0010100290CBF0220032010BD4FF0B6
:10B36000000010BD4FF0000010BD4FF0000010BDF8
:10B370004FF0010010BD00BF10B54CF2C014C4F274
:10B380000F0423686FF3DF7323604FF0410046F230
:10B39000AC71C0F206010978FFF7F0FD206840F0BB
:10B3A0000042226010BD00BF38B54CF2C014C4F298
:10B3B0000F0423686FF3DF7323604FEA400000F14E
:10B3C000010545F04001CDB2284646F2B072C0F208
:10B3D00006021178FFF7D2FD284646F2CC73C0F280
:10B3E00006031978FFF7CAFD206840F0004121608C
:10B3F00038BD00BF38B503464FEA400000F10100F8
:10B40000C0B24CF2C014C4F20F0425686FF3DF75AC
:10B4100025604CF20824C2F20804256845F0800536
:10B4200025604FF0020463F385044CF22823C2F236
:10B4300008031C604CF22423C2F208031A604CF289
:10B440000022C2F20802136813F0800F12D101F13A
:10B4500004014CF21C24C2F208044CF20022C2F295
:10B46000080251F8043C2360136801F1040113F051
:10B47000800FF6D0FFF764FD4FF0FA00FFF760FD94
:10B480004CF2C011C4F20F01086840F000420A609B
:10B4900038BD00BFF0B583B04FEA400E5FFA8EFCB6
:10B4A0004CF2C013C4F20F031C686FF3DF741C600E
:10B4B0004CF20827C2F208073B6843F040043C60A6
:10B4C0004FF0010760F385074CF22820C2F2080014
:10B4D00007604CF22027C2F208073B6813F4006FA4
:10B4E000FBD04CF22020C2F2080007684FEA8753D5
:10B4F0004FEA9357BA4238BF17464CF20020C2F2C7
:10B500000800036813F0400F31D1032A2FD901F14D
:10B5100004034CF21825C2F208054CF20026C2F2D0
:10B520000806A2F10401C1F380042868194643F813
:10B53000040CA2F10402306810F0400F5AD016E05B
:10B540002C68194643F8044CA2F1040422463068E2
:10B5500010F0400F0BD103F104032A68194643F899
:10B56000042CA4F10402346814F0400F57D04CF2BC
:10B570000023C2F20803186810F0400F1ED1EAB190
:10B580004CF21824C2F20804206801904FF0000326
:10B5900002F1FF3404F00104C85403F101039342A3
:10B5A0001ED10BE001A8185CC85403F1010301A8E7
:10B5B000C05CC85403F101039342F3D16046FFF726
:10B5C000BFFC4FF0F200FFF7BBFC4CF2C011C4F21D
:10B5D0000F010A6842F000430B60384603B0F0BD2B
:10B5E000002CDFD001A8185CC85403F1010393427A
:10B5F000D8D1E3E703F10403032AB8D9002C9FD084
:10B600002868194643F8040CA2F10402306810F0CF
:10B61000400FACD103F10403032A91D8A7E703F14B
:10B620000403032A8CD8A2E710B54FF00000FFF7FF
:10B6300017FE4FF00100FFF713FE4FF00200FFF777
:10B640000FFE4FF00300FFF70BFE4FF00400FFF773
:10B6500007FE4FF00500FFF703FE4FF00600FFF76F
:10B66000FFFD4FF00700FFF7FBFD4CF2C014C4F2E2
:10B670000F0423686FF3DF7323604FF0D8004FF09F
:10B680000101FFF77BFC206840F00041216010BD04
:10B69000F8B5054641F28C23C1F200031868002872
:10B6A0004AD0634C41F28C21C1F20001CA6C002ADD
:10B6B00077D004F14C0441F28C26C1F20006D6F892
:10B6C0009870002F70D004F14C0441F28C23C1F229
:10B6D0000003D3F8E400002869D004F14C0441F2DF
:10B6E0008C21C1F20001D1F83021002A62D004F18E
:10B6F0004C0441F28C26C1F20006D6F87C71002F72
:10B700005BD004F14C0441F28C23C1F20003D3F866
:10B71000C801002854D004F14C0441F28C21C1F23C
:10B720000001D1F81422002A4DD004F14C0400F09D
:10B7300069FA4FF0080705E04FF0000741F28C244A
:10B74000C1F200042E7A36B346F2B473C0F2060397
:10B7500053F82660317848B2B0F1FF3F1ED040F276
:10B760004472C1F2000210884BB240FA03F111F0AA
:10B77000010F0DD006F101031E4613F8012B51B243
:10B78000B1F1FF3F0AD040FA01F111F0010FF3D1FE
:10B7900096F900601AE04FF0000617E000F032FA68
:10B7A000F6E74FF00107CDE74FF00207CAE74FF089
:10B7B0000307C7E74FF00407C4E74FF00507C1E7E9
:10B7C0004FF00607BEE74FF00707BBE740F24470B3
:10B7D000C1F200004FF0010303FA06F3028813439D
:10B7E0000380287A6989FFF785FBA060287AA989F8
:10B7F000FFF780FBE06041F25821C1F200018F5554
:10B80000274647F8205B38464FF000014FF01C02F6
:10B8100032F086FF26626868A06304F110004FF0E2
:10B8200006012A683B4612F08FFD3046F8BD00BF86
:10B83000D812001038B54FF0000360F3060363F030
:10B840007F04032915D14CF2C015C4F20F052868F6
:10B850006FF3DF7028604FF0D0002146FFF78EFBBA
:10B860004FF0D0002146FFF789FB296841F00042E4
:10B870002A6038BD70B584B0002879D04CF2C4017C
:10B88000C4F20F010C6844F000450D604CF6F476EC
:10B89000C2F208064FF0FF33336046F2A472C0F2E2
:10B8A000060210684CF6F871C2F208010C680440F8
:10B8B000A042FBD14FF003054CF21016C2F208066D
:10B8C00035604FF064001BF027F94CF6F473C2F2B8
:10B8D00008031A686FF3C3021A604FF00004009463
:10B8E00001944FF00106029620464FF01F012A46B0
:10B8F0002346FDF7BDFC00940194029520464FF0CD
:10B900000E012A462346FDF7B3FC009401944FF044
:10B910000200029030464FF01E012A462346FDF7F2
:10B92000A7FC4BF2D110C0F202004FF00F014FF014
:10B93000180200F085FA4FF0FF314CF23823C2F2C2
:10B94000080319604CF20822C2F2080211604CF29E
:10B950000420C2F208004FF00C0101602046294685
:10B96000FFF768FF4FF0FE003146FFF707FB15E0D9
:10B970004FF000044FF0FE002146FFF7FFFA20468B
:10B980004FF00F014FF0180200F05AFA4CF2C403C6
:10B99000C4F20F031A6842F00040186004B070BD92
:10B9A000F8B54CF2C403C4F20F031A6842F4006005
:10B9B000186046F2E471C0F206010C684CF22005F2
:10B9C000C2F209052C604CF20406C2F2090637687F
:10B9D00017F0010FFBD146F6D003C0F206031A6838
:10B9E0004CF20000C2F2090002604CF20011C4F2F5
:10B9F0000F014FF001040C6046F6C805C0F20605C1
:10BA00002E684CF20807C2F209073E6046F6E803CA
:10BA1000C0F20603196846F2E870C0F20600A0F111
:10BA2000040500F1DC0005F104026C68216002F1FC
:10BA30000405566831608542F5D14CF2A017C4F276
:10BA40000F073B7843F001013970387820F002028B
:10BA50003A703C7824F004053D7046F6CC06C0F2FE
:10BA6000060633684CF20017C2F209073B604FF03C
:10BA700001044CF23001C2F209010C604CF23400B6
:10BA8000C2F209004FF0040202604FF008054CF2C8
:10BA90003806C2F2090635604CF23C03C2F20903D3
:10BAA0001C604CF24001C2F209010D604FF0020629
:10BAB0004CF24400C2F2090006604CF24802C2F2A5
:10BAC00009024FF00D0313604CF24C01C2F2090160
:10BAD0000D604CF25000C2F2090005604FF0030502
:10BAE0004CF25402C2F2090215604CF25803C2F241
:10BAF00009031D6046F2E071C0F2060108684CF2CD
:10BB00000415C2F2090528604CF22802C2F20902AB
:10BB100014604CF2DC13C4F20F0340F605211960E7
:10BB200046F6D400C0F2060005684CF20002C2F2EC
:10BB30000902156046F6E003C0F2060319684CF2EC
:10BB40002005C2F2090529604FF032001AF0E4FF27
:10BB500046F6E400C0F2060002682A604FF0640076
:10BB60001AF0DAFF2B6866F3C8132B6020461AF030
:10BB7000D3FF4CF22406C2F20906346020461AF0C4
:10BB8000CBFF4FF07501316020461AF0C5FF2868E1
:10BB900064F3C810286046F6DC02C0F2060213887F
:10BBA00040F20006CAF2000646EA03310B6820465E
:10BBB0001AF0B2FF46F6D800C0F2060002682A600A
:10BBC0003B6843F4002139604FF47A701AF0A4FF07
:10BBD0003046054A931B48BF03334FF000014FEA3C
:10BBE000A30200F071F8F8BD030000A146F6EC03D3
:10BBF000C0F206031A684EF60C50CEF20000026046
:10BC0000FEE700BF08B5FFF7F1FF00BF51E8002FC6
:10BC1000BFF35F8F41E80003012B3FF4F7AF1046FD
:10BC2000704700BF13461A462DE9F00F092AC0F0ED
:10BC30000980B1E8F80FA0E8F80FA2F10902092A7B
:10BC4000BFF4F7AF4FF00C0303FB02F21D4B1A4495
:10BC5000974600F032B800BF00BF00BF00BF0B68BE
:10BC6000036000F02AB800BF00BF91E8180080E828
:10BC7000180000F022B891E8380080E8380000F0A1
:10BC80001CB891E8780080E8780000F016B891E8D8
:10BC9000F80080E8F80000F010B891E8F80180E8BA
:10BCA000F80100F00AB891E8F80380E8F80300F022
:10BCB00004B891E8F80780E8F807BDE8F00F70478E
:10BCC0001346000052BC020013461A462DE9F00F3D
:10BCD0000B460C460D460E460F46884689468A4658
:10BCE0008B46092AC0F00780A0E8F80FA2F10902EC
:10BCF000092ABFF4F9AF4FF0080303FB02F2144B1B
:10BD00001A44974600F020B800BF00BF046000F05E
:10BD10001BB800BF80E8300000F016B880E8700063
:10BD200000F012B880E8F00000F00EB880E8F001F2
:10BD300000F00AB880E8F00300F006B880E8F007E9
:10BD400000F002B880E8F00FBDE8F00F704713462E
:10BD500004BD0200EFF3118070474FF0000000BFF8
:10BD6000EFF311804FF0800181F3118870474FF09D
:10BD7000000000BF80F31188704700BF30B440F26C
:10BD80000003C0F2000340F2E402C0F20002D01A45
:10BD9000B0F5697F03D2274B934201D324E0FEE73D
:10BDA000254D264C621B22F003054FF0000340F2A4
:10BDB0000002C1F2000240F20001C0F2000105F1F0
:10BDC0000400C5F380045D589D5003F104038342D1
:10BDD00026D109E05C589C5003F104035C58D45010
:10BDE00003F104038342F5D14EF60853CEF200036B
:10BDF00040F20002C1F200021A604FF0B501CBF22E
:10BE00006B1147F6E430C1F2000001604EF61453A6
:10BE1000CEF200031A6842F01001196030BC70477E
:10BE2000002CD7D05C589C5003F104038342D1D13D
:10BE3000DAE700BF0000000004000000E700000097
:10BE400010B4034600283ED002F1100440F2000076
:10BE5000C1F2000040F82430002A0ADA12F10C0F77
:10BE600035DB02F10C024EF61850CEF200001154F0
:10BE70002DE04EF20014CEF200040F299CBF090100
:10BE8000C9B24EF20043CEF20003D1541146002A4B
:10BE9000B8BF02F11F014FEA611004EB80014FF0BF
:10BEA0001F03C8F200031340002B05DA03F1FF3231
:10BEB00062F01F0303F1010358B24FF0010202FACE
:10BEC00000F30B6003E0002AC8DB024CD5E710BC8E
:10BED000704700BF80E100E003460028B8BF00F1D2
:10BEE0001F034FEA63114EF28022CEF2000202EBF2
:10BEF00081024FF01F03C8F200030340002B05DA54
:10BF000003F1FF3060F01F0303F1010358B24FF05B
:10BF1000010101FA00F31360704700BF1EF0040F27
:10BF20000CBFEFF30880EFF3098020E9F00F00F079
:10BF300001B800BF10B5026847F69033C1F20003A4
:10BF40001A604168596082689A60C168D960026964
:10BF50001A614169596182699A61C169D961026A4C
:10BF60001A62416A5962826A9A62C16AD962026B34
:10BF70001A63416B5963826B9A63C16BD96300F199
:10BF8000400018644EF62850CEF2000002685A6451
:10BF900035F040F9002800F0DD8146F6F000C0F2EF
:10BFA000060035F053FA4EF62C54CEF20004236806
:10BFB000002B05DA46F60010C0F2060035F046FA0E
:10BFC0004EF62C51CEF20001086810F0020F05D099
:10BFD00046F61010C0F2060035F038FA4EF6285238
:10BFE000CEF200025478002C63D046F62810C0F23E
:10BFF000060035F02BFA4EF62853CEF2000359789E
:10C0000011F0010F05D046F63810C0F2060035F0E9
:10C010001DFA4EF62850CEF20000427802F00204DB
:10C02000E3B22BB146F65810C0F2060035F00EFA16
:10C030004EF62851CEF20001487800F00402D4B246
:10C040002CB146F67C10C0F2060035F0FFF94EF632
:10C050002853CEF20003597801F00800C2B22AB189
:10C0600046F6A010C0F2060035F0F0F94EF628545E
:10C07000CEF20004637803F01001C8B228B146F68E
:10C08000C010C0F2060035F0E1F94EF62852CEF2AB
:10C090000002547804F08003D9B251B14EF6385002
:10C0A000CEF20000016846F6E010C0F2060035F05E
:10C0B000CDF94EF62852CEF200025488A3B2002BDE
:10C0C0005ED046F60020C0F2060035F0BFF94EF60D
:10C0D0002851CEF20001488810F0010F05D046F635
:10C0E0001020C0F2060035F0B1F94EF62852CEF21B
:10C0F0000002548804F0020399B229B146F63C20AC
:10C10000C0F2060035F0A2F94EF62850CEF200003B
:10C11000428802F00404A3B22BB146F66020C0F2BC
:10C12000060035F093F94EF62851CEF2000148880A
:10C1300000F0080294B22CB146F6A020C0F206002E
:10C1400035F084F94EF62853CEF20003598801F4F5
:10C15000807082B22AB146F6D020C0F2060035F0D7
:10C1600075F94EF62854CEF20004638803F400718A
:10C1700088B228B146F6EC20C0F2060035F066F928
:10C180004EF62852CEF200021478002C54D046F617
:10C190000430C0F2060035F059F94EF62853CEF2BD
:10C1A0000003197811F0010F05D046F61430C0F2E3
:10C1B000060035F04BF94EF62850CEF2000002781A
:10C1C00002F00204E3B22BB146F63430C0F20600AE
:10C1D00035F03CF94EF62851CEF20001087800F017
:10C1E0000802D4B22CB146F64C30C0F2060035F04D
:10C1F0002DF94EF62853CEF20003197801F0100005
:10C20000C2B22AB146F67030C0F2060035F01EF90F
:10C210004EF62854CEF20004237803F08001C8B211
:10C2200050B14EF63452CEF20002116846F6943008
:10C23000C0F2060035F00AF947F69034C1F2000466
:10C24000216A46F6C030C0F2060035F0FFF8616A98
:10C2500046F6D430C0F2060035F0F8F8A16A46F68A
:10C26000E830C0F2060035F0F1F8E16A46F6FC303D
:10C27000C0F2060035F0EAF8216846F61040C0F238
:10C28000060035F0E3F8616846F62440C0F2060087
:10C2900035F0DCF8A16846F63840C0F2060035F00B
:10C2A000D5F8E16846F64C40C0F2060035F0CEF80D
:10C2B000216946F66040C0F2060035F0C7F86169B2
:10C2C00046F67440C0F2060035F0C0F8A16946F6A3
:10C2D0008840C0F2060035F0B9F8E16946F69C40A6
:10C2E000C0F2060035F0B2F8216B46F6B040C0F25D
:10C2F000060035F0ABF8216C46F6C440C0F20600EB
:10C3000035F0A4F8616B46F6D840C0F2060035F06F
:10C310009DF8A16B46F6FC40C0F2060035F096F899
:10C3200047F6D833C1F200031A6846F62050C0F22F
:10C3300006001146126835F089F840F63071C1F2F6
:10C3400000010B6846F63850C0F2060019461A681C
:10C3500035F07CF8FFF756FC10BD00BF00B518F0B3
:10C360006FFB002808BF5DF804FBEFF30981EFF3D2
:10C37000118221E9F40F5DF804EB1EF0100F08BFE5
:10C3800021ED108A41F804ED0B4C2268002A18BFF9
:10C39000516018F0C7FB2268516851F804EB1EF099
:10C3A000100F08BFB1EC108AB1E8F40F82F31188C6
:10C3B00081F3098870470000D87B001008B54CF263
:10C3C0005D30C0F202004FF0FF016FF00102FFF795
:10C3D00037FD08BDF8B507460C461E460799089D6F
:10C3E00014F0030F00D0FEE722B1A4EB8500A0F10A
:10C3F000480401E004F14800012D01D8A16205E0E4
:10C400002A46FDF761F9A7EB8507A7624FF0000305
:10C4100063604FF01130E0624FF0223121634FF042
:10C42000333262634FF04433A3604FF05530E06025
:10C430004FF0663121614FF0773262614FF08833FF
:10C44000A3614FF09930E0614FF0AA3121624FF0C3
:10C45000BB3262624FF0CC33A363E663069820647C
:10C460004FF0807161646FF00202226005F11200EA
:10C47000F8BD00BF62B64EF60453CEF200031A6850
:10C4800042F08050186000BF00B518F0D9FA0028BB
:10C4900008BF5DF804FBEFF30981EFF3118221E996
:10C4A000F40F5DF804EB41F804ED094C2268002A12
:10C4B00018BF516018F036FB2268516851F804EB40
:10C4C000B1E8F40F82F3118881F309887047000006
:10C4D000D87B001006EE900AF8EEE67A00EE101A0D
:10C4E000B8EEC07A9CED056ADCED040A27EE201A4E
:10C4F00007EE861ADCED031A31EE212A82ED002ABE
:10C50000DCED022A9CED013A67EE033A47EEA23ACF
:10C510009CED004A73EE844AC3ED004A704700BFA9
:10C5200041B940F25873C1F20003987E10704FF089
:10C53000000070474FF01400704700BF000000007B
:10C54000F8B507460E46086828F09AFC10A3D3E910
:10C55000002328F0B3FE28F0AFFC28F091FC04463D
:10C560000D46384628F09AFA4FF000024FF00003CB
:10C57000C4F2340328F058FF02460B4620462946F1
:10C5800028F058FD28F098FC3060F8BDAFF300802B
:10C59000666666666666EE3F08B54FF00100187085
:10C5A00071B940F25173C1F200031A7072B94FF0C1
:10C5B000000001460246F6F767F94FF0000008BD9B
:10C5C0004FF000021A704FF0140008BD4FF0000049
:10C5D00008BD00BF00B58BB040F25873C1F2000334
:10C5E00093ED005A93ED044AD3ED035AD3ED026A5A
:10C5F000D3ED014A93ED056A9FED487A65EE877A9F
:10C6000027EEA60A05EE040A64EE873A03EE860AD0
:10C6100065EE070A06EE600A24EE071A06EEC10A66
:10C6200005EEE40A66EE071A34EE613A83EE002A5C
:10C630008DED092A66EE872A32EEE47AC7EE007A9B
:10C64000CDED087A24EE264A14EE864AC4EE004A5E
:10C65000CDED074A71EEE53AC3EE800ACDED060A4C
:10C6600035EE621AC1EE001ACDED051A25EE065A16
:10C6700015EEA65AC5EE005ACDED045A0DF1100C78
:10C680004FF0EB004FF0830102AA6B46FFF722FF49
:10C690000DF1100C4FF0F5004FF08D0103AA01AB26
:10C6A000FFF718FFDDED036A9DED026A36EE660ABC
:10C6B0008DED020A9DED013A9DED002A72EE432AAE
:10C6C000CDED002A10EE100A2DF0D2FD28F0D8FB97
:10C6D0004FF000024FF00003C3F6E07328F0AAFC0D
:10C6E00028F02CFB40F27871C1F20001086000983C
:10C6F0002DF0BEFD28F0C4FB4FF000024FF0000308
:10C70000C3F6E07328F096FC28F018FB40F6D00240
:10C71000C1F2000210600BB000BD00BF00000000BD
:10C7200030B585B040F25874C1F200042046FBF7E2
:10C73000A5FF258B4FF0000323834FF6FF702146A2
:10C740004FF01C021AF000FAA84214BF002001208A
:10C75000C1B2A07609B1FFF73DFF4FF0000300938F
:10C7600040F27C72C1F2000201924FF05000029040
:10C7700046F6A850C0F206004FF006014CF6517282
:10C78000C0F2020217F08AFE4FF00A0046F674511A
:10C79000C0F2060140F6C002C1F200021BF070FFB9
:10C7A00005B030BD000000002DE9F04F2DED088BE5
:10C7B000BFB00592002940F0A2834FF0140008900A
:10C7C0004FF0F00209924FF4E6710A910B904FF08E
:10C7D00088040C944FF0FC050D954FF07E500146F7
:10C7E0004FF000021346F7F7F9FA0B9E089F1A97CD
:10C7F0001B9609981C901D960A9A1E921F960C9BD8
:10C800002097219322902393249225930D99269784
:10C810002791289029912A922B914FF07F40F6F78B
:10C8200001F84FF00000F4F739FD00F1050446F679
:10C83000B055C0F2060500954FF000004FF005011D
:10C8400022464FF0FF33F4F76BFE4FF00000F4F791
:10C8500011FD221846F6C856C0F2060600964FF0A3
:10C8600000004FF005014FF0FF33F4F759FE4FF091
:10C87000000001464FF0FF321346F5F797FF41F2F3
:10C88000883017F069FF40F25077C1F2000738781E
:10C89000002800F03B834FF0320540F25074C1F2A3
:10C8A0000004284617F058FF2278002AF9D12DE31A
:10C8B000039850F8044F03903EAA02EBC40353F8C8
:10C8C000901C1AAE029FB95153F88C4C0298321842
:10C8D00054604FF07F40F5F7A5FF1AAB0299CE5890
:10C8E0004FF0FF3700974FF00100019006F1FF3045
:10C8F00004F1FF314FF002021346F6F7DDFE4FF070
:10C900000000F4F7CBFC04F10A0216184FF0000007
:10C91000F4F7BAFC00EB40018B19B3F5887F88BFB0
:10C92000C1EB040646F6EC54C0F206040094049FE2
:10C9300057F8040F049701904FF00000014632466B
:10C940004FF0FF33F4F7ECFD4FF0000001464FF0DD
:10C95000FF321346F5F72AFF4FF0320740F2487BCB
:10C96000C1F2000B40F24C7AC1F2000A8DED06BA1A
:10C970008DED07BA2A782AB1384617F0EDFE2E78E9
:10C98000002EF9D1297829B9384617F0E5FE2B7821
:10C99000002BF9D0DBF8000006A9FFF7D1FDDAF88B
:10C9A000000007A9FFF7CCFDDDED067A9DED079AA3
:10C9B00029EE099A07EEA79A4FF0010840F6CC0439
:10C9C000C1F200044FF000092DE0DBF8000006A9D9
:10C9D000FFF7B6FDDAF8000007A9FFF7B1FD08F18F
:10C9E0000108DDED06AA9DED07AA6AEE0A9A4AEE55
:10C9F000AA9AB8F1640F14D9F4EEC99AF1EE10FABC
:10CA0000CCBF89EE299A89EE899A19EE100A28F08E
:10CA100037FA53EC182B28F0B1FEA0B9B0EE699AA2
:10CA200001E0B0EE699A84F80090207838B94FF0B0
:10CA30000A06304617F090FE2278002AF9D02978AD
:10CA4000002993D0C1E72CABFDEEEAAA1AEE900ABA
:10CA5000029EF0509A19BDEECAAA82ED01AA4FF0CB
:10CA600001001CF0E7FD06F1080602960399F24C5E
:10CA7000A1427FF41DAF9FEDF10A2C9D01EE905A6B
:10CA8000F8EEE16A76EE800A2D9B02EE103AB8EEDF
:10CA9000C26A36EE001A1A9802EE900AF8EEE24ADE
:10CAA00074EE808A1B9E03EE106AF8EEC35A35EED0
:10CAB000808A05FB05F204EE102AF8EEC43A73EE04
:10CAC000809A03FB05F105EE101AB8EEC57A37EE31
:10CAD000009A03FB03F407EE904AF8EEE71A31EEF2
:10CAE000805A00FB05F206EE902AB8EEE62A72EEB6
:10CAF000001A00FB03F006EE100AF8EEC62A32EE2A
:10CB0000803A06FB05F504EE905AF8EEE45A35EE4D
:10CB1000802A06FB03F304EE103AF8EEC43A33EE33
:10CB2000800A2E9D07EE105AF8EEC77A70EEA70A1B
:10CB30002F9B06EE903AB8EEE66A31EE061A1C9E7E
:10CB400002EE906AF8EEE24A78EEA48A1D9905EEAC
:10CB5000901AB8EEE54A38EE048A05FB05F403EEB8
:10CB6000904AB8EEE37A79EE879A03FB05F207EE76
:10CB7000902AF8EEE76A39EE269A03FB03F006EEF8
:10CB8000100AF8EEC62A35EE225A06FB05F404EE2A
:10CB9000904AF8EEE45A71EEA51A06FB03F604EE8D
:10CBA000106AF8EEC43A73EE235A01FB05F503EE62
:10CBB000105AB8EEC37A32EE073A01FB03F502EEE3
:10CBC000105AF8EEC27A30EE270A309A06EE902A12
:10CBD000B8EEE66A70EE860A319B02EE903AF8EE05
:10CBE000E24A31EE241A1E9804EE100AF8EEC43A16
:10CBF00078EEA38A1F9907EE101AB8EEC72A38EE0E
:10CC0000028A02FB02F407EE904AF8EEE76A79EE38
:10CC1000A69A03FB02F606EE106AF8EEC62A39EE73
:10CC2000229A03FB03F504EE905AB8EEE44A75EE3F
:10CC3000043A00FB02F405EE104AB8EEC57A31EE74
:10CC4000874A00FB03F001EE900AB8EEE12A75EE88
:10CC5000821A01FB02F205EE902AF8EEE57A73EEF5
:10CC6000275A01FB03F303EE103AF8EEC36A30EEE5
:10CC7000260A329A06EE102AF8EEC62A70EEA20AAA
:10CC8000339B04EE903AB8EEE45A31EE051A209E3A
:10CC900007EE106AB8EEC72A78EE828A219907EE6D
:10CCA000901AB8EEE73A38EE038A02FB02F506EE78
:10CCB000905AB8EEE66A79EE869A03FB02F402EE29
:10CCC000904AF8EEE24A39EE249A03FB03F005EEAF
:10CCD000100AB8EEC57A73EE873A06FB02F502EE4B
:10CCE000105AF8EEC27A34EE274A06FB03F603EE3A
:10CCF000106AF8EEC36A31EEA65A01FB02F201EEA9
:10CD0000902AB8EEE16A75EE866A01FB03F205EE41
:10CD1000902AF8EEE52A70EE225A349D359B22982F
:10CD2000239903FB05F400EE104AF8EEC04A34EEF6
:10CD3000899A07EE105AB8EEC72A72EE200A07EE5B
:10CD4000903AB8EEE73A33EE011A01EE900AB8EEE7
:10CD5000E16A76EE288A02EE901AB8EEE20A30EE28
:10CD6000082A05FB05F608EE106AF8EEC84A74EECC
:10CD7000A99A03FB03F207EE102AF8EEC77A77EEC2
:10CD8000A33A00FB05F403EE104AF8EEC31A31EEA5
:10CD9000840A00FB03F004EE100AB8EEC46A36EE13
:10CDA000055A01FB05F502EE905AB8EEE28A78EEDC
:10CDB000264A89EEA06AC9EE016A89EE203AC3EEDE
:10CDC000812A80EE200A85EE018A84EEA04A01FBCA
:10CDD00003F509EE105AF8EEC99A79EEA55AC5EE98
:10CDE000813AF1EE047A80EEA77AC1EE275AC8EEB6
:10CDF000A74A82EE275A36EE472A32EEE51A76EE39
:10CE0000C71A73EE650A61EEA07A52EE017A30EE2F
:10CE1000649A78EE648A40F25874C1F2000460EEBD
:10CE2000A89A51EE099AC9EEA79AC4ED009A21EE8C
:10CE3000899A12EE289A03E0886E0600000000002E
:10CE400089EE279A84ED019A66EEA48A58EE078A45
:10CE500020EE079A16EE249A62EE894A43EE284A9B
:10CE600026EE088A16EE808A45EE884AC4EEA74A66
:10CE7000C4ED024A34EE450A73EEC54A60EEA40AD8
:10CE800051EE000AC0EEA70AC4ED030A61EE801A53
:10CE900052EE241A81EEA70A84ED040A66EE854A52
:10CEA00053EE874A24EE077A16EE057A62EE872A59
:10CEB00043EE242A26EE236A16EE846A45EE862A7D
:10CEC00082EEA73A84ED053A4FF0000525834FF036
:10CED0000106A6764FF6FF7021464FF01C0219F0AE
:10CEE00033FE20832046FBF7C1FBFFF773FB4FF0B7
:10CEF0007F40F5F797FC059C267028461BE04FF015
:10CF00000003059C23704FF0140014E046F678638C
:10CF1000C0F20603A3F1040103910B4E04964FF0F7
:10CF2000000702979FED09BA40F25075C1F2000563
:10CF30009FED038BBCE43FB0BDEC088BBDE8F08FE8
:10CF40001EA7E8482EFFEF3F4C6D060000000000D2
:10CF50002DE9F04F85B04FF0000303931D464FF0CD
:10CF6000050411E0204617F0F7FB039800F10100DB
:10CF70000390B0F5FA6F07D140F27471C1F200016D
:10CF80004FF001020A700BE028462946FBF7A6FB8A
:10CF90000028E7D104E04FF0320017F0DDFB0CE091
:10CFA00040F2587AC1F2000A40F2787BC1F2000BDD
:10CFB00040F6D006C1F2000601964FF0000001468F
:10CFC000FBF78CFB0028E6D04FF0000426462546F0
:10CFD00003E03E4645464FF0010403A802A9FBF7D3
:10CFE0007DFB814604F10104E4B203982D18029BF5
:10CFF000F61895FBF4F896FBF4F79AF81A10E9B1D5
:10D000004045B4BFC0EB0800C8EB0000BB42B4BF52
:10D01000C3EB0703C7EB0303DBF8002090424CDCB3
:10D02000019801688B4248DC4FF01E0017F094FB1A
:10D03000B9F1000FC1D0042CCFD902E0B9F1000F33
:10D04000BBD040F24874C1F20004C4F8008040F242
:10D050004C75C1F200052F6040F25073C1F200031D
:10D060004FF001061E7040F6CC02C1F200021670AD
:10D070001F78002FA1D04FF0320940F25074C1F256
:10D08000000440F24877C1F2000740F24C76C1F24A
:10D0900000061546484617F05FFB03A802A9FBF7F8
:10D0A0001DFB207003983860029931604FF0010336
:10D0B0002B702278002AEDD17FE74FF01E0017F089
:10D0C0004BFBB9F1000F84D177E700BF2DE9F8439E
:10D0D0002DED028B05460C4640F27473C1F200033D
:10D0E000187848B140F27470C1F200004FF00003AC
:10D0F00003704FF00200B7E040F25071C1F200013E
:10D10000087840F6CC02C1F2000213789BB90028DF
:10D1100000F0AA802DB140F25472C1F200021368EF
:10D120002B60002C00F0A08040F6BC01C1F2000191
:10D130000A68226098E040F6CC03C1F200034FF089
:10D14000000C40F25077C1F2000740F24870C1F283
:10D15000000040F24C71C1F2000183F800C03E783B
:10D16000D0F80090D1F800801A78002AF5D140F26A
:10D170005873C1F20003987E002861D007EE909AA0
:10D18000B8EEE78A00EE108AF8EEC08A40F25877CF
:10D19000C1F20007D7ED000A97ED017A28EE871A51
:10D1A00008EE201AD7ED021A31EE212A12EE100AEB
:10D1B00027F066FE4FF000024FF00003C3F6E07365
:10D1C00027F038FF27F0BAFD804640F25471C1F2D3
:10D1D00000010860D7ED032A97ED043A68EE838AD0
:10D1E00048EE228AD7ED053A38EEA34A14EE100A2B
:10D1F00027F046FE4FF000024FF00003C3F6E07345
:10D2000027F018FF27F09AFD024640F6BC03C1F252
:10D210000003186040F25170C1F20000017879B14A
:10D220002EB14FF001004146F5F72EFB09E04FF01B
:10D23000000001460246F5F727FB4FF0000013E01F
:10D240007EB12DB140F25472C1F2000213682B601E
:10D250004CB140F6BC00C1F20000016821603046CC
:10D2600002E0304600E03046BDEC028BBDE8F883BA
:10D2700000F5E07003688B4203D842689B1899421E
:10D2800002D380680028F5D1704700BF82B040F615
:10D29000AC23C1F200031868F0B940F6AC23C1F228
:10D2A00000034FF480529A605A604FF0FF31D9600A
:10D2B0004FF4001018614FF000025A6140F6D4019B
:10D2C000C1F20001C1F8BC2101A880F0553222F062
:10D2D000070141F0080018604FF0010002B07047EC
:10D2E00001F1080313F0070F1ABF5B4203F00703B5
:10D2F0000023C918D21A8161C26042F001034B6059
:10D3000089184FF028024A6040F6AC23C1F20003AE
:10D310001969C161704700BF2DE9F04104460D460F
:10D3200040F6AC23C1F20003186808B9FFF7AEFF5E
:10D3300015F1410F55D8A169002955D005F12805EF
:10D34000E668B54257D240F6AC22C1F20002D2F8EC
:10D3500008802046FFF78CFF0746C16811F0080FD0
:10D3600049D1464406F1FF335D1BB5FBF8F000F1EF
:10D37000FF3208FB02F64FF6FE71C7F6FF718E42D0
:10D3800088BFC8F100464FF00000F6F70DFF3D687A
:10D390007B68ED1885422ED1C6F10000F6F704FF38
:10D3A00006464FF00000F6F7FFFEB6F1FF3F22D031
:10D3B000854220D92D1A1ED07B68581B7860D4F87E
:10D3C000B021511BC4F8B011E3682046A1695A1B73
:10D3D000FFF786FF0AE04FF0FF31E1614FF00005F3
:10D3E00004E04FF0000501E04FF00005281C18BFD5
:10D3F0000120BDE8F081E068E2699042EBD84FF08F
:10D400000005F3E72DE9F84306460C46154601EB07
:10D4100002084B6813F0010F40F0C6800A6813F051
:10D42000030F00F071828C1AAD1800698442C0F0BD
:10D43000B78071698C4200F0A0804FEAD2021F2AA7
:10D4400025D8A368E76806EBC20C0CF1280C6345ED
:10D4500006D0984200F24282D9688C4240F03E8267
:10D460009F4208D14FF0010303FA02F2316821EA2A
:10D470000201316098E0674506D0B84200F231827F
:10D48000B868844240F02D82DF60BB608CE0D4F845
:10D490001890E768BC420DD0A368984207D8DA68B4
:10D4A000944200F0218202E0DF60BB601FE0F6F7EB
:10D4B000A9FE1CE004F11401676937B904F11001F9
